:0200000460009A
:100000004643464200000156000000000103030081
:1000100000000000000000000000000000000000E0
:1000200000000000000000000000000000000000D0
:1000300000000000000000000000000000000000C0
:1000400000000000010408000000000000000000A3
:100050000000800000000000000000000000000020
:100060000000000000000000000000000000000090
:100070000000000000000000000000000000000080
:10008000EB04180A063204260000000000000000FD
:10009000050404240000000000000000000000002F
:1000A0000000000000000000000000000000000050
:1000B0000604000000000000000000000000000036
:1000C0000000000000000000000000000000000030
:1000D00020041808000000000000000000000000DC
:1000E0000000000000000000000000000000000010
:1000F0000000000000000000000000000000000000
:10010000D8041808000000000000000000000000F3
:100110000204180804200000000000000000000095
:1001200000000000000000000000000000000000CF
:10013000600400000000000000000000000000005B
:1001400000000000000000000000000000000000AF
:10015000000000000000000000000000000000009F
:10016000000000000000000000000000000000008F
:10017000000000000000000000000000000000007F
:10018000000000000000000000000000000000006F
:10019000000000000000000000000000000000005F
:1001A000000000000000000000000000000000004F
:1001B000000000000000000000000000000000003F
:1001C000000100000010000001000000000000001D
:1001D000000001000000000000000000000000001E
:1001E000000000000000000000000000000000000F
:1001F00000000000000000000000000000000000FF
:10020000FFFFFFFFFFFFFFFFFFFFFFFFFFFFFFFFFE
:10021000FFFFFFFFFFFFFFFFFFFFFFFFFFFFFFFFEE
:10100000D100204327140060000000000000000011
:10101000201000600010006000A4016000000000CB
:101020000000006000B0010000000000FFFFFFFFB3
:10103000FFFFFFFFFFFFFFFFFFFFFFFFFFFFFFFFC0
:10104000FFFFFFFFFFFFFFFFFFFFFFFFFFFFFFFFB0
:10105000FFFFFFFFFFFFFFFFFFFFFFFFFFFFFFFFA0
:10106000FFFFFFFFFFFFFFFFFFFFFFFFFFFFFFFF90
:10140000884207D0904205D251F8043B40F8043B93
:101410008242F9D87047884204D2002340F8043B46
:101420008142FBD870472DE9F843644A644B5A6403
:10143000644A1A644FF42A029A63634B9D46BFF3D1
:101440004F8FBFF36F8F00F019FA604B082260498D
:101450006048C3F85421604AFFF7D2FF5F4A6049F1
:101460006048FFF7CDFF60496048FFF7D4FF4FF4B5
:1014700070025F4B5F491A6000235F4A42F82310F5
:1014800001335D4DB02BF9D15C4B80215C4A03F8F0
:10149000011B9342FBD14D4C4FF08037594A5A4BB8
:1014A000DFF89C91DFF89C811D60C4F80471C4F8DA
:1014B0000091C4F8F470C4F8F0801368534E43F4FC
:1014C000E02313604FF0FF32F36923F07F0343F012
:1014D0004003F361736A23F07F0343F040037362B8
:1014E000374B9A66DA661A675A6700F0CAF9484BB2
:1014F0006322AB63474BEB630025474B1A60032223
:101500005D6043F8042C454AC3F80C2D444A136827
:1015100043F080731360434A136843F00103136080
:10152000414B1A68414B1A6000F064FBC4F8047127
:101530003F48C4F80091C4F8F470C4F8F08000F09B
:10154000E3FCF36E43F44053F3663A4B1D60C3F87B
:101550000851C3F81851C3F82851C3F8385103F59E
:10156000A0239A6BD20708D4334A5A6542F6156213
:101570001A659A6B42F001029A639A6842F001126E
:101580009A6000F0EDF900F08DFC00F0C5FC00F071
:101590005FFB00F074F9294A1368284C132BFBD920
:1015A00000F0E4FB2368B3F5967FFBD300F068F905
:1015B00000F0B6FC00F0A4FC30BFFDE7BFAAAAAA69
:1015C00000C00A40070020000080062000800D4077
:1015D0006454006000000000900E0100C03E002036
:1015E000F86201600000002020870120C03E00203A
:1015F00088ED00E051E30000003C002000E400E042
:10160000A0E400E024ED00E008ED00E000C00F40A1
:1016100039F500003DF5000014E000E00000202056
:10162000FCED00E0001000E0041000E0047B00206E
:10163000002CA330004008400000C056087B00206A
:101640001B1018200C0D1113F8B58F005A4B0C46C7
:1016500038461A6000F06CFC584B054618601E4670
:1016600020B95749574800F067FCF8BD3A460021B9
:1016700000F066FC25F01F033D44BFF34F8F524A34
:10168000136020339D42FBD8BFF34F8FBFF36F8FA2
:101690004E4B32681A604E4A4E4B1C80D36F43F457
:1016A0004023D3674C4B4D4A1A674FF43162C3F85D
:1016B000802042F21072C3F890201A6F22F48052F8
:1016C0001A67196F444A0029FBDAD2F870310126F3
:1016D00043494FF4803523F40003424823F4004388
:1016E000C2F87031136F23F48033136702F51032A0
:1016F000D36923F4406343F40063D361936A23F412
:10170000FF7323F0010343F079039362A2F5A02253
:10171000536823F4002323F0070343F400235360AA
:101720000022314B1A66DE60196130495D619861B3
:10173000D961C3F8E020C3F88C6006F1E066C3F815
:101740009060C3F89450C3F898000320C3F89C102D
:101750002749C1F82801C1F82401C1F88001D3F854
:101760008810244841F01041C3F88810224999603C
:101770002249C1F8200122484FF08075056080F8A9
:1017800083237F201F4A10701F4AC1F85821D0219F
:101790001E4A0C4811704021A2F23E3211609A6834
:1017A0001B4942F480729A6000F0CEFB2146054846
:1017B00000F0CEFBF8BD00BFE46400200041002033
:1017C0000C3600207039002070EF00E040650020EA
:1017D00000C00F40167B002000800D401B20110030
:1017E000010000471B1F010000403840001F1F1F61
:1017F00000801F403100000001000090003C0020EC
:1018000004E100E038E400E08501000046E400E087
:101810002D360020024B186808B100F09DBB7047C0
:10182000004100200004084B012200F47020C3F89E
:10183000A010C3F8A400C3F8B0205A69D207FCD5A1
:101840000122014B5A61704700402A40094B0A4A65
:10185000C3F8A000C3F8A4200122C3F8B02059693E
:10186000044AC907FBD5D2F80001212380B2536195
:10187000704700BF00402A400400030070477047D3
:10188000704710B5214A0020214C102321492060C7
:101890001360214B19601121116020491960122138
:1018A00011601F4919601F4911601F4919601F49C4
:1018B00011601F4919601F4941F0150111601E494F
:1018C000196001F181510D3111601C4919601C49E9
:1018D00011601C4919601C4911601C4919601C49A0
:1018E00011601C4A1A6001232360BFF34F8FBFF3BE
:1018F0006F8F194B1860BFF34F8FBFF36F8F174A6D
:10190000136843F44033136010BD00BF9CED00E04A
:1019100094ED00E03F000010A0ED00E0250008037A
:10192000090010001300200021000207140000200D
:1019300025000813208701200900001027000B1341
:101940001700004033001013180000602F000B0731
:10195000190000702F000B1350EF00E014ED00E0B1
:1019600073B58F4B4FF400548E4A8F49C3F85C22F5
:10197000C3F8601248F20C71C3F86422A2F5304239
:10198000C3F8682202F5E042C3F86C22C3F8702263
:10199000C3F87422C3F878221822DA661A675A67E5
:1019A0009A67DA67C3F88020C3F88420C3F88820D8
:1019B0000122C3F82C27C3F83027C3F83427C3F813
:1019C0003827C3F83C27C3F85027784A936923F097
:1019D000604323F4407343F0204343F44073936126
:1019E000D2F8843043F00C03C2F88430704B1A688C
:1019F00042F002021A601A6811406E4A0A436E49A8
:101A00001A604FF0FF325A6002F57702886802F5DB
:101A10006052024042F000529A60DA6822F0780286
:101A2000DA60664A186A024042F0004242F0400220
:101A30001A62624A186A0240614842F0004242F06B
:101A400040025A625F4A9A62DA62D1F8B82022F004
:101A50003F0242F00102C3F8B820D1F8BC2040F2A6
:101A6000056122F03F0242F00102C3F8BC200022CF
:101A70001A611C661867C3F880105C665867C3F863
:101A800084101968504821F0020119604F4999618A
:101A90000221D9614E4941F8042B8142FBD11A68D9
:101AA00042F001021A60424A1468414B14F00104EA
:101AB000FAD1464A0226214620469A6140F2F56252
:101AC000DE61C3F8002240F26642C3F8102240F201
:101AD0009942C3F820223F4AC3F8302242F2014221
:101AE000C3F8342240F23542C3F840223A4AC3F8E0
:101AF00050223A4AC3F85422394AC3F8602242F2CB
:101B00000122C3F86422FFF78DFE21460120FFF772
:101B100089FE21463046FFF785FE2046FFF796FEF8
:101B200045F60D530546984231D121460420FFF772
:101B300079FE20464FF400012A4CFFF773FE4FF464
:101B400000010120FFF76EFE4FF400013046FFF761
:101B500069FE4FF40000FFF779FEA84207D14FF469
:101B600000010420FFF75EFE1023237001E008232C
:101B700023701D4900231D4A2078521A0093012327
:101B800002EB00521A4800F0CFF902B070BD1022EB
:101B90002146174802B0BDE8704000F0D1B900BF3F
:101BA00000801F40F9B00100F910010000C00F4093
:101BB00000402A401200FFFF00802A4000FFF07C16
:101BC00063000200FF000F8300432A40F05AF05ADE
:101BD00000422A409F041830EB06180A06320126FC
:101BE0003806180A478600200000007000000070C8
:101BF000C4860120F0B5154B40204FF480314FF4DE
:101C000080544FF400554FF4404643F242071A699E
:101C100012F0020F03D09E6159619F61F7E712F441
:101C2000005F01D15D61F2E712F4805F01D15C6178
:101C3000EDE7002AEBDA12F4803F01D09961E6E784
:101C4000520601D45861E2E7F0BD00BF00800D40AC
:101C5000394AB3EE096A394813689FED395A23F0BF
:101C6000010310B513600323364C1361364BD3F8D0
:101C7000E030D9B2016007EE901AC3F30B201B0DC0
:101C8000B8EEE77A314907EE900A2060F8EEE76A8D
:101C900007EE903A37EE455A2D4BF8EEE77A37EEDD
:101CA000466A77EEE67A81ED006A25EE275AC3EDA3
:101CB000007A1368C5EE065A75EEA65AFCEEE55A90
:101CC00015EE901ADFED235A37EE657A43EA015399
:101CD000136027EE277A204B66EE277AD2F8101190
:101CE000C7EE065A35EEA67ABCEEC77A17EE100A92
:101CF00087EE867A03EA00430B43C2F81031D2F82C
:101D0000101177EE267AFCEEE77A17EE903AC3F3DD
:101D10000B030B43C2F81031136843F00203136046
:101D200000220E4B1A700E4A0E4BC3F840210122BE
:101D30000D4B1A6010BD00BF80810D40F47A002069
:101D40000000AA42F07A002000441F40F87A0020E8
:101D5000FC7A00200000B4420000FF0F40E400E0E5
:101D6000F5E40000003C002008E100E038B540F652
:101D700061722D4BC3F8202100F0F2F82B4A2C4958
:101D8000D2F8803043F00303C2F8803040F20442BE
:101D9000284BC3F86021284A1068014019B9D3F8CC
:101DA000A811890718D04FF000415163D3F84021A2
:101DB00042F00202C3F840211E4AD2F840319B078C
:101DC000FBD44FF400321D4B19201A604FF0004233
:101DD000194B9A6300F09CF8174B00214FF080429A
:101DE000174D144C9A63284619600A234FF4207249
:101DF000C4F8A83100F0A4F84FF48103114A2B6015
:101E00004FF480032B6440F24313C4F85851C4F8D4
:101E100048310D4BC3F804220C4B4FF400321A60CA
:101E20000123C4F8403138BD00800D4000C00F4090
:101E3000001C1E0000002E4000900D408CE200E0CF
:101E400000000020B1E70000003C00200CE100E0B1
:101E500008B50E4B1B6E9B0701D4FBBE16E072B695
:101E600000220B4BC3F84021A3F50D13094A1A6455
:101E7000A3F1FF53A3F52B239D46BFF34F8F064BD2
:101E800006480360064B1B689B68984700441F4048
:101E900000002E4003002000000012EB00802020F4
:101EA0001C0020000F4BDA6E42F44032DA66DA6E24
:101EB00042F44072DA66A3F5603340F237625A6446
:101EC000A0229A649A6C1206FCD4074B40F2376247
:101ED0005A64A0229A649A6C12F08002FBD1034BE0
:101EE0001A70704700C00F4000800C403E860020F2
:101EF000F8B500BFF8BC08BC9E4670470000000063
:101F00005FF800F01DFA00005FF800F035FB0000FC
:101F10005FF800F031E200005FF800F071FE0000B1
:101F20005FF800F0E1FF00005FF800F02FFF000015
:101F30005FF800F02D0001005FF800F0A10C000038
:101F40005FF800F091E100005FF800F0850C000000
:101F50005FF800F0B50C00005FF800F03D000100F4
:101F60005FF800F00DED0000250200008D1D00005F
:101F7000ED3D000095430000454C000065810000E8
:101F80001C224A564C201E001824427E4242420027
:101F90007C22223C22227C001C22404040221C0049
:101FA00078242222222478007E40407840407E001F
:101FB0007E404078404040001C22404E42221C009F
:101FC0004242427E424242001C08080808081C00A7
:101FD0000E0404040444380042444870484442005B
:101FE0004040404040407E0042665A5A42424200D1
:101FF0004262524A46424200182442424224180099
:102000007C42427C40404000182442424A241A004C
:102010007C42427C484442003C42403C02423C00FC
:102020003E080808080808004242424242423C007A
:1020300042424224241818004242425A5A66420040
:1020400042422418244242002222221C080808008E
:102050007E02041820407E003C20202020203C00EE
:102060000C10103C10706E003C04040404043C008E
:1020700000081C2A08080808000010207F20100013
:102080000000000000000000080808080000080028
:10209000242424000000000024247E247E24240024
:1020A000081E281C0A3C080000626408102646002E
:1020B000304848304A443A0004081000000000004C
:1020C0000408101010080400201008080810200050
:1020D000082A1C3E1C2A08000008083E08080000C8
:1020E00000000000000808100000007E0000000052
:1020F0000000000000181800000204081020400032
:102100003C42465A62423C000818280808083E0033
:102110003C42020C30407E003C42021C02423C0029
:10212000040C14247E0404007E4078040244380029
:102130001C20407C42423C007E42040810101000EB
:102140003C42423C42423C003C42423E0204380097
:102150000000080000080000000008000008081047
:102160000E18306030180E0000007E007E00000067
:1021700070180C060C1870003C42020C1000100085
:1021800000000000FF000000081C3E7F7F1C3E0096
:102190001010101010101010000000FF00000000C0
:1021A0000000FF000000000000FF00000000000031
:1021B0000000000000FF0000202020202020202020
:1021C000040404040404040400000000E0100808EF
:1021D000080808040300000008080810E0000000D8
:1021E00080808080808080FF804020100804020171
:1021F0000102040810204080FF8080808080808061
:10220000FF01010101010101003C7E7E7E7E3C0058
:10221000000000000000FF00367F7F7F3E1C0800AA
:102220004040404040404040000000000304080897
:102230008142241818244281003C424242423C0020
:10224000081C2A772A08080002020202020202027F
:10225000081C3E7F3E1C080008080808FF08080804
:10226000A050A050A050A05008080808080808086E
:102270000000013E54141400FF7F3F1F0F070301AD
:102280000000000000000000F0F0F0F0F0F0F0F0CE
:1022900000000000FFFFFFFFFF0000000000000043
:1022A00000000000000000FF80808080808080802F
:1022B000AA55AA55AA55AA5501010101010101011A
:1022C00000000000AA55AA55FFFEFCF8F0E0C0800F
:1022D0000303030303030303080808080F0808089F
:1022E000000000000F0F0F0F080808080F00000083
:1022F00000000000F8080808000000000000FFFFD0
:10230000000000000F08080808080808FF00000087
:1023100000000000FF08080808080808F808080876
:10232000C0C0C0C0C0C0C0C0E0E0E0E0E0E0E0E0AD
:102330000707070707070707FFFF00000000000067
:10234000FFFFFF00000000000000000000FFFFFF93
:1023500001010101010101FF00000000F0F0F0F0B7
:102360000F0F0F0F0000000008080808F800000019
:10237000F0F0F0F000000000F0F0F0F00F0F0F0FA1
:10238000E3DDB5A9B3DFE1FFE7DBBD81BDBDBDFF87
:1023900083DDDDC3DDDD83FFE3DDBFBFBFDDE3FF45
:1023A00087DBDDDDDDDB87FF81BFBF87BFBF81FF4F
:1023B00081BFBF87BFBFBFFFE3DDBFB1BDDDE3FFAF
:1023C000BDBDBD81BDBDBDFFE3F7F7F7F7F7E3FF87
:1023D000F1FBFBFBFBBBC7FFBDBBB78FB7BBBDFFB3
:1023E000BFBFBFBFBFBF81FFBD99A5A5BDBDBDFF1D
:1023F000BD9DADB5B9BDBDFFE7DBBDBDBDDBE7FF35
:1024000083BDBD83BFBFBFFFE7DBBDBDB5DBE5FF60
:1024100083BDBD83B7BBBDFFC3BDBFC3FDBDC3FF90
:10242000C1F7F7F7F7F7F7FFBDBDBDBDBDBDC3FFF2
:10243000BDBDBDDBDBE7E7FFBDBDBDA5A599BDFF0C
:10244000BDBDDBE7DBBDBDFFDDDDDDE3F7F7F7FF9E
:1024500081FDFBE7DFBF81FFC3DFDFDFDFDFC3FF1E
:10246000F3EFEFC3EF8F91FFC3FBFBFBFBFBC3FF5E
:10247000FFF7E3D5F7F7F7F7FFFFEFDF80DFEFFFB9
:10248000FFFFFFFFFFFFFFFFF7F7F7F7FFFFF7FF84
:10249000DBDBDBFFFFFFFFFFDBDB81DB81DBDBFF68
:1024A000F7E1D7E3F5C3F7FFFF9D9BF7EFD9B9FF3E
:1024B000CFB7B7CFB5BBC5FFFBF7EFFFFFFFFFFF00
:1024C000FBF7EFEFEFF7FBFFDFEFF7F7F7EFDFFFDC
:1024D000F7D5E3C1E3D5F7FFFFF7F7C1F7F7FFFF44
:1024E000FFFFFFFFFFF7F7EFFFFFFF81FFFFFFFF9A
:1024F000FFFFFFFFFFE7E7FFFFFDFBF7EFDFBFFF9A
:10250000C3BDB9A59DBDC3FFF7E7D7F7F7F7C1FF77
:10251000C3BDFDF3CFBF81FFC3BDFDE3FDBDC3FF61
:10252000FBF3EBDB81FBFBFF81BF87FBFDBBC7FF41
:10253000E3DFBF83BDBDC3FF81BDFBF7EFEFEFFF5F
:10254000C3BDBDC3BDBDC3FFC3BDBDC1FDFBC7FF93
:10255000FFFFF7FFFFF7FFFFFFFFF7FFFFF7F7EFC3
:10256000F1E7CF9FCFE7F1FFFFFF81FF81FFFFFF83
:102570008FE7F3F9F3E78FFFC3BDFDF3EFFFEFFF45
:10258000FFFFFFFF00FFFFFFF7E3C18080E3C1FF14
:10259000EFEFEFEFEFEFEFEFFFFFFF00FFFFFFFFCA
:1025A000FFFF00FFFFFFFFFFFF00FFFFFFFFFFFF39
:1025B000FFFFFFFFFF00FFFFDFDFDFDFDFDFDFDF2A
:1025C000FBFBFBFBFBFBFBFBFFFFFFFF1FEFF7F73B
:1025D000F7F7F7FBFCFFFFFFF7F7F7EF1FFFFFFF32
:1025E0007F7F7F7F7F7F7F007FBFDFEFF7FBFDFE79
:1025F000FEFDFBF7EFDFBF7F007F7F7F7F7F7F7F69
:1026000000FEFEFEFEFEFEFEFFC381818181C3FF50
:10261000FFFFFFFFFFFF00FFC9808080C1E3F7FFDE
:10262000BFBFBFBFBFBFBFBFFFFFFFFFFCFBF7F7D1
:102630007EBDDBE7E7DBBD7EFFC3BDBDBDBDC3FF28
:10264000F7E3D588D5F7F7FFFDFDFDFDFDFDFDFDA9
:10265000F7E3C180C1E3F7FFF7F7F7F700F7F7F704
:102660005FAF5FAF5FAF5FAFF7F7F7F7F7F7F7F77A
:10267000FFFFFEC1ABEBEBFF0080C0E0F0F8FCFE1B
:10268000FFFFFFFFFFFFFFFF0F0F0F0F0F0F0F0FDA
:10269000FFFFFFFF0000000000FFFFFFFFFFFFFF45
:1026A000FFFFFFFFFFFFFF007F7F7F7F7F7F7F7F39
:1026B00055AA55AA55AA55AAFEFEFEFEFEFEFEFE2E
:1026C000FFFFFFFF55AA55AA000103070F1F3F7F19
:1026D000FCFCFCFCFCFCFCFCF7F7F7F7F0F7F7F769
:1026E000FFFFFFFFF0F0F0F0F7F7F7F7F0FFFFFF65
:1026F000FFFFFFFF07F7F7F7FFFFFFFFFFFF0000F8
:10270000FFFFFFFFF0F7F7F7F7F7F7F700FFFFFF1F
:10271000FFFFFFFF00F7F7F7F7F7F7F707F7F7F710
:102720003F3F3F3F3F3F3F3F1F1F1F1F1F1F1F1FB9
:10273000F8F8F8F8F8F8F8F80000FFFFFFFFFFFFDF
:10274000000000FFFFFFFFFFFFFFFFFFFF00000093
:10275000FEFEFEFEFEFEFE00FFFFFFFF0F0F0F0F4F
:10276000F0F0F0F0FFFFFFFFF7F7F7F707FFFFFFCD
:102770000F0F0F0FFFFFFFFF0F0F0F0FF0F0F0F025
:102780001C224A564C201E00000038043C443A00EB
:1027900040405C6242625C0000003C4240423C00BF
:1027A00002023A4642463A0000003C427E403C006B
:1027B0000C12107C1010100000003A46463A023C01
:1027C00040405C62424242000800180808081C00B1
:1027D00004000C0404044438404044485068440059
:1027E0001808080808081C000000764949494900F3
:1027F00000005C624242420000003C4242423C0017
:1028000000005C62625C404000003A46463A0202C8
:1028100000005C624040400000003E403C027C0002
:1028200010107C1010120C000000424242463A0088
:102830000000424242241800000041494949360044
:10284000000042241824420000004242463A023C62
:1028500000007E0418207E003C20202020203C0028
:102860000C10103C10706E003C04040404043C0086
:1028700000081C2A08080808000010207F2010000B
:102880000000000000000000080808080000080020
:10289000242424000000000024247E247E2424001C
:1028A000081E281C0A3C0800006264081026460026
:1028B000304848304A443A00040810000000000044
:1028C0000408101010080400201008080810200048
:1028D000082A1C3E1C2A08000008083E08080000C0
:1028E00000000000000808100000007E000000004A
:1028F000000000000018180000020408102040002A
:102900003C42465A62423C000818280808083E002B
:102910003C42020C30407E003C42021C02423C0021
:10292000040C14247E0404007E4078040244380021
:102930001C20407C42423C007E42040810101000E3
:102940003C42423C42423C003C42423E020438008F
:10295000000008000008000000000800000808103F
:102960000E18306030180E0000007E007E0000005F
:1029700070180C060C1870003C42020C100010007D
:1029800000000000FF0000001824427E4242420086
:102990007C22223C22227C001C22404040221C003F
:1029A00078242222222478007E40407840407E0015
:1029B0007E404078404040001C22404E42221C0095
:1029C0004242427E424242001C08080808081C009D
:1029D0000E04040404443800424448704844420051
:1029E0004040404040407E0042665A5A42424200C7
:1029F0004262524A4642420018244242422418008F
:102A00007C42427C40404000182442424A241A0042
:102A10007C42427C484442003C42403C02423C00F2
:102A20003E080808080808004242424242423C0070
:102A300042424224241818004242425A5A66420036
:102A400042422418244242002222221C0808080084
:102A50007E02041820407E0008080808FF080808C5
:102A6000A050A050A050A050080808080808080866
:102A7000CCCC3333CCCC3333CC663399CC6633995E
:102A80000000000000000000F0F0F0F0F0F0F0F0C6
:102A900000000000FFFFFFFFFF000000000000003B
:102AA00000000000000000FF808080808080808027
:102AB000AA55AA55AA55AA55010101010101010112
:102AC00000000000AA55AA55993366CC993366CC0C
:102AD0000303030303030303080808080F08080897
:102AE000000000000F0F0F0F080808080F0000007B
:102AF00000000000F8080808000000000000FFFFC8
:102B0000000000000F08080808080808FF0000007F
:102B100000000000FF08080808080808F80808086E
:102B2000C0C0C0C0C0C0C0C0E0E0E0E0E0E0E0E0A5
:102B30000707070707070707FFFF0000000000005F
:102B4000FFFFFF00000000000000000000FFFFFF8B
:102B5000010244485060400000000000F0F0F0F036
:102B60000F0F0F0F0000000008080808F800000011
:102B7000F0F0F0F000000000F0F0F0F00F0F0F0F99
:102B8000E3DDB5A9B3DFE1FFFFFFC7FBC3BBC5FFB3
:102B9000BFBFA39DBD9DA3FFFFFFC3BDBFBDC3FFBF
:102BA000FDFDC5B9BDB9C5FFFFFFC3BD81BFC3FFF3
:102BB000F3EDEF83EFEFEFFFFFFFC5B9B9C5FDC33D
:102BC000BFBFA39DBDBDBDFFF7FFE7F7F7F7E3FF6D
:102BD000FBFFF3FBFBFBBBC7BFBFBBB7AF97BBFFA5
:102BE000E7F7F7F7F7F7E3FFFFFF89B6B6B6B6FFEB
:102BF000FFFFA39DBDBDBDFFFFFFC3BDBDBDC3FFA7
:102C0000FFFFA39D9DA3BFBFFFFFC5B9B9C5FDFDD4
:102C1000FFFFA39DBFBFBFFFFFFFC1BFC3FD83FF7A
:102C2000EFEF83EFEFEDF3FFFFFFBDBDBDB9C5FFD4
:102C3000FFFFBDBDBDDBE7FFFFFFBEB6B6B6C9FFF8
:102C4000FFFFBDDBE7DBBDFFFFFFBDBDB9C5FDC3BA
:102C5000FFFF81FBE7DF81FFC3DFDFDFDFDFC3FFD4
:102C6000F3EFEFC3EF8F91FFC3FBFBFBFBFBC3FF56
:102C7000FFF7E3D5F7F7F7F7FFFFEFDF80DFEFFFB1
:102C8000FFFFFFFFFFFFFFFFF7F7F7F7FFFFF7FF7C
:102C9000DBDBDBFFFFFFFFFFDBDB81DB81DBDBFF60
:102CA000F7E1D7E3F5C3F7FFFF9D9BF7EFD9B9FF36
:102CB000CFB7B7CFB5BBC5FFFBF7EFFFFFFFFFFFF8
:102CC000FBF7EFEFEFF7FBFFDFEFF7F7F7EFDFFFD4
:102CD000F7D5E3C1E3D5F7FFFFF7F7C1F7F7FFFF3C
:102CE000FFFFFFFFFFF7F7EFFFFFFF81FFFFFFFF92
:102CF000FFFFFFFFFFE7E7FFFFFDFBF7EFDFBFFF92
:102D0000C3BDB9A59DBDC3FFF7E7D7F7F7F7C1FF6F
:102D1000C3BDFDF3CFBF81FFC3BDFDE3FDBDC3FF59
:102D2000FBF3EBDB81FBFBFF81BF87FBFDBBC7FF39
:102D3000E3DFBF83BDBDC3FF81BDFBF7EFEFEFFF57
:102D4000C3BDBDC3BDBDC3FFC3BDBDC1FDFBC7FF8B
:102D5000FFFFF7FFFFF7FFFFFFFFF7FFFFF7F7EFBB
:102D6000F1E7CF9FCFE7F1FFFFFF81FF81FFFFFF7B
:102D70008FE7F3F9F3E78FFFC3BDFDF3EFFFEFFF3D
:102D8000FFFFFFFF00FFFFFFE7DBBD81BDBDBDFF14
:102D900083DDDDC3DDDD83FFE3DDBFBFBFDDE3FF3B
:102DA00087DBDDDDDDDB87FF81BFBF87BFBF81FF45
:102DB00081BFBF87BFBFBFFFE3DDBFB1BDDDE3FFA5
:102DC000BDBDBD81BDBDBDFFE3F7F7F7F7F7E3FF7D
:102DD000F1FBFBFBFBBBC7FFBDBBB78FB7BBBDFFA9
:102DE000BFBFBFBFBFBF81FFBD99A5A5BDBDBDFF13
:102DF000BD9DADB5B9BDBDFFE7DBBDBDBDDBE7FF2B
:102E000083BDBD83BFBFBFFFE7DBBDBDB5DBE5FF56
:102E100083BDBD83B7BBBDFFC3BDBFC3FDBDC3FF86
:102E2000C1F7F7F7F7F7F7FFBDBDBDBDBDBDC3FFE8
:102E3000BDBDBDDBDBE7E7FFBDBDBDA5A599BDFF02
:102E4000BDBDDBE7DBBDBDFFDDDDDDE3F7F7F7FF94
:102E500081FDFBE7DFBF81FFF7F7F7F700F7F7F733
:102E60005FAF5FAF5FAF5FAFF7F7F7F7F7F7F7F772
:102E70003333CCCC3333CCCC3399CC663399CC665A
:102E8000FFFFFFFFFFFFFFFF0F0F0F0F0F0F0F0FD2
:102E9000FFFFFFFF0000000000FFFFFFFFFFFFFF3D
:102EA000FFFFFFFFFFFFFF007F7F7F7F7F7F7F7F31
:102EB00055AA55AA55AA55AAFEFEFEFEFEFEFEFE26
:102EC000FFFFFFFF55AA55AA66CC993366CC99330C
:102ED000FCFCFCFCFCFCFCFCF7F7F7F7F0F7F7F761
:102EE000FFFFFFFFF0F0F0F0F7F7F7F7F0FFFFFF5D
:102EF000FFFFFFFF07F7F7F7FFFFFFFFFFFF0000F0
:102F0000FFFFFFFFF0F7F7F7F7F7F7F700FFFFFF17
:102F1000FFFFFFFF00F7F7F7F7F7F7F707F7F7F708
:102F20003F3F3F3F3F3F3F3F1F1F1F1F1F1F1F1FB1
:102F3000F8F8F8F8F8F8F8F80000FFFFFFFFFFFFD7
:102F4000000000FFFFFFFFFFFFFFFFFFFF0000008B
:102F5000FEFDBBB7AF9FBFFFFFFFFFFF0F0F0F0FC0
:102F6000F0F0F0F0FFFFFFFFF7F7F7F707FFFFFFC5
:102F70000F0F0F0FFFFFFFFF0F0F0F0FF0F0F0F01D
:102F800078E367E443424D424153494330C841C767
:102F90001DCDF7C8A4CBBECB80D005CCA4C99FC89B
:102FA00070C827C91CC882C8D1C83AC92EC84AC926
:102FB0002CD864E152E161E1B2D323D87FCA9FCA21
:102FC00056C89BC65DC685CA26E1BAE1C3E17ACB85
:102FD00041C639DCCCDC58DC00007DD39ED371DFE8
:102FE00094E0EAD9EDDF61E268E2B1E20BE30DD8EB
:102FF0007CD765D4ADD78BD7ECD600D72CD737D7B5
:103000007969D87952D87B2ADA7B11DB7F7ADF5055
:10301000E8CF46E5CF7DB3DF5AD3CE6415D0454E19
:10302000C4464FD24E4558D4444154C1494E5055E0
:1030300054A3494E5055D44449CD524541C44C4502
:10304000D4474F54CF5255CE49C6524553544F5290
:10305000C5474F5355C25245545552CE5245CD5394
:10306000544FD04FCE574149D44C4F41C453415691
:10307000C55645524946D94445C6504F4BC5505296
:10308000494E54A35052494ED4434F4ED44C495309
:10309000D4434CD2434DC45359D34F5045CE434CE7
:1030A0004F53C54745D44E45D7544142A854CF4607
:1030B000CE535043A8544845CE4E4FD4535445D0D8
:1030C000ABADAAAFDE414EC44FD2BEBDBC5347CE5E
:1030D000494ED44142D35553D24652C5504FD35393
:1030E00051D2524EC44C4FC74558D0434FD3534989
:1030F000CE5441CE4154CE504545CB4C45CE535491
:1031000052A45641CC4153C3434852A44C45465463
:10311000A45249474854A44D4944A447CF00544FB2
:103120004F204D414E592046494C45D346494C45C8
:10313000204F5045CE46494C45204E4F54204F50CD
:1031400045CE46494C45204E4F5420464F554EC41F
:10315000444556494345204E4F542050524553450F
:103160004ED44E4F5420494E5055542046494CC5DC
:103170004E4F54204F55545055542046494CC54D40
:10318000495353494E472046494C45204E414DC571
:10319000494C4C4547414C20444556494345204EF7
:1031A000554D4245D24E45585420574954484F55E5
:1031B0005420464FD253594E5441D852455455523B
:1031C0004E20574954484F555420474F5355C24FEE
:1031D0005554204F4620444154C1494C4C45474129
:1031E0004C205155414E544954D94F564552464CA6
:1031F0004FD74F5554204F46204D454D4F52D9552E
:103200004E44454627442053544154454D454ED4E1
:10321000424144205355425343524950D4524544AD
:10322000494D27442041525241D9444956495349B6
:103230004F4E204259205A4552CF494C4C454741A8
:103240004C204449524543D454595045204D49538C
:103250004D415443C8535452494E4720544F4F2078
:103260004C4F4EC746494C4520444154C1464F52ED
:103270004D554C4120544F4F20434F4D504C45D855
:1032800043414E275420434F4E54494E55C5554E49
:1032900044454627442046554E4354494FCE564553
:1032A000524946D94C4F41C49EC1ACC1B5C1C2C1FF
:1032B000D0C1E2C1F0C1FFC110C225C235C23BC2BC
:1032C0004FC25AC26AC272C27FC290C29DC2AAC213
:1032D000BAC2C8C2D5C2E4C2EDC200C30EC31EC387
:1032E00024C383C30D4F4B0D000D204552524F5246
:1032F0000020494E20000D0A52454144592E0D0A26
:10330000000D0A425245414B00A0BAE8E8E8E8BD8A
:103310000101C981D021A54AD00ABD02018549BD5C
:103320000301854ADD0301D007A549DD0201F0074D
:103330008A186912AAD0D8602008C485318432382E
:10334000A55AE55F8522A8A55BE560AAE898F02369
:10335000A55A38E522855AB003C65B38A558E52240
:103360008558B008C6599004B15A915888D0F9B11F
:103370005A9158C65BC659CAD0F2600A693EB03548
:103380008522BAE422902E60C4349028D004C5333C
:10339000902248A2099848B557CA10FA2026D5A20B
:1033A000F7689561E830FA68A868C4349006D005DB
:1033B000C533B00160A2106C00038A0AAABD26C3FF
:1033C0008522BD27C3852320CCFFA900851320D7E4
:1033D000CA2045CBA000B12248297F2047CBC8682E
:1033E00010F4207AC6A969A0C3201ECBA43AC8F065
:1033F0000320C2DDA976A0C3201ECBA9802090FFA8
:103400006C02032060C5867A847B207300AAF0F0EA
:10341000A2FF863A90062079C54CE1C7206BC920EF
:1034200079C5840B2013C69044A001B15F8523A504
:103430002D8522A5608525A55F88F15F18652D85FE
:103440002D8524A52E69FF852EE560AA38A55FE5A8
:103450002DA8B003E8C6251865229003C62318B12D
:10346000229124C8D0F9E623E625CAD0F22059C615
:103470002033C5AD0002F08818A52D855A650B854F
:1034800058A42E845B9001C8845920B8C3A514A405
:10349000158DFE018CFF01A531A432852D842EA44B
:1034A0000B88B9FC01915F8810F82059C62033C5FC
:1034B0004C80C4A52BA42C8522842318A001B12202
:1034C000F01DA004C8B122D0FBC8986522AAA000B4
:1034D0009122A5236900C891228622852390DD6070
:1034E000A200200FE1C90DF00D9D0002E8E0599007
:1034F000F1A2174C37C44CCACA6C0403A67AA004C4
:10350000840FBD00021007C9FFF03EE8D0F4C920C7
:10351000F0378508C922F056240F702DC93FD0041A
:10352000A999D025C9309004C93C901D8471A00090
:10353000840B88867ACAC8E8BD000238F99EC0F0BC
:10354000F5C980D030050BA471E8C899FB01B9FB1F
:1035500001F03638E93AF004C949D002850F38E95C
:1035600055D09F8508BD0002F0DFC508F0DBC89983
:10357000FB01E8D0F0A67AE60BC8B99DC010FAB9F5
:103580009EC0D0B4BD000210BE99FD01C67BA9FF4C
:10359000857A60A52BA62CA001855F8660B15FF0BF
:1035A0001FC8C8A515D15F9018F00388D009A514CD
:1035B00088D15F900CF00A88B15FAA88B15FB0D75C
:1035C0001860D0FDA900A8912BC8912BA52B1869D4
:1035D00002852DA52C6900852E208EC6A900D02D30
:1035E00020E7FFA537A43885338434A52DA42E8584
:1035F0002F843085318432201DC8A219861668A810
:1036000068A2FA9A489848A900853E85106018A5D6
:103610002B69FF857AA52C69FF857B609006F004F5
:10362000C9ABD0E9206BC92013C6207900F00CC9C2
:10363000ABD08E207300206BC9D0866868A51405B6
:1036400015D006A9FF85148515A001840FB15FF080
:1036500043202CC820D7CAC8B15FAAC8B15FC5151E
:10366000D004E414F002B02C844920CDDDA920A4BC
:1036700049297F2047CBC922D006A50F49FF850FD6
:10368000C8F011B15FD010A8B15FAAC8B15F865F62
:103690008560D0B54C74C46C060310D7C9FFF0D355
:1036A000240F30CF38E97FAA8449A0FFCAF008C8A8
:1036B000B99EC010FA30F5C8B99EC030B22047CBD1
:1036C000D0F5A980851020A5C9208AC3D0058A69B4
:1036D0000FAA9A6868A90920FBC32006C918986533
:1036E0007A48A57B690048A53A48A53948A9A4208D
:1036F000FFCE208DCD208ACDA566097F256285620B
:10370000A98BA0C7852284234C43CEA9BCA0D92075
:10371000A2DB207900C9A9D006207300208ACD2021
:103720002BDC2038CEA54A48A54948A98148202C41
:10373000C8A57AA47BC002EAF004853D843EA000BF
:10374000B17AD043A002B17A18D0034C4BC8C8B1AB
:103750007A8539C8B17A853A98657A857A9002E691
:103760007B6C080320730020EDC74CAEC7F03CE92A
:10377000809011C923B0170AA8B90DC048B90CC070
:10378000484C73004CA5C9C93AF0D64C08CFC94B78
:10379000D0F9207300A9A420FFCE4CA0C838A52BD7
:1037A000E901A42CB00188854184426020E1FFB08A
:1037B0000118D03CA57AA47BA63AE8F00C853D849C
:1037C0003EA539A43A853B843C6868A981A0C39092
:1037D000034C69C44C74C4D017A21AA43ED0034C45
:1037E00037C4A53D857A847BA53BA43C8539843AC2
:1037F0006008A9002090FF28D0034C59C62060C65D
:103800004C97C8A90320FBC3A57B48A57A48A53AD5
:1038100048A53948A98D4820790020A0C84CAEC7DA
:10382000206BC92009C938A539E514A53AE515B0BA
:103830000B9838657AA67B9007E8B004A52BA62CD8
:103840002017C6901EA55FE901857AA560E900856D
:103850007B60D0FDA9FF854A208AC39AC98DF00BF1
:10386000A20C2CA2114C37C44C08CF68688539686B
:10387000853A68857A68857B2006C99818657A85B7
:103880007A9002E67B60A23A2CA2008607A0008410
:1038900008A508A60785078608B17AF0E8C508F0EC
:1038A000E4C8C922D0F3F0E9209ECD207900C9896F
:1038B000F005A9A720FFCEA561D0052009C9F0BB5E
:1038C000207900B0034CA0C84CEDC7209ED748C952
:1038D0008DF004C989D091C665D004684CEFC7202B
:1038E0007300206BC9C92CF0EE6860A200861486B4
:1038F00015B0F7E92F8507A5158522C919B0D4A5FC
:10390000140A26220A262265148514A52265158527
:103910001506142615A514650785149002E61520D2
:1039200073004C71C9208BD08549844AA9B220FF0D
:10393000CEA50E48A50D48209ECD682A2090CDD05A
:1039400018681012201BDC20BFD1A000A56491498B
:10395000C8A5659149604CD0DB68A44AC0DFD04C53
:1039600020A6D6C906D03DA000846184668471205B
:103970001DCA20E2DAE671A471201DCA200CDCAA5F
:10398000F005E88A20EDDAA471C8C006D0DF20E295
:10399000DA209BDCA664A463A5654CDBFFB1222082
:1039A000800090034C48D2E92F4C7EDDA002B16428
:1039B000C5349017D00788B164C533900EA465C490
:1039C0002E9008D00DA564C52DB007A564A4654C44
:1039D00068CAA000B1642075D4A550A451856F8435
:1039E00070207AD6A961A0008550845120DBD6A032
:1039F00000B1509149C8B1509149C8B15091496046
:103A00002086CA4CB5CB209ED7F005A92C20FFCE2E
:103A10000886132015E1284CA0CA2021CB2079006C
:103A2000F035F043C9A3F050C9A618F04BC92CF0EB
:103A300037C93BF05E209ECD240D30DE20DDDD2039
:103A400087D42021CB203BCBD0D3A9009D0002A25C
:103A5000FFA001A513D010A90D2047CB24131005FA
:103A6000A90A2047CB49FF603820F0FF9838E90BBE
:103A7000B0FC49FF6901D016083820F0FF84092006
:103A80009BD7C929D0592890068AE5099005AAE84C
:103A9000CAD0062073004CA2CA203BCBD0F22087AC
:103AA000D420A6D6AAA000E8CAF0BCB1222047CBF9
:103AB000C8C90DD0F320E5CA4C28CBA513F003A943
:103AC000202CA91D2CA93F2009E129FF60A511F098
:103AD000113004A0FFD004A53FA4408539843A4C9E
:103AE00008CFA513F005A2184C37C4A90CA0CD200F
:103AF0001ECBA53DA43E857A847B6020A6D3C92336
:103B0000D010207300209ED7A92C20FFCE86132032
:103B10001BE1A201A002A9008D0102A940200FCC47
:103B2000A613D01360209ED7A92C20FFCE86132089
:103B30001BE120CECBA51320CCFFA200861360C9C9
:103B400022D00B20BDCEA93B20FFCE2021CB20A62A
:103B5000D3A92C8DFF0120F9CBA513F00D20B7FFC1
:103B60002902F00620B5CB4CF8C8AD0002D01EA546
:103B700013D0E32006C94CFBC8A513D0062045CBC3
:103B8000203BCB4C60C5A641A442A9982CA9008536
:103B90001186438444208BD08549844AA57AA47B2E
:103BA000854B844CA643A444867A847B207900D03C
:103BB000202411500C2021E18D0002A2FFA001D091
:103BC0000C3075A513D0032045CB20F9CB867A8421
:103BD0007B207300240D103124115009E8867AA946
:103BE000008507F00C8507C922F007A93A8507A9C7
:103BF0002C188508A57AA47B69009001C8208DD473
:103C000020E2D720DAC94C91CC20F3DCA50E20C2EB
:103C1000C9207900F007C92CF0034C4DCBA57AA43C
:103C20007B85438444A54BA44C857A847B20790012
:103C3000F02D20FDCE4C15CC2006C9C8AAD012A26A
:103C40000DC8B17AF06CC8B17A853FC8B17AC88521
:103C50004020FBC8207900AAE083D0DC4C51CCA5E1
:103C600043A444A61110034C27C8A000B143F00B95
:103C7000A513D007A9FCA0CC4C1ECB603F455854DF
:103C800052412049474E4F5245440D003F52454452
:103C90004F2046524F4D2053544152540D00D004F2
:103CA000A000F003208BD08549844A208AC3F00508
:103CB000A20A4C37C49A8A186904486906852468A0
:103CC000A00120A2DBBABD09018566A549A44A204E
:103CD00067D820D0DBA001205DDCBA38FD0901F0F7
:103CE00017BD0F018539BD1001853ABD1201857AD6
:103CF000BD1101857B4CAEC78A6911AA9A20790053
:103D0000C92CD0F12073002024CD209ECD1824385A
:103D1000240D3003B00360B0FDA2164C37C4A67A60
:103D2000D002C67BC67AA20024488A48A90120FB9B
:103D3000C32083CEA900854D20790038E9B19017C2
:103D4000C903B013C9012A4901454DC54D9061858C
:103D50004D2073004CBBCDA64DD02CB07B69079095
:103D600077650DD0034C3DD669FF85220A6522A8F0
:103D700068D980C0B067208DCD482020CE68A44B84
:103D80001017AAF056D05F460D8A2AA67AD002C62E
:103D90007BC67AA01B854DD0D7D980C0B04890D9BA
:103DA000B982C048B981C0482033CEA54D4CA9CDB9
:103DB0004C08CFA566BE80C0A8688522E62268852B
:103DC000239848201BDCA56548A56448A56348A541
:103DD0006248A561486C2200A0FF68F023C964F026
:103DE00003208DCD844B684A851268856968856A91
:103DF00068856B68856C68856D68856E4566856FBE
:103E0000A561606C0A03A900850D207300B0034C06
:103E1000F3DC2013D190034C28CFC9FFD00FA9A801
:103E2000A0CE20A2DB4C730082490FDAA1C92EF08C
:103E3000DEC9ABF058C9AAF0D1C922D00FA57AA427
:103E40007B69009001C82087D44CE2D7C9A8D01361
:103E5000A018D03B20BFD1A56549FFA8A56449FFA4
:103E60004C91D3C9A5D0034CF4D3C9B490034CA74B
:103E7000CF20FACE209ECDA9292CA9282CA92CA090
:103E800000D17AD0034C7300A20B4C37C4A0156844
:103E9000684CFACD38A564E900A565E9C09008A989
:103EA00087E564A9E3E56560208BD085648465A619
:103EB00045A446A50DF026A90085702014CF901CBE
:103EC000E054D018C0C9D0142084CF845E88847197
:103ED000A006845DA0242068DE4C6FD460240E1000
:103EE0000DA000B164AAC8B164A88A4C91D3201473
:103EF000CF902DE054D01BC049D0252084CF98A26C
:103F0000A04C4FDC20DEFF866484638565A00084BE
:103F10006260E053D00AC054D00620B7FF4C3CDCAE
:103F2000A564A4654CA2DB0A48AA207300E08F9028
:103F30002020FACE209ECD20FDCE208FCD68AAA5D0
:103F40006548A564488A48209ED768A88A484CD608
:103F5000CF20F1CE68A8B9EABF8555B9EBBF855629
:103F60002054004C8DCDA0FF2CA000840B20BFD18D
:103F7000A564450B8507A565450B850820FCDB205E
:103F8000BFD1A565450B2508450BA8A564450B25A4
:103F900007450B4C91D32090CDB013A56E097F251A
:103FA0006A856AA969A000205BDCAA4C61D0A900DF
:103FB000850DC64D20A6D6856186628463A56CA456
:103FC0006D20AAD6866C846DAA38E561F008A90137
:103FD0009004A661A9FF8566A0FFE8C8CAD007A61D
:103FE00066300F18900CB16CD162F0EFA2FFB002F6
:103FF000A201E88A2A2512F002A9FF4C3CDC20FD30
:10400000CEAA2090D0207900D0F460A200207900C0
:10401000860C85452079002013D1B0034C08CFA22F
:1040200000860D860E20730090052013D1900BAAF8
:1040300020730090FB2013D1B0F6C924D006A9FF4D
:10404000850DD010C925D013A510D0D0A980850E1C
:10405000054585458A0980AA2073008646380510E3
:10406000E928D0034CD1D1A0008410A52DA62E861E
:1040700060855FE430D004C52FF022A545D15FD024
:1040800008A546C8D15FF07D8818A55F690790E153
:10409000E8D0DCC9419005E95B38E9A5606848C90A
:1040A0002AD005A913A0DF60A545A446C954D00BAA
:1040B000C0C9F0EFC049D0034C08CFC953D004C0E9
:1040C00054F0F5A52FA430855F8460A531A4328516
:1040D0005A845B1869079001C88558845920B8C371
:1040E000A558A459C8852F8430A000A545915FC864
:1040F000A546915FA900C8915FC8915FC8915FC84C
:10410000915FC8915FA55F186902A4609001C8859E
:1041100047844860A50B0A6905655FA4609001C8E3
:104120008558845960908000000020BFD1A564A408
:104130006560207300209ECD208DCDA566300DA535
:1041400061C9909009A9A5A0D1205BDCD07A4C9BD5
:10415000DCA50C050E48A50D48A0009848A54648CA
:10416000A5454820B2D168854568854668A8BABD8E
:10417000020148BD010148A5649D0201A5659D019C
:1041800001C8207900C92CF0D2840B20F7CE6885B5
:104190000D68850E297F850CA62FA530865F85606A
:1041A000C532D004E431F039A000B15FC8C545D0B4
:1041B00006A546D15FF016C8B15F18655FAAC8B101
:1041C0005F656090D7A2122CA20E4C37C4A213A533
:1041D0000CD0F72094D1A50BA004D15FD0E74CEA16
:1041E000D22094D12008C4A0008472A205A54591D4
:1041F0005F1001CAC8A546915F1002CACA8671A5A0
:104200000BC8C8C8915FA20BA900240C50086818FD
:104210006901AA686900C8915FC88A915F204CD380
:1042200086718572A422C60BD0DC6559B05D8559B4
:10423000A88A65589003C8F0522008C4853184329A
:10424000A900E672A471F005889158D0FBC659C642
:1042500072D0F5E65938A531E55FA002915FA5322D
:10426000C8E560915FA50CD062C8B15F850BA9005D
:1042700085718572C868AA8564688565D15F900E6E
:10428000D006C88AD15F90074C45D24C35C4C8A52A
:1042900072057118F00A204CD38A6564AA98A4228A
:1042A00065658671C60BD0CA8572A205A545100149
:1042B000CAA5461002CACA8628A9002055D38A6515
:1042C0005885479865598548A8A547608422B15FFD
:1042D000852888B15F8529A910855DA200A0008A84
:1042E0000AAA982AA8B0A406712672900B188A65AB
:1042F00028AA986529A8B093C65DD0E360A50DF003
:104300000320A6D62026D538A533E531A8A534E567
:1043100032A200860D85628463A2904C44DC382072
:10432000F0FFA900F0EBA63AE8D0A0A2152CA21B42
:104330004C37C420E1D320A6D320FACEA980851023
:10434000208BD0208DCD20F7CEA9B220FFCE48A55E
:104350004848A54748A57B48A57A4820F8C84C4F4F
:10436000D4A9A520FFCE098085102092D0854E8447
:104370004F4C8DCD20E1D3A54F48A54E4820F1CE1E
:10438000208DCD68854E68854FA002B14E8547AA25
:10439000C8B14EF0998548C8B147488810FAA4487A
:1043A00020D4DBA57B48A57A48B14E857AC8B14EAA
:1043B000857BA54848A54748208ACD68854E6885F5
:1043C0004F207900F0034C08CF68857A68857BA080
:1043D0000068914E68C8914E68C8914E68C8914E69
:1043E00068C8914E60208DCDA00020DFDD6868A9EF
:1043F000FFA000F012A664A4658650845120F4D476
:1044000086628463856160A22286078608856F8440
:104410007085628463A0FFC8B16FF00CC507F0041B
:10442000C508D0F3C922F00118846198656F8571C1
:10443000A6709001E88672A570F004C902D00B98AE
:104440002075D4A66FA4702088D6A616E022D005C9
:10445000A2194C37C4A5619500A5629501A5639585
:1044600002A00086648465847088840D8617E8E85D
:10447000E8861660460F4849FF386533A434B0011A
:1044800088C4329011D004C531900B8533843485B3
:10449000358436AA6860A210A50F30B62026D5A9AB
:1044A00080850F68D0D0A637A53886338534A00024
:1044B000844F844EA531A632855F8660A919A2007B
:1044C00085228623C516F00520C7D5F0F7A90785F4
:1044D00053A52DA62E85228623E430D004C52FF0C7
:1044E0000520BDD5F0F385588659A9038553A558F5
:1044F000A659E432D007C531D0034C06D6852286B2
:1045000023A000B122AAC8B12208C8B122655885EB
:1045100058C8B122655985592810D38A30D0C8B1FE
:1045200022A0000A6905652285229002E623A623BF
:10453000E459D004C558F0BA20C7D5F0F3B1223001
:1045400035C8B1221030C8B122F02BC8B122AAC898
:10455000B122C5349006D01EE433B01AC56090165F
:10456000D004E45F9010865F8560A522A623854E67
:10457000864FA5538555A55318652285229002E6DE
:1045800023A623A00060A54F054EF0F5A5552904EC
:104590004AA88555B14E655F855AA5606900855B5F
:1045A000A533A6348558865920BFC3A455C8A5583D
:1045B000914EAAE659A559C8914E4C2AD5A56548F1
:1045C000A564482083CE208FCD68856F688570A054
:1045D00000B16F1871649005A2174C37C42075D4D0
:1045E000207AD6A550A45120AAD6208CD6A56FA497
:1045F0007020AAD620CAD44CB8CDA000B16F48C84C
:10460000B16FAAC8B16FA86886228423A8F00A48AF
:1046100088B122913598D0F86818653585359002B3
:10462000E63660208FCDA564A4658522842320DB37
:10463000D608A000B12248C8B122AAC8B122A868F1
:1046400028D013C434D00FE433D00B481865338519
:10465000339002E634688622842360C418D00CC5E7
:1046600017D0088516E9038517A0006020A1D78A16
:1046700048A901207DD468A000916268684CCAD422
:104680002061D7D150989004B150AA98488A482008
:104690007DD4A550A45120AAD668A86818652285A3
:1046A000229002E62398208CD64CCAD42061D718D9
:1046B000F15049FF4C06D7A9FF8565207900C9292B
:1046C000F00620FDCE209ED72061D7F04BCA8A4845
:1046D00018A200F150B0B649FFC56590B1A565B00C
:1046E000AD20F7CE68A8688555686868AA688550C7
:1046F000688551A555489848A0008A602082D74C0B
:10470000A2D320A3D6A200860DA8602082D7F008ED
:10471000A000B122A84CA2D34C48D2207300208A1A
:10472000CD20B8D1A664D0F0A6654C79002082D700
:10473000D0034CF7D8A67AA47B86718472A6228611
:104740007A1865228524A623867B9001E88625A019
:1047500000B1244898912420790020F3DC68A0005F
:104760009124A671A472867A847B60208ACD20F77A
:10477000D720FDCE4C9ED7A566309DA561C991B0CE
:1047800097209BDCA564A4658414851560A5154855
:10479000A5144820F7D7A000B114A868851468852F
:1047A000154CA2D320EBD78AA00091146020EBD740
:1047B0008649A200207900F00320F1D7864AA000A4
:1047C000B114454A2549F0F860A911A0DF4C67D81B
:1047D000208CDAA56649FF8566456E856FA5614C1C
:1047E0006AD82099D9903C208CDAD0034CFCDBA607
:1047F000708656A269A569A8F0CE38E561F02490CC
:10480000128461A46E846649FF6900A0008456A2E8
:1048100061D004A0008470C9F930C7A8A570560102
:1048200020B0D9246F1057A061E069F002A0693868
:1048300049FF65568570B90400F5048565B9030024
:10484000F5038564B90200F5028563B90100F5013D
:104850008562B0032047D9A0009818A662D04AA666
:10486000638662A6648663A6658664A67086658490
:10487000706908C920D0E4A9008561856660655625
:104880008570A565656D8565A564656C8564A563A2
:10489000656B8563A562656A85624C36D9690106D8
:1048A00070266526642663266210F238E561B0C77B
:1048B00049FF69018561900EE661F04266626663B8
:1048C00066646665667060A56649FF8566A562498F
:1048D000FF8562A56349FF8563A56449FF8564A5DB
:1048E0006549FF8565A57049FF8570E670D00EE6C5
:1048F00065D00AE664D006E663D002E66260A20FE5
:104900004C37C4A225B4048470B4039404B4029454
:1049100003B4019402A4689401690830E8F0E6E960
:1049200008A8A570B01416019002F6017601760170
:104930007602760376046AC8D0EC18608100000025
:1049400000037F5E56CB7980139B0B64807638938F
:10495000168238AA3B20803504F334813504F334C1
:10496000808000000080317217F8202BDCF00210EC
:10497000034C48D2A561E97F48A9808561A9D6A0EA
:10498000D92067D8A9DBA0D9200FDBA9BCA0D920EA
:1049900050D8A9C1A0D92040E0A9E0A0D92067D86B
:1049A00068207EDDA9E5A0D9208CDAD0034C8BDA13
:1049B00020B7DAA9008526852785288529A57020B6
:1049C00059DAA5652059DAA5642059DAA56320597A
:1049D000DAA562205EDA4C8FDBD0034C83D94A091A
:1049E00080A8901918A529656D8529A528656C856D
:1049F00028A527656B8527A526656A852666266610
:104A000027662866296670984AD0D6608522842356
:104A1000A004B122856D88B122856C88B122856B96
:104A200088B122856E4566856FA56E0980856A8886
:104A3000B1228569A56160A569F01F1865619004C0
:104A4000301D182C101469808561D0034CFBD8A54B
:104A50006F856660A56649FF300568684CF7D84CDD
:104A60007ED9200CDCAAF010186902B0F2A20086F0
:104A70006F2077D8E661F0E7608420000000200C0A
:104A8000DCA9F9A0DAA200866F20A2DB4C12DB20A1
:104A90008CDAF076201BDCA90038E561856120B74F
:104AA000DAE661F0BAA2FCA901A46AC462D010A43B
:104AB0006BC463D00AA46CC464D004A46DC465083C
:104AC0002A9009E89529F0321034A90128B00E0681
:104AD0006D266C266B266AB0E630CE10E2A8A56D76
:104AE000E565856DA56CE564856CA56BE563856BF7
:104AF000A56AE562856A984C4FDBA940D0CE0A0AC8
:104B00000A0A0A0A8570284C8FDBA2144C37C4A508
:104B1000268562A5278563A5288564A52985654C1A
:104B2000D7D885228423A004B122856588B1228547
:104B30006488B122856388B1228566098085628890
:104B4000B1228561847060A25C2CA257A000F004A1
:104B5000A649A44A201BDC86228423A004A56591D3
:104B60002288A564912288A563912288A566097F81
:104B70002562912288A5619122847060A56E856668
:104B8000A205B5689560CAD0F9867060201BDCA2CA
:104B900006B5609568CAD0F9867060A561F0FB061D
:104BA0007090F7206FD9D0F24C38D9A561F009A5E3
:104BB000662AA9FFB002A90160202BDC8562A9004A
:104BC0008563A288A56249FF2AA900856585648658
:104BD00061857085664CD2D846666085248425A0A0
:104BE00000B124C8AAF0C4B124456630C2E461D043
:104BF00021B1240980C562D019C8B124C563D0127F
:104C0000C8B124C564D00BC8A97FC570B124E565BF
:104C1000F028A566900249FF4C31DCA561F04A38C6
:104C2000E9A024661009AAA9FF8568204DD98AA2A7
:104C300061C9F910062099D9846860A8A566298001
:104C400046620562856220B0D9846860A561C9A00A
:104C5000B020209BDC8470A566846649802AA9A0C8
:104C60008561A56585074CD2D88562856385648595
:104C700065A860A000A20A945DCA10FB900FC92D20
:104C8000D0048667F004C92BD005207300905BC95F
:104C90002EF02EC945D0302073009017C9ABF00E0E
:104CA000C92DF00AC9AAF008C92BF004D007666024
:104CB000207300905C2460100EA90038E55E4C491A
:104CC000DD665F245F50C3A55E38E55D855EF0124A
:104CD000100920FEDAE65ED0F9F00720E2DAC65EBF
:104CE000D0F9A5673001604CB4DF48245F1002E6BC
:104CF0005D20E2DA6838E930207EDD4C0ADD4820AC
:104D00000CDC68203CDCA56E4566856FA6614C6AAC
:104D1000D8A55EC90A9009A964246030114C7ED9D7
:104D20000A0A18655E0A18A000717A38E930855EB3
:104D30004C30DD9B3EBC1FFD9E6E6B27FD9E6E6B57
:104D40002800A971A0C320DADDA53AA639856286BC
:104D500063A290382049DC20DFDD4C1ECBA001A9E6
:104D60002024661002A92D99FF0085668471C8A9C8
:104D700030A661D0034C04DFA900E080F002B00946
:104D8000A9BDA0DD2028DAA9F7855DA9B8A0DD209E
:104D90005BDCF01E1012A9B3A0DD205BDCF002107A
:104DA0000E20E2DAC65DD0EE20FEDAE65DD0DC2031
:104DB00049D8209BDCA201A55D18690A3009C90BFE
:104DC000B00669FFAAA90238E902855E865D8AF00D
:104DD000021013A471A92EC899FF008AF006A93009
:104DE000C899FF008471A000A280A565187919DF19
:104DF0008565A5647918DF8564A5637917DF856308
:104E0000A5627916DF8562E8B00410DE300230DA80
:104E10008A900449FF690A692FC8C8C8C88447A492
:104E200071C8AA297F99FF00C65DD006A92EC8992E
:104E3000FF008471A4478A49FF2980AAC024F00496
:104E4000C03CD0A6A471B9FF0088C930F0F8C92EC3
:104E5000F001C8A92BA65EF02E1008A90038E55E67
:104E6000AAA92D990101A9459900018AA22F38E824
:104E7000E90AB0FB693A9903018A990201A90099EC
:104E80000401F00899FF00A900990001A900A00100
:104E9000608000000000FA0A1F0000989680FFF072
:104EA000BDC0000186A0FFFFD8F0000003E8FFFFAF
:104EB000FF9C0000000AFFFFFFFFFFDF0A800003E6
:104EC0004BC0FFFF736000000E10FFFFFDA8000045
:104ED000003CBFAAAAAAAAAAAAAAAAAAAAAAAAAA35
:104EE000AAAAAAAAAAAAAAAAAAAAAAAAAAAAAAAA22
:104EF000AA200CDCA911A0DF20A2DBF070A569D0EC
:104F0000034CF9D8A24EA00020D4DBA56E100F20D0
:104F1000CCDCA94EA000205BDCD00398A40720FEC7
:104F2000DB984820EAD9A94EA0002028DA20EDDF3E
:104F3000684A900AA561F006A56649FF856660810A
:104F400038AA3B29077134583E5674167EB31B7736
:104F50002FEEE3857A1D841C2A7C6359580A7E75DE
:104F6000FDE7C680317218108100000000A9BFA0C3
:104F7000DF2028DAA570695090032023DC855620B5
:104F80000000000000000000000000000000000021
:104F90000000000000000000000000000000000011
:104FA0000000000000000000000000000000000001
:104FB00000000000000000000000000000000000F1
:104FC00000000000000000000000000000000000E1
:104FD00000000000000000000000000000000000D1
:104FE00000000000000000000000000000000000C1
:104FF00000000000000000000000000000000000B1
:1050000000000000000000000000000000000000A0
:105010000000000000000000000000000000000090
:105020000000000000000000000000000000000080
:105030000000000000000000000000000000000070
:105040000000000000000000000000000000000060
:105050000000000000000000000000000000000050
:105060000000000000000000000000000000000040
:105070000000000000000000000000000000000030
:105080000000000000000000183C3C181800180048
:10509000363600000000000036367F367F36360098
:1050A0000C3E031E301F0C00006333180C666300B7
:1050B0001C361C6E3B336E00060603000000000029
:1050C000180C0606060C1800060C1818180C06001A
:1050D00000663CFF3C660000000C0C3F0C0C00001E
:1050E00000000000000C0C060000003F0000000063
:1050F00000000000000C0C006030180C06030100DA
:105100003E63737B6F673E000C0E0C0C0C0C3F0073
:105110001E33301C06333F001E33301C30331E005C
:10512000383C36337F3078003F031F3030331E0069
:105130001C06031F33331E003F3330180C0C0C00C9
:105140001E33331E33331E001E33333E30180E0021
:10515000000C0C00000C0C00000C0C00000C0C06E9
:10516000180C0603060C180000003F00003F00006A
:10517000060C1830180C06001E3330180C000C00FA
:105180003E637B7B7B031E000C1E33333F333300B7
:105190003F66663E66663F003C66030303663C006E
:1051A0001F36666666361F007F46161E16467F004F
:1051B0007F46161E16060F003C66030373667C00CE
:1051C0003333333F333333001E0C0C0C0C0C1E00F6
:1051D0007830303033331E006766361E366667001F
:1051E0000F06060646667F0063777F7F6B6363006A
:1051F00063676F7B736363001C36636363361C00F5
:105200003F66663E06060F001E3333333B1E3800F2
:105210003F66663E366667001E33070E38331E0053
:105220003F2D0C0C0C0C1E003333333333333F0053
:1052300033333333331E0C006363636B7F77630058
:105240006363361C1C3663003333331E0C0C1E00A4
:105250007F6331184C667F001E06060606061E0098
:1052600003060C18306040001E18181818181E008D
:10527000081C36630000000000000000000000FF72
:105280000C0C18000000000000001E303E336E00C1
:105290000706063E66663B0000001E3303331E0011
:1052A0003830303E33336E0000001E333F031E00A3
:1052B0001C36060F06060F0000006E33333E301F0B
:1052C0000706366E666667000C000E0C0C0C1E009E
:1052D000300030303033331E070666361E36670026
:1052E0000E0C0C0C0C0C1E000000337F7F6B630057
:1052F00000001F333333330000001E3333331E00EE
:1053000000003B66663E060F00006E33333E307889
:1053100000003B6E66060F0000003E031E301F00BB
:10532000080C3E0C0C2C18000000333333336E0095
:1053300000003333331E0C000000636B7F7F3600A8
:10534000000063361C36630000003333333E301FE9
:1053500000003F190C263F00380C0C070C0C3800DD
:105360001818180018181800070C0C380C0C070037
:105370006E3B000000000000000000000000000084
:10538000A2A0D0EBE5B9334487C068B6B72699C769
:1053900016035500530042002000530065007200C0
:1053A000690061006C0018035400650065006E0020
:1053B000730079006400750069006E006F000403DB
:1053C000090409024B00020100C032080B0002026E
:1053D000020100090400000102020100052400107E
:1053E0000105240101010424020605240600010729
:1053F00005820310001009040100020A00000007E2
:105400000503024000000705840240000009024B2A
:1054100000020100C032080B000202020100090470
:105420000000010202010005240010010524010111
:10543000010424020605240600010705820310006A
:105440000509040100020A0000000705030200022A
:1054500000070584020002000A060002EF02014074
:045460000100010046
:105464000000000000000000000000000000000038
:105474000000000000000000000000000000000028
:10548400024B1B780BB103F015BF7047498600200F
:105494000E480F4B02881B6833F8121001320D4B73
:1054A40019800D4B19884B00013B13409BB20380BC
:1054B40013B90A4A137004E0994205D10122074B3B
:1054C4001A704022064B1A60704700BF187B0020F8
:1054D4004065002022403840167B0020843A00209A
:1054E40008E200E0324A70B5B2F86E30C3F30E033E
:1054F400A2F86E30B2F8743023F030031B041B0C96
:10550400A2F8743072B62B4C2B4B21682B4D29B169
:10551400187801210EF0D2F8002303E018780EF079
:10552400CDF801232B6023680133236040F20D235F
:105534002168B1FBF3F203FB1213214A23602368B1
:105544001268283BD3401F4A126893422CD21E4A49
:105554001E4916681E4A1F4D14680A686343F018F2
:1055640010601D4A126812F0800F15BF02F00F027E
:1055740002F00C02D2189B1814BFB3189B192A68A6
:105584001360164A0B79D3762B79D37620F01F0259
:105594002318BFF34F8F12490A6020329342FBD87D
:1055A400BFF34F8FBFF36F8F62B6BFF34F8F70BDE2
:1055B40000401E40E06400208A3A0020C4790020A4
:1055C400F0640020147A002020420020787A002021
:1055D400187A0020707A0020287A002000800E407B
:1055E40070EF00E0194B1A78194B70B5194E1A4D2B
:1055F4001A4C8AB131881B682868984731882A6810
:10560400490822F01F0302EB8102BFF34F8F23608E
:1056140020339A42FBD814E031882A6848081B6872
:1056240002EB8000984733882A685B089900531876
:1056340023F01F020B44BFF34F8F226020329342AA
:10564400FBD8BFF34F8FBFF36F8F70BD843A002038
:10565400E4640020167B00200041002070EF00E08D
:1056640010B5054C237833B9044B13B10448AFF398
:1056740000800123237010BDF05F002000000000B3
:10568400940E0100084B10B51BB108490848AFF34C
:1056940000800848036803B910BD074B002BFBD0FA
:1056A400BDE81040184700BF00000000F45F002070
:1056B400940E0100C03E0020000000000122014BB6
:1056C4001A707047498600200022026070477047B4
:1056D4004160704710B50446FFF7F6FF0023044904
:1056E4002046638223756375FFF7F2FF204610BDE1
:1056F40080841E0010B50446FFF7E9FF204610BD64
:1057040081607047418270470175704701440A7394
:1057140070470000FF2149F21113014AD154704728
:10572400678600200F4A49F21113017BD35C11B93B
:1057340043F03C0303E003F0DF0343F01C03417B2D
:1057440009B103F0FB03817B09B103F0F703C17BCB
:1057540009B103F0EF0349F21111535449F21F1137
:105764005354704767860020094B49F2221149F2CD
:10577400201259569A5C0029017CA8BF42F080028D
:1057840009B102F07F0249F220115A54704700BF58
:1057940067860020194A49F2201370B5448AD55C03
:1057A400E1B225B9002C14BF0B46FF231FE0260AE3
:1057B400B54204D1002914BF0B46FF2300E0FF23A8
:1057C400F72D07D1007D90B174B1F72E0CD101F003
:1057D400FD030CE0DF2D0AD1407D40B134B1DF2E52
:1057E40004D101F0FE0302E0FD2300E0FE2349F2B0
:1057F4002111535449F22F11535470BD6786002070
:10580400F8B5404C49F2271649F2261E49F22D12EA
:1058140014F806C049F22E1314F80E1049F21917A1
:10582400A55C49F2181251EA0C21E35CA25CE75D25
:1058340005D145F0400549F22D1165540BE001F105
:10584400FF3C023989B204F80EC04FEA112E04F865
:1058540006E00029EDD049F229162A49A65D46B38F
:1058640052EA072215D149F2281245F02005A15C1D
:1058740049F21812A15449F2191249F22911A654F5
:105884000022625449F22A11625449F22D12A5549D
:105894000FE002F1FF3E023A49F2181792B201F802
:1058A40007E049F219174FEA122E01F807E0002A1F
:1058B400D9D003F07F031D4223D0806803F09AFB04
:1058C400F8B1690616D549F22B120E4BA25C5206AA
:1058D4000BD549F224110C4A585C49F2261112885E
:1058E400585449F2271112125A5405F0BF0549F2CF
:1058F4002D13E554AB0642BF25F0200349F22D12C7
:10590400A354F8BD678600208B17012010B5044608
:10591400FFF776FF2046FFF705FF2046FFF724FF39
:105924002046FFF737FF23680133236010BD0000D2
:1059340010B50446FFF7C8FE00230449204623722D
:105944000123A373FFF7C4FE204610BD20E8100016
:1059540010B50446FFF7BBFE204610BD104B0022D5
:105964001A70FF225A70A0229A705F22DA70A7225E
:105974001A715C225A710B229A71D822DA71C822E8
:105984001A72F5225A72F2229A729F22DA72F32262
:105994001A739E225A7393229A73FA22DA73704707
:1059A400487B0020EF2910B510D8094A49F20F03AB
:1059B4000846D35C074A03F00703D45C03F0D4FB26
:1059C40000F5A07300F8014B9842FBD110BD00BF55
:1059D40067860020487B00202DE9F04F98468BB065
:1059E400654849F20303B8F1100F0191C35C04D177
:1059F400C3F34503162BC8BF521008FB02FB019BDF
:105A04005B44EF2B00F3B48049F2020349F2050131
:105A14000024C35C415C03F07F079B00890103F40D
:105A240000737A4301F4E051C7F128059BB2AD003D
:105A34001944A3F5D8439BB211441A44411883185E
:105A440002914E4A039349F20F03C35C03F007012A
:105A54001B09D35C515C8DF82430FB008DF82510B4
:105A6400059325EAE5730793444580F28180019B01
:105A740003EB0B00204403F077FB9DF8252003463D
:105A8400191A8D4202DD03F8012BF9E7079B002662
:105A9400DFF8F0E0C3183A4ADFF8E0C000931EF8DC
:105AA400093B009903F00F0332F813309DF82420CA
:105AB400234404920693BE424BDA029B40F6FE70E6
:105AC400069A9B5D03FB08239BB203F55F42FF32FA
:105AD40092B28242284A9CBF03F5C0439BB212F89B
:105AE4000390039B9B5D03F0070203F008031CF87B
:105AF40002A003F0FF028DF826A08BB94B1C09FA13
:105B040002F001320133000656BF9DF8100003F87D
:105B140002AC03F8020C082AF1D108310136CAE7B5
:105B24009EF800301B091CF803308DF82730002341
:105B340009FA03F20AA801EB030AC2F38112024430
:105B440012F8042CCA5402338AF80120082BEFD12E
:105B5400E3E7059B009A1A4410469DF82520034666
:105B6400191A8D4202DD03F8012BF9E701347BE7B2
:105B74000BB0BDE8F08F00BF67860020487B002093
:105B8400180F00206C160120002383737047807B5C
:105B940070470000F8B547230D4601680446B1FB81
:105BA400F3F203FB1213F3B9344849F2030649F242
:105BB4000403825DC15CD31143EA4101D3074BD492
:105BC400B1F59C7F3ADC0823013149F2030649F21E
:105BD4000407825D02F07F0242EAC11282554A1034
:105BE400C255A2891AB923681D442560F8BD678986
:105BF400B9421FD33A4491421CDAC81B591E90FB88
:105C0400F3F203FB1202D2B28A42ECD1227A394671
:105C14002046FFF7E1FE237A184A0133DBB22372F0
:105C2400925DC2F345029342DDDB0023237201231C
:105C3400A373D8E72046FFF7B5FED4E7C2F34502C5
:105C44000823D200A281A2890221C2F1F00292FBB0
:105C5400F1F200216281B8E7B1F59C7F01DC1023E9
:105C6400B2E7C2F345021201A281835DC3F3450387
:105C7400162B01DDDB00A3811023E4E767860020F7
:105C84000020704770477047704701207047704785
:105C9400006910B10368DB6818477047006910B1E8
:105CA40003681B6918477047006910B103685B6992
:105CB40018474FF0FF307047006910B103689B69C3
:105CC4001847704707B5006910B94FF0FF3009E075
:105CD400036801220DF107019B6898470028F4D05E
:105CE4009DF8070003B05DF804FB07B500698DF863
:105CF400071028B1036801220DF10701DB689847FA
:105D040003B05DF804FB0000314B012201461A7018
:105D1400304B93F86E00402820D13D291BD007DC7E
:105D2400242916D0262918D0222908BF232115E0BA
:105D3400E0290CD003DCA72908BF5E210EE0E72987
:105D440003D0E92908BF402108E07B2106E07D213A
:105D540004E05D2102E07E2100E07C211E4B1B78E3
:105D6400002B32D0D72920D00ADC0A2922D02029BE
:105D740025D009292BD1194A137823F0400322E0B6
:105D8400D92903D00CDBDA2905D07047134A1378DC
:105D940023F0080317E0114A137823F0040312E0F8
:105DA4000E4A137823F002030DE00C4A137823F013
:105DB400010308E0094A137823F0100303E0074ABB
:105DC400137823F020031370704703F037BB704738
:105DD4005B7B0020C04C0020853A002036860020E2
:105DE400314B012201461A70304B93F86E00402863
:105DF40020D13D291BD007DC242916D0262918D010
:105E0400222908BF232115E0E0290CD003DCA729AF
:105E140008BF5E210EE0E72903D0E92908BF40212D
:105E240008E07B2106E07D2104E05D2102E07E2183
:105E340000E07C211E4B1B78002B32D0D72920D0C8
:105E44000ADC0A2922D0202925D009292BD1194A74
:105E5400137843F0400322E0D92903D00CDBDA297C
:105E640005D07047134A137843F0080317E0114A2A
:105E7400137843F0040312E00E4A137843F002034C
:105E84000DE00C4A137843F0010308E0094A137843
:105E940043F0100303E0074A137843F02003137020
:105EA400704703F0BDBA70475B7B0020C04C0020F4
:105EB400853A00203686002013B50346006D0C4653
:105EC40028B10DF1060201A909F04BFD08E0586D57
:105ED40008B9002021E00DF1060201A907F0D2FB68
:105EE4000028F6D0BDF80430BDF806200BB9002A0E
:105EF400EFD002F01F0149002170C2F34511D21204
:105F04006170A27003F01F022271C3F343125B128B
:105F1400013A03F5EA636271A37102B010BD13B5CF
:105F24000346006D0C4628B10DF1060201A909F0E3
:105F340028FD08E0586D08B9002021E00DF10602A3
:105F440001A907F0AFFB0028F6D0BDF80430BDF876
:105F540006200BB9002AEFD002F01F01490021707E
:105F6400C2F34511D2126170A27003F01F022271B4
:105F7400C3F343125B12013A03F5EA636271A3713E
:105F840002B010BD38B5856D0446BDB94FF48070BC
:105F94000FF07CFA0146A06570B10570206D20B148
:105FA4004FF480720AF0C6FE08E0606D30B14FF421
:105FB400807208F0C1FE01E0014BA365A06D38BDFD
:105FC4003C860020D0B5046D6CB1012B08BF002ABB
:105FD40014D21146204609F0DCFA78B1204609F0C3
:105FE400DDFE58B1D0BD446D44B1204607F093FCAA
:105FF40020B12046BDE8D04008F058BA0020D0BDFA
:1060040010B5044600684368013B43603BB903682C
:10601400DB6A9847206810B103685B6898470023DF
:10602400236010BD054B10B503600446036913B12A
:106034001030FFF7E5FF204610BD00BFF406002036
:1060440010B50446FFF7EEFF142120460EF020FFA2
:10605400204610BD10B5084C04F13C00FFF7E2FFE8
:1060640004F12800FFF7DEFF04F11400FFF7DAFF64
:106074002046FFF7D7FF10BD8039002010B1036818
:106084009B681847704710B103681B6B184770472B
:1060940038B50B6804460D4613B15A6801325A608C
:1060A40023691BB104F11000FFF7AAFF2B682046F7
:1060B400236138BD036D13B1586900217047436DE6
:1060C40013B193E8030070471846F6E7036D13B164
:1060D400D86900217047436D13B118695969704735
:1060E4001846F6E770B5044608460D460FF037FB30
:1060F40023680246294620465B68BDE8704018477D
:1061040038B50546FFF7EEFF044628460EF024FD99
:10611400204438BD38B505460EF07DFD04462846BA
:106124000EF01AFD204438BD826B30B562B113788D
:1061340003F0080303F0FF00FBB1D3695069181A98
:106144001BD56FF0004018E0C06BB0B190F831304F
:106154001B0707D5D0E90445D0E90023A01A65EB55
:10616400030101E00020002100236FF000428B4274
:1061740008BF824201D2104630BD30BD08B5103090
:10618400FFF7D2FF08BD08B51830FFF7CDFF08BDF3
:10619400836B1BB11B7813F0700F05E0C06B30B13B
:1061A40090F8313013F0500F14BF012000207047D5
:1061B40008B51830FFF7ECFF08BD10B504461830D9
:1061C400FFF7E6FF60B1206D10B1002109F0E1F99D
:1061D400606D28B100220023BDE8104007F09BBB8E
:1061E40010BD836B23B9C06B003018BF012070470A
:1061F4000120704708B51830FFF7F3FF08BD10B54C
:106204000446806D18B10FF049F90023A3651834D2
:106214002046FFF7E6FF20B12046BDE810400AF013
:1062240072BF10BD064B10B503600446FFF7E7FFCD
:10623400044B04F11800A3600AF065FF204610BD6A
:10624400440700209405002010B50446FFF7EAFF38
:106254005C2120460EF01CFE204610BD0346806BD8
:1062640008B109F066B9D86B08B107F03FBB4FF02D
:10627400FF30704708B51030FFF7F0FF08BD08B5D0
:106284001830FFF7EBFF08BD0346806B08B109F037
:1062940095B8D86B08B107F067BA4FF0FF30704774
:1062A40007B501220DF107011030FFF7EDFF0128BA
:1062B4000CBF9DF807004FF0FF3003B05DF804FBFE
:1062C40008B51830FFF7E0FF08BDD0B4846B44B1C3
:1062D400012B08BF002A09D220461146D0BC09F080
:1062E40058B9C06B10B1D0BC07F015BB0020D0BCAE
:1062F400704738B50146049814461D4610B901F19B
:1063040018001DE001280AD10B6D01F118000BB132
:106314005A6912E04B6D7BB1D3E900230EE00228E9
:1063240011D10B6D01F118000BB1DA6905E04B6D69
:1063340013B1D3E9042301E00022002312196B41B5
:10634400FFF7C3FF38BD002038BD0346806B08B19A
:1063540009F04ABAD86B08B107F0B8BE704708B55F
:106364001030FFF7F2FF08BD08B51830FFF7EDFF56
:1063740008BDF0B5D0F838E09DF814409DF81850E9
:106384009DF81C609DF82070BEF1000F08D008979E
:106394007046079606950594BDE8F04009F0A7BC41
:1063A400C06B38B10897079606950594BDE8F04090
:1063B40007F0F2BFF0BD1FB58A79A2F150031B06A6
:1063C40011D40C7802F26C724B79183003944C7827
:1063D40001330294DBB28C78019409790091042191
:1063E400FFF7C7FF00E0002004B010BD1FB58A7995
:1063F400A2F150031B0611D40C7802F26C724B7993
:10640400183003944C7801330294DBB28C780194F5
:10641400097900910221FFF7ACFF00E0002004B0ED
:1064240010BD0346806B08B109F0ECBCD86B08B111
:1064340008F09CB8704708B51830FFF7F2FF08BDA4
:1064440008B51030FFF7EDFF08BD07B502AB012218
:10645400103003F8011D1946FFF7E3FF03B05DF8A0
:1064640004FB000000234FF47A7203710373054B9D
:10647400826003600B69036113B15A6801325A6088
:10648400704700BFF406002010B50446006940B10F
:106494000368DB6A984704F11000BDE81040FFF779
:1064A400AFBD10BD38B500250E4B04461031456014
:1064B400183040F8183C11F80C3C00F80C3C0A4B1E
:1064C40040F8103C51F8083C40F8083C11F8043CF2
:1064D40000F8043C0AF0E6FD044BA5652046A360E1
:1064E40038BD00BF44070020A0070020200700207B
:1064F4002DE9F04395B000251C4B4FF47A760DF14D
:1065040050082A461831044604A848F8503D8DF82E
:10651400045002968DF80C50129513950AF046FE1D
:1065240004A8DFF85090FFF75CFE80B15C200EF009
:10653400ADFC07464146FFF7B5FF7B682571013383
:10654400A6602573C4F8009027617B6005E0207184
:10655400A6602073C4F800902061054B04A8009342
:106564000AF0D1FD204615B0BDE8F08320070020D5
:1065740094050020F4060020012B70B5044694B065
:1065840005D0022B40F2022318BF002301E044F29D
:106594000223043168460AF099FE04A8FFF721FE9D
:1065A400114E90B15C200EF071FC69460546FFF770
:1065B40079FF00234FF47A722660237123736B688A
:1065C400A260013325616B6006E04FF47A73207199
:1065D4002073A36026602061044B04A800930AF092
:1065E40092FD204614B070BDF406002094050020EE
:1065F40070B5324B8AB00024314A00934FF47A7359
:10660400304905A8029323468DF804408DF80C40C8
:106614000494FFF7B1FF2C4E09A92B48FFF738FD6E
:1066240005A8FFF7FFFC316929B10B68002205A812
:10663400DB6B984703E0244905A8FFF713FF09A97A
:106644006846FFF725FD05A8FFF7ECFC0498FFF763
:106654001AFD48B3049820B103685B6B984705465C
:1066640000E01A4D29461A48FFF74AFD049868B11C
:1066740003689B6B984748B1164928460FF05DF8AC
:1066840068B1154928460FF058F840B1134B18204B
:106694001722294600FB043001340FF07DF86846C8
:1066A400FFF7F2FE3F2CBEDD0748FFF7EDFE68461C
:1066B400FFF7B8FC20460AB070BD00BFF406002006
:1066C400F68500200C600020D4390020BB3800205F
:1066D400703900206335002062350020CD7C002015
:1066E4000146024808B5FFF70BFD08BD70390020CC
:1066F4000146024808B5FFF70DFD08BD70390020BA
:1067040010B5064C01460023102220460EF048FA2C
:106714002046BDE810400EF01FBA00BF70390020BB
:10672400044B28B91A780AB1187001E001221A70D2
:1067340018787047447B0020014B1888704700BFCD
:10674400147B00202DE9F04F232085B00CF0D6FFF8
:1067540000284FF0240014BF002404240CF0CEFFC2
:1067640010B944F00804A4B226200CF0C7FF10B9F5
:1067740044F00104A4B225200CF0C0FF10B944F089
:106784000204A4B222200CF0B9FF10B944F01004A2
:10679400A4B2A04B1B780BB92402A4B29E4B1B7865
:1067A4005E0744BF44F00404A4B21D0744BF44F090
:1067B4000804A4B298074FF0290044BF44F002042F
:1067C400A4B2D90744BF44F00104A4B2DA0644BF1A
:1067D40044F01004A4B29F0644BF44F02004A4B2C1
:1067E4005E0644BF44F04004A4B20CF087FF10B925
:1067F40044F02004A4B228200CF080FF10B944F027
:106804004004A4B2854A4FF0FF33854D0027106839
:106814000DF1040B2B6001AB5168DFF808A203C330
:10682400906818601BF81760012130460CF078FF5F
:10683400002130460CF042FF13200CF05FFFB0FA49
:1068440080F812200CF05AFF00284FEA58184FF035
:10685400110014BF0023022348EA03080CF04EFF82
:1068640000284FF0050014BF0023042348EA03085E
:106874000CF044FF00284FF01D0014BF0023082330
:1068840048EA03080CF03AFF00284FF01E0014BF3A
:106894000023102348EA03080CF030FF00284FF0CF
:1068A400200014BF0023202348EA03090CF026FF2C
:1068B40000284FF00101304614BF4FF000084FF09C
:1068C40040080CF0FBFE304649EA080805210CF0AC
:1068D40027FF544E0AF807800137062FA2D1737997
:1068E40003F0080202F0FF011AB123F008030121AA
:1068F4007371727902F0100000F0FF0320B1494B6C
:1069040022F010025A7101230027D5F800E038461E
:10691400325C002A18BF864600F1010018BF012727
:106924000628F5D10FB1C5F800E0550644BF44F080
:106934000204A4B2900644BF44F00104A4B2D707F1
:10694400394F48BF44F00804BE4648BFA4B25507B7
:10695400364D44BF44F00404A4B2900738682A6852
:1069640048BF44F01004A0EB020248BFA4B2642A5A
:1069740007D92F4A286015780DB9012500E00025B4
:1069840015702C4D2C4F2D4A13B101232B703CE074
:106994002B70002938D097F800C02949BCF1000FAA
:1069A4001BD1D1F800E0BEF1000F03D1254B1860D4
:1069B400012325E00EF1010EBEF1010FC1F800E044
:1069C4001FD90B601F490968401AB0F5FA7F18D225
:1069D400117801B90123137013E00868012810D15C
:1069E400DEF80000DFF85CE0DEF800E0CEEB00004B
:1069F400B0F57A7F05D91078B0FA80F040091070AC
:106A04000B6001233B7000E039701378E3B1084B4D
:106A140019781EE0447B0020368600201C0D0020DF
:106A2400D0390020EF850020087B00201C7A00204C
:106A34005A7B0020EE820020ED820020587B00204B
:106A440034650020006500203B780BB9297801B13A
:106A540001210E200CF032FE3B78002B3AD0327923
:106A640044F04003102A9BB202D144F06004A3B264
:106A74002A78002A2DD0194B9C6BDA6C42F0010263
:106A8400DA649A6B22F002029A639A6B9207FCD43E
:106A940072B61248036D426D466D1049B242056DDF
:106AA400F8D1AB42F6D1D20B42EA434302338B65B1
:106AB4008A6D0A489342FBD144F002038363836BDB
:106AC400064A9B07FBD5936B43F04003936330BFA7
:106AD400FDE71C46204605B0BDE8F08F00400D40A0
:106AE40008B5FFF72FFE034A1388108020EA03033A
:106AF40098B208BD147B00201B4B1C4A19781278ED
:106B04001B4B30B549B10AB11A4A0FE01A4A127840
:106B14000AB11A4A0AE01A4A08E00AB1194A05E019
:106B2400154A12780AB1184A00E0184A1A60184A3D
:106B34001268002A15DB1102164801F47F41825CB9
:106B440015481143002230F8125054008D4205D1EB
:106B54000021124A1B681160185B30BD01322A2AD9
:106B6400F1D1002030BD00BF587B0020ED82002011
:106B74008079002030110020EE820020DC100020FB
:106B84008810002034100020E00F00208C0F00201B
:106B9400D0390020EF850020380F00203465002014
:106BA40008B5022123200CF0BBFD022124200CF0A7
:106BB400B7FD022126200CF0B3FD022125200CF0A4
:106BC400AFFD022122200CF0ABFD022129200CF0A4
:106BD400A7FD022128200CF0A3FD01210E200CF0BA
:106BE4009FFD01210E200CF069FD012110200CF005
:106BF40097FD012106200CF093FD012118200CF0D3
:106C04008FFD012119200CF08BFD01211C200CF0BB
:106C140087FD01211F200CF083FD012110200CF0C1
:106C24004DFD012106200CF049FD012118200CF036
:106C340045FD012119200CF041FD01211C200CF01F
:106C44003DFD01211F200CF039FD022113200CF021
:106C540067FD022112200CF063FD022111200CF0CB
:106C64005FFD022105200CF05BFD02211D200CF0CC
:106C740057FD02211E200CF053FD02212020BDE807
:106C840008400CF04DBD000030B50B4C01250B4BFA
:106C940085B0204600211D7003F0F6F81F2203235F
:106CA400204602958DE80C000022054B114603F0A6
:106CB4003BF905B030BD00BF5E860020823A00205B
:106CC400E434002041F2100303402DE9F04F934DCA
:106CD4009BB0002B31D092490AA80EF038FD91499F
:106CE4000AA80EF01BFD90490AA80EF017FD0AA988
:106CF4008B480EF02CFD8D48FFF7F2FC8848FFF717
:106D0400EFFC05A80023864A8949FFF735FC09985A
:106D140008B981240BE003689B6B98470028F8D0DE
:106D2400844B00241C60FFF763FC834B1860012331
:106D340005A82B70FFF776F973E000F02004A1B2E8
:106D440099B1012378497D4882242B700EF0FFFC11
:106D540073497B480EF0FBFC724979480EF0DEFC67
:106D6400764977480EF0DAFC5BE000F04004A2B20A
:106D740032B1012308462B70FFF7D2FC0C4650E0D9
:106D840040F20444044044B16A490B68002B43D0E8
:106D94000120013B28700B6042E040F201130340E4
:106DA4006BB1644A1368082B03DD0121093B297088
:106DB40003E08BB30121013B2970136031E040F6FD
:106DC4000804044064B15C4A5A4914680A68601EA5
:106DD400904221DD2CB301320A6001222A701BE0AB
:106DE40040F202230340BBB1534B52491A680B686B
:106DF400A2F109009842084605DD22B109330B606F
:106E040001232B700DE0511E8B4207DA42B101338E
:106E1400036001232B7001E01C4602E0002400E023
:106E240014462B78002B74D0434B1A689B46002AD7
:106E34006FD090230126202230214248DFF810A190
:106E44008DE84800C023002603F04CF8394A374641
:106E540013689146082BD4BF0023043BCAF80030C2
:106E6400DBF8002097421FDB00261F200323C822E3
:106E740030218DE84900344B324803F055F808239B
:106E8400C82278210093C0232E48019603F02AF8E3
:106E9400FF230296C822009378210196274B2948A4
:106EA40003F042F82E7034E0DAF800309F422BDB16
:106EB40033449A4227DD254A4FF0180808FB072877
:106EC400D9F8002093424FF0010306F10202029325
:106ED4004FEA02120ED1FC21E02312B219488DE8C8
:106EE4000A004346302103F01FF841460E480EF0D5
:106EF4002EFC08E00193FF2312B230210093434695
:106F0400104803F011F80136082E07F10107A7DD38
:106F1400AAE720461BB0BDE8F08F00BF823A0020EC
:106F2400F6850020653400209D7C0020F834002084
:106F34000C600020D4790020047A0020B57C002065
:106F44005D7B00205E86002008350020CD7C00207B
:106F54000C7A0020014B1878704700BF853A002056
:106F6400034B18B101221A70FFF78EBE18707047D8
:106F7400853A002000487047F68500202DE9F0414D
:106F8400044686B01D4D0027DFF884802869FFF78A
:106F94007AF80646D8F8100086F00106FFF773F871
:106FA400F6B2864208D101371435042FEED11448C5
:106FB4000024FFF795FB1DE022460023114901A898
:106FC400FFF7DAFA05A92846FFF762F80069FFF728
:106FD4005AF8044601A8FFF725F824B17C1C204682
:106FE400FFF78EFB06E008492846FFF751F80748EB
:106FF400FFF776FB204606B0BDE8F081803900201B
:10700400113500200C600020E439002026350020D2
:10701400D439002030B50B4B87B00D46013A14210A
:10702400044601A801FB0231FFF71CFA21462A4657
:107034000598FFF723F8044601A8FEF7F3FF20465E
:1070440007B030BD8039002010B50B4B0138142433
:1070540086B004FB003401A82146FFF703FA01A817
:10706400FFF712FA01A8FEF7DDFF04492046FFF7F7
:107074000FF806B010BD00BF80390020E4390020AD
:1070840030B5044687B0134DFFF72AFB2246002390
:10709400114901A8FFF770FA05A92846FEF7F8FF81
:1070A4000069FEF7F0FF044601A8FEF7BBFF6CB1D0
:1070B4000A48FFF715FB286910B103689B6A9847D3
:1070C4000446FFF715FB0348FFF7DEF9204607B037
:1070D40030BD00BFE83900200C6000204A35002094
:1070E400F8B52D4940F2EE272C4B0C462C4D186870
:1070F4002C4E0A784AB12A78D20706D51A68D6F8EF
:1071040000E0CEEB02020E2A09D81A6894F800E0D7
:10711400121ABEF1000F3CD0B2F5FA6FE9D903F0B0
:107124004BF8214B214A9A64214ADA64FE21214812
:1071340006F074F940B920492048FEF7E1FF4FF406
:107144007A700CF0A5FAF1E700241D4D1D491E4884
:107154000EF0FDFA281914341C49FEF799FF502C3F
:10716400F8D11B4CFFF744FA1A4920601348FEF784
:10717400B9FF21681148FEF7CDFFFFF711FD00228A
:10718400154B1A700122154B1A70BDE8F840FFF731
:107194007BBDBA42C2E700BF63860020087B0020A3
:1071A40062860020DC860120C04C0020810900009A
:1071B400A90800000C6000208635002070390020EA
:1071C40080390020A3350020F6850020E439002012
:1071D400047A0020A7350020447B0020853A002053
:1071E4000022014B1A7070473686002070B54B4858
:1071F40000244B4D20264B4B44608460C0F824038C
:10720400C0F84403036004F075FD21466C60AC6073
:1072140032462C6105F128006C61EC6185F8204050
:107224006C620CF0E5F9404B284685F8854203F181
:1072340040022B606C332C65EA60AB616C6585F8A9
:107244007840C5F8804285F8844285F8864285F8FE
:10725400874205F02BFA3548354D364B446084603F
:10726400C0F89006036080F87546C0F87846C0F808
:107274007C4680F8804680F8A44604F077F93246CC
:1072840021466C6005F11C00AC602C612C75AC616E
:107294000CF0AEF9284B284685F841402B60383372
:1072A400EC63EB6085F8404085F8424085F8434044
:1072B4006C64AC64EC642C6505F0E4FE1F4D204B5B
:1072C4006C6028462B6005F59F63AC606B6305F525
:1072D400A7632D62AB6305F5AF631A4EEB6305F547
:1072E400B7636B644023A5F84A305023A5F84C30AB
:1072F40005F084FD144B314614482B60144D2A4686
:107304000EF079F82A46134920460EF074F82A46FE
:1073140031461148BDE870400EF06DB800490020B8
:10732400C04C0020C40700206C060020404200200E
:10733400987A0020B8050020F0050020604F002056
:10734400D4050020C50B000078050020D4390020A6
:1073540014390020F50B0000E839002083885A1CFA
:10736400828018467047000083885A1C10B592B278
:10737400044C8280E15C02338380A05C01EB00203A
:1073840080B210BD6786002083885A1C8280014A1F
:10739400D05C7047678600200020704782880649C9
:1073A400531C9BB283808A5C90B2120648BF40F49F
:1073B4007F40184480B270476786002082880B495A
:1073C40010B5541CA4B284808B5C023282800A5DA6
:1073D40043EA02235A1C03F47F40CB5C51FA82F245
:1073E400105C03EB002080B210BD00BF6786002054
:1073F40083885A1C8280034AD25C4378D018C0B276
:10740400704700BF6786002083885A1C8280034A25
:10741400D25C8378D018C0B2704700BF6786002062
:10742400838807495A1C92B210B58280CC5C02331F
:10743400838043788A5CE01800EB022080B210BDA0
:1074440067860020838807495A1C92B210B582804F
:10745400CC5C0233838083788A5CE01800EB0220E2
:1074640080B210BD6786002083885A1C8280064A39
:10747400D15C43780B44DBB2591CD35CC9B2505C79
:1074840003EB002080B27047678600208288531C7B
:107494008380064B995C4A1C595CD2B29A5C83780F
:1074A400C81800EB022080B2704700BF6786002036
:1074B400012241F20843C254704700002D4B027868
:1074C400F0B55D5C8379AC1885EA020703F001012D
:1074D400214411F0FF0F0C460CBF43F0020323F0CC
:1074E40002038371837913F0080F24D002F00F0E86
:1074F40005F00F067546354403F001063544092DA1
:10750400C8BF8C1D21064CBF63F07F0303F07F03CB
:1075140017F0800F8371837905D16240160602D576
:1075240043F0400301E023F04003992C83718379F5
:107534001BD9603416E00D064CBF63F07F0303F0E3
:107544007F0317F0800F8371837905D14A401206B7
:1075540002D543F0400301E023F04003FF29837187
:10756400837902DD43F0010301E023F00103837119
:107574000470F0BD678600200B4B5A5C03781A40F8
:10758400837912F0800F02D063F07F0305E003F0EB
:107594007F0312B943F0020303E08371837923F07C
:1075A40002038371027070476786002010B5114C86
:1075B4008379625C12F0800F4FEA4202D2B214BFA8
:1075C40043F0010323F0010312F0800F83718379E8
:1075D40002D063F07F0305E003F07F0312B943F0A8
:1075E400020303E08371837923F0020383716254FD
:1075F40010BD00BF678600200278837912F0800FE7
:107604004FEA4202D2B214BF43F0010323F0010354
:1076140012F0800F8371837902D063F07F0305E059
:1076240003F07F0312B943F0020303E0837183790B
:1076340023F002038371027070478379DB0758BF1C
:10764400818070478379DB0748BF818070478379E5
:107654009B0748BF818070470D4B5A5C0178837942
:10766400114022F03F0211F0800F14BF63F07F033A
:1076740003F07F038371837903F03F031343837122
:1076840011B943F0020301E023F002038371704750
:107694006786002090F90630002BB8BF81807047C0
:1076A40083799B0758BF8180704790F90630002B7F
:1076B400A8BF8180704783795B0658BF818070477B
:1076C40083795B0648BF81807047837923F0010387
:1076D40083717047837923F008038371704783793A
:1076E40023F0040383717047837923F0400383718B
:1076F400704700000F4A0378525C9A1A8379FF2A74
:1077040094BF43F0010323F0010312F0800F83714F
:10771400837914BF63F07F0303F07F0312F0FF0F3C
:10772400837183790CBF43F0020323F00203837156
:10773400704700BF678600200F4A4378525C9A1A4C
:107744008379FF2A94BF43F0010323F0010312F06D
:10775400800F8371837914BF63F07F0303F07F0389
:1077640012F0FF0F837183790CBF43F0020323F0FF
:1077740002038371704700BF678600200F4A837835
:10778400525C9A1A8379FF2A94BF43F0010323F0D1
:10779400010312F0800F8371837914BF63F07F03B8
:1077A40003F07F0312F0FF0F837183790CBF43F062
:1077B400020323F002038371704700BF6786002031
:1077C4000C4B10B55A5C013A12F0800FD4B21A4631
:1077D400837914BF63F07F0303F07F03837183799C
:1077E40014B943F0020301E023F0020383715454FB
:1077F40010BD00BF678600204378013B13F0800F63
:10780400DAB2837914BF63F07F0303F07F038371DB
:10781400837912B943F0020301E023F00203837178
:10782400427070478378013B13F0800FDAB283799A
:1078340014BF63F07F0303F07F038371837912B96C
:1078440043F0020301E023F0020383718270704766
:107854000B4B5A5C03785A40837912F0800F02D0A4
:1078640063F07F0305E003F07F0312B943F00203E2
:1078740003E08371837923F00203837102707047FC
:10788400678600200C4B10B55A5C013212F0800F51
:10789400D4B21A46837914BF63F07F0303F07F03E5
:1078A4008371837914B943F0020301E023F00203E6
:1078B4008371545410BD00BF6786002043780133A0
:1078C40013F0800FDAB2837914BF63F07F0303F0FF
:1078D4007F038371837912B943F0020301E023F03B
:1078E40002038371427070478378013313F0800F71
:1078F400DAB2837914BF63F07F0303F07F038371EB
:10790400837912B943F0020301E023F00203837187
:1079140082707047818070470A4B5A5C837912F0F9
:10792400800F02D063F07F0305E003F07F0312B9F8
:1079340043F0020303E08371837923F0020383712C
:1079440002707047678600200A4B5A5C837912F0F4
:10795400800F02D063F07F0305E003F07F0312B9C8
:1079640043F0020303E08371837923F002038371FC
:1079740042707047678600200A4B5A5C837912F084
:10798400800F02D063F07F0305E003F07F0312B998
:1079940043F0020303E08371837923F002038371CC
:1079A40082707047678600200E4B70B55A5C1C4687
:1079B400837912F0010F14BF43F0010323F0010394
:1079C400837153108279DEB202F07F0585711BB991
:1079D40045F00205857102E002F07D028271665471
:1079E40070BD00BF678600200278837912F0010F12
:1079F40014BF43F0010323F0010383715310827910
:107A040002F07F0110B58171DCB21BB941F00201B3
:107A1400817102E002F07D028271047010BD704732
:107A24000B4B5A5C03781A43837912F0800F02D00F
:107A340063F07F0305E003F07F0312B943F0020310
:107A440003E08371837923F002038371027070472A
:107A54006786002030B5124C8279635CD5074FEA03
:107A6400430348BF43F00103FF2BDDB28CBF42F058
:107A7400010222F0010213F0800F8271827914BF97
:107A840062F07F0202F07F028271827915B942F0BE
:107A9400020201E022F002028271635430BD00BF91
:107AA4006786002082790378D1074FEA430348BFF1
:107AB40043F00103FF2BD9B28CBF42F0010222F044
:107AC400010213F0800F8271827914BF62F07F0289
:107AD40002F07F028271827911B942F0020201E060
:107AE40022F002028271037070470000827910B59F
:107AF400114C12F0010F635C18BF43F4807313F050
:107B0400010F4FEA630314BF42F0010222F00102A5
:107B140013F0800F8271827914BF62F07F0202F049
:107B24007F028271827913B942F0020201E022F0ED
:107B340002028271635410BD678600208279037843
:107B4400D10748BF43F48073D9074FEA63034CBF9E
:107B540042F0010222F0010213F0800F8271827957
:107B640014BF62F07F0202F07F028271827913B93E
:107B740042F0020201E022F00202827103707047B7
:107B84008279234B30B55C5C02F00103017883F009
:107B940001030D1BEB1A1D064CBF62F07F0202F0BD
:107BA4007F0213F0FF0F827182790CBF42F0020250
:107BB40022F00202827181EA030212F0800F8279BC
:107BC40006D084EA01052D0602D542F0400201E008
:107BD40022F040028271827915070ED502F0010568
:107BE40001F00F0104F00F0485F00105491BA142C7
:107BF400B8BF063B992B02D9603BFF2B02D842F059
:107C0400010201E022F001028271037030BD00BF65
:107C140067860020837943F0010383717047837979
:107C240043F0080383717047837943F0040383713D
:107C3400704700000278014B5A5470476786002051
:107C44004278014B5A547047678600208278014B72
:107C54005A547047678600200278837912F0800FA7
:107C640002D063F07F0305E003F07F0312B943F011
:107C7400020303E08371837923F00203837142706A
:107C840070470278837912F0800F02D063F07F038B
:107C940005E003F07F0312B943F0020303E08371AC
:107CA400837923F00203837182707047C2788379E9
:107CB40012F0800F02D063F07F0305E003F07F032E
:107CC40012B943F0020303E08371837923F00203C2
:107CD4008371427070474278837912F0800F02D02A
:107CE40063F07F0305E003F07F0312B943F002035E
:107CF40003E08371837923F0020383710270704778
:107D04004378C37070478278837912F0800F02D071
:107D140063F07F0305E003F07F0312B943F002032D
:107D240003E08371837923F0020383710270704747
:107D34000378054A134483F8001103780BB9FF2331
:107D440000E0013B037070476786002081880131A1
:107D540038B589B2C51C04468180090A2846FFF754
:107D6400E7FF21792846FFF7E3FFA179284641F090
:107D74001001FFF7DDFFA379064A43F00403A37162
:107D84004FF6FF73D15C4FF6FE73D35C03EB012314
:107D9400A38038BD6786002070B50E468188C51C57
:107DA4000446013989B28180090A2846FFF7C0FFD9
:107DB40021792846FFF7BCFFA68070BD10F8031B8D
:107DC400FFF7B6BF8179033041F01001FFF7B0BF70
:107DD4000378054AFF2B0CBF00230133037003789B
:107DE400134493F80001704767860020014603306E
:107DF40008B5FFF7EDFF10F0800F08708B7902D003
:107E040063F07F0305E003F07F0310B943F002033E
:107E140003E08B718B7923F002038B7108BD01465B
:107E2400033008B5FFF7D4FF40F02000887108BD87
:107E340038B5C51C01462846FFF7CAFF8871284695
:107E4400FFF7C6FF04462846FFF7C2FF44EA0020B6
:107E5400888038BD38B5C51C04462846FFF7B8FFEE
:107E640001462846FFF7B4FF41EA00200130A08014
:107E740038BD0020704700002DE9F04F024600F5A0
:107E8400A055DFF8D0E30021F14F0023C2F808E049
:107E9400D160143242F8047C11601371AA42ED4C93
:107EA400F3D1ED4D0221ED4A4FF0030EC0F8EC572B
:107EB4004FF0050BEA4DEB4FEB4EDFF8C0C3DFF894
:107EC400C083DFF8C093C0F83C280422C0F89C5754
:107ED4000625C0F8DC78E54FC0F84498C0F88C68F3
:107EE400C0F8949880F89C28C0F8F497C0F8A49738
:107EF40080F8AC57C0F8E49880F8EC58C0F834998E
:107F040080F83C29C0F84038C0F8483880F84C184C
:107F1400C0F89038C0F89838C0F8F037C0F8F8378F
:107F240080F8FCE7C0F8A037C0F8A837C0F8E038FC
:107F3400C0F8E838C0F82CC9C0F83039C0F838396E
:107F4400C0F8CC89C0F8D039C0F8D499C0F87C798D
:107F5400C24FC0F88499C0F83C73BF4FDFF8289330
:107F6400C0F8EC72BE4F80F8DC29C0F89C72BD4F9B
:107F740080F88C29C0F8DC73BC4FC0F84493C0F877
:107F84008C63C0F8949380F89C23C0F8F492C0F8F2
:107F9400A49280F8AC52C0F8E493C0F8D839C0F881
:107FA4008039C0F88839C0F84033C0F8483380F8C5
:107FB4004C13C0F89033C0F89833C0F8F032C0F8CE
:107FC400F83280F8FCE2C0F8A032C0F8A832C0F859
:107FD400E033C0F8E83380F8ECB3DFF8B0A2C0F8BF
:107FE4002CC4C0F87C749C4FC0F83494C0F8D4946A
:107FF400C0F88494C0F88070DFF89492C0F8D8A0D8
:108004009B4FDFF890A280F83C2480F8DC2480F8B1
:108014008C24C0F82061C0F8289180F83051C0F851
:108024008890C0F8D0704FF00707C0F8C891C0F826
:108034003034C0F83834C0F8CC84C0F8D034C0F838
:10804400D834C0F88034C0F88834C0F82431C0F87B
:108054002C31C0F88430C0F88C3080F890B0C0F86F
:10806400D430C0F8DC3080F8E010C0F8C0C1C0F8EB
:10807400C431C0F8CC31C0F850ABDFF81CA2C0F852
:108084006892C0F8D0AD41F2C82ADFF8109280F8A7
:10809400D05180F87072C0F8489BC0F8C89DC0F8F1
:1080A4006082C0F86432C0F86C32C0F84C3BC0F84F
:1080B400543B80F8581BC0F8CC3DC0F8D43D80F840
:1080C400D81D40F80A9041F2CC2A6A4F40F80A3091
:1080D40041F2D02A40F80A7041F2D42A5E4F40F8A7
:1080E4000A3041F2D82A00F80A10DFF8B4A1C0F827
:1080F4007863C0F880A3C0F8E0A2DFF8A8A180F8F4
:108104008823C0F8D872C0F8C893C0F87C33C0F88C
:108114008433C0F8DC32C0F8E43280F8E8E2C0F816
:10812400CC33C0F8D0A341F2480AC0F8D43380F865
:10813400D81340F80A9041F24C0A4F4F40F80A30E5
:1081440041F2500A40F80A7041F2540A4FF007070E
:1081540040F80A3041F2580A00F80A10C0F8489171
:10816400C0F84896C0F8C898DFF83CA1DFF83C9105
:10817400C0F850A1C0F8D098DFF834A1DFF83491EA
:10818400C0F810A0C0F8F09141F2E809DFF828A186
:108194000776C0F850A6C0F84C31C0F8543180F8C6
:1081A40058118460C3604361C0F84C36C0F854363B
:1081B40080F85816C0F8CC38C0F8D43880F8D818ED
:1081C400C0F8E841C0F8EC31C0F8F43180F8F81197
:1081D40040F8094041F2EC09DFF8E0A040F809302A
:1081E40041F2F0091D4F40F809A041F2F40941F2AF
:1081F4000C0A40F8093041F2F80900F80910DFF8D8
:10820400C090C0F8BC7FC0F8F096DFF8B890C0F812
:10821400E846C0F8709EDFF8B090C0F8EC36C0F8BD
:10822400C49FC0F8F43680F8F816C0F8684EC0F859
:108234006C3EC0F8743E80F8781EC0F8C03FC0F8A9
:10824400C83F80F8CC1F40F80A6041F2100A3DE0B4
:1082540051200000391F0000291F0000FD1E0000EE
:10826400092000002D200000091F0000E51F000068
:10827400132A0000EF21000041220000911F00009A
:10828400C11F00005D200000192100009921000099
:108294004D210000DB210000E52100003D1F00000E
:1082A400F9210000352200004B2200006122000069
:1082B400ED2800006B220000572200007522000008
:1082C4007F2200008922000095220000F74F40F829
:1082D4000A3041F2140A40F80A9041F2180A40F8B0
:1082E4000A3041F21C0A00F80A2041F25C0AC0F884
:1082F4006C7FEF4FC0F8749FC0F81C7FED4FC0F83F
:10830400703FC0F8783F80F87CEFC0F8203FC0F899
:10831400249F80F82C5FC0F8283F40F80A7000F5CD
:10832400835AE54FCAF8003041F2640A40F80A90D3
:1083340041F2680A40F80A3041F26C0A00F80AE097
:1083440041F2AC0A40F80AC041F2B00A40F80A30DF
:1083540041F2B40A40F80A9041F2B80A40F80A30EF
:1083640041F2BC0A00F80A2041F24C1A40F80A8093
:1083740041F2501A40F80A3041F2541A40F80A9077
:1083840041F2581A40F80A3041F25C1A00F80A2007
:1083940041F2FC0A40F80A7000F5885AC74FCAF83F
:1083A400003041F2041A40F80A9041F2081941F2EF
:1083B400901A40F8093041F20C1900F8092041F2F2
:1083C400881940F8097041F28C19B84F40F8093007
:1083D400DFF8EC9240F80A9041F2941A40F80A301F
:1083E40041F2981A00F80A1041F2782A40F80A601B
:1083F40041F27C2A40F80A3000F5945ACAF80090F9
:1084040041F2842A40F80A3041F2882A00F80A200E
:1084140041F2D81A40F80A7041F2DC1AA74F40F82A
:108424000A3000F58F5ACAF8009041F2E41900F5B9
:10843400805A40F8093041F2E81900F809E0DFF801
:108444008492C0F8087FC0F8109FC0F8F86FC0F895
:108454000C3FC0F8143F80F8181FC0F8FC3FCAF85E
:10846400009041F2040A914F40F80A3041F2080AA0
:1084740000F80A2041F2280AC0F8609F00F58159EB
:10848400C0F8587FC0F85C3FC0F8643F80F868EFDC
:10849400C9F8006041F2240940F80930DFF8289255
:1084A40040F80A9041F22C0A40F80A3041F2300AAE
:1084B40000F80A5000F5865AC0F8807F4FF007078D
:1084C400C0F8889FC0F8843FC0F88C3F80F890BF04
:1084D400CAF800C041F2C40A40F80A3041F2C80A9E
:1084E40040F80A9041F2CC0A40F80A3041F2D00A2E
:1084F40000F80A5000F58B5ACAF8008041F2641A59
:1085040040F80A3041F2681A40F80A9041F26C19B6
:1085140041F2A82A40F8093041F2701900F80970B4
:10852400664FDFF8A891C0F8BC75604FC0F8D89FBB
:10853400C0F86C75DFF898915D4FC0F8B09AC0F838
:108544001C75DFF890915B4FC0F8C495C0F80C66B9
:10855400C0F8149680F81C26C0F87495C0F8D04F63
:10856400C0F8D43FC0F8DC3F80F8E01FC0F8A84A48
:10857400C0F8AC3AC0F8B43A80F8B81AC0F8C035BC
:10858400C0F8C83580F8CC15C0F81036C0F81836D5
:10859400C0F87035C0F8783580F87CE5C0F820352F
:1085A400C0F82495C0F85C76C0F86496C0F8B49618
:1085B400C0F85497C0F8049700F595593E4F80F8D9
:1085C4002C5580F8BC2680F85C27C0F8FC7680F82F
:1085D4000C27C0F82835C0F86036C0F8683680F833
:1085E4006CB6C0F8ACC6C0F8B036C0F8B836C0F83F
:1085F4004C87C0F85037C0F85837C0F80037C0F877
:108604000837C9F8006041F2A429284F40F809301E
:10861400DFF8C49040F80A9041F2AC2A40F80A30DE
:1086240041F2B02A00F80A5000F5905ACAF80070D6
:1086340041F2042A4FF0070740F80A3041F2082AB1
:1086440040F80A9041F20C2A40F80A3041F2102A0C
:1086540000F80AB000F59A5ACAF800C041F2443A48
:1086640040F80A3041F2483A40F80A9041F24C3A54
:1086740040F80A3041F2503A00F80A5000F59F5A87
:10868400CAF8008041F2E43A40F80A3041F2E83A8C
:1086940040F80A9041F2EC39DFF840A040F8093084
:1086A40041F2F03900F809701AE000BF291F0000F8
:1086B400092000002D200000E51F0000FD1E000021
:1086C400D92200001D23000061230000992300002B
:1086D400C5230000F1230000252400005D240000D0
:1086E40041F22829F14F40F8094041F22C2940F881
:1086F400093041F2302940F809A041F23429DFF869
:10870400C8A340F8093041F2382900F80910DFF80D
:10871400BC93C0F8F865C0F8B09FDFF8B493C0F814
:1087240078A8C0F80096C0F88098DFF8A893C0F83D
:108734008862C0F8A84FC0F8AC3FC0F8B43F80F8D6
:10874400B81FC0F8FC35C0F8043680F808E6C0F855
:108754007C38C0F8843880F888B8C0F88C32C0F807
:108764009092C0F83C7DD24FDFF86C93C0F8EC7C5B
:10877400D04F80F89852C0F89C7CCF4FC0F8449DED
:10878400C0F8DC7DCD4FC0F88C6DC0F8949D80F8A6
:108794009C2DC0F8F49CC0F8A49C80F8AC5CC0F894
:1087A400E49DC0F8349E80F83C2EC0F89432C0F8A2
:1087B400403DC0F8483D80F84C1DC0F8903DC0F8DD
:1087C400983DC0F8F03CC0F8F83C80F8FCECC0F8E8
:1087D400A03CC0F8A83CC0F8E03DC0F8E83D80F8F3
:1087E400ECBDC0F82CCEC0F8303EC0F8383EC0F81E
:1087F400CC8EC0F87C7EAD4FC0F8D49EC0F8B07C5F
:10880400AB4FC0F8849EC0F8007DAC4FDFF8CC922B
:10881400C0F8E07EAA4F80F8DC2EC0F8407EA34F5B
:1088240080F88C2EC0F8B89CC0F8A06DC0F8A89D44
:1088340080F8B02DC0F8089DC0F8E89E80F8F02EAE
:10884400C0F8489EC0F8D03EDFF89492C0F8D83EF5
:10885400C0F8803EC0F8883EC0F8B43CC0F8BC3CC8
:1088640080F8C01CC0F8A43DC0F8AC3DC0F8043D7D
:10887400C0F80C3D80F810EDC0F8E43EC0F8EC3EC2
:10888400C0F8443EC0F84C3EC0F8887C884FC0F81D
:10889400909CC0F8809DC0F8D87CC0F8E09CC0F8DB
:1088A400209EC0F8C09EC0F88075DFF83892854FCE
:1088B40080F8502EC0F8786D80F8882D80F8282E26
:1088C40080F8C82EC0F82066C0F8289680F8305684
:1088D400C0F88C3CC0F8943C80F8981CC0F87C3DEF
:1088E400C0F8843DC0F8DC3CC0F8E43C80F8E8EC17
:1088F400C0F818CEC0F81C3EC0F8243EC0F8B88EAC
:10890400C0F8BC3EC0F8C43EC0F82436C0F82C36CB
:10891400DFF8D4A1C0F88435C0F88895C0F8D075C4
:108924004FF00707C0F8C896C0F8689741F250297D
:10893400C0F8D8A580F8D05680F87077C0F88C3588
:1089440080F890B5C0F8D435C0F8DC3580F8E0156F
:10895400C0F8C0C6C0F8C436C0F8CC36C0F86087CA
:10896400C0F86437C0F86C3740F8094041F2542924
:10897400DFF878A140F8093041F258294B4F40F80C
:1089840009A041F25C29DFF868A140F8093000F53C
:10899400935989F80010DFF85C91C0F8BC70444F1B
:1089A400C0F8C490C0F80C61C0F81491C0F8C0308D
:1089B400C0F8C83080F8CC10C0F81031C0F81831B5
:1089C40080F81C21C7663B4FC0F87490C7613A4FCA
:1089D400C0F82490C0F85C71C0F86491C0F8B491F8
:1089E400C0F85492C0F80492344FDFF80C9180F828
:1089F4002C5080F8BC2180F85C22C0F8FC7180F80F
:108A04000C220367836780F87CE003628362C0F80A
:108A14006031C0F8683180F86CB1C0F8ACC1C0F8FE
:108A2400B031C0F8B831C0F84C82C0F85032C0F848
:108A34005832C0F80032C0F80832C0F8A845C0F86F
:108A4400AC35C0F8B095DFF8B490194FC0F8B090C9
:108A5400DFF8AC90C0F80073C0F83098194FDFF815
:108A6400A490C0F850734FF00707C0F83093DFF8B4
:108A7400989080F8382880F83823C0F8A063C0F8AC
:108A8400A89380F8B053C0F80893C0F858A3C0F86E
:108A9400B43580F8B8E5C0F8A840C0F8AC30C0F8E8
:108AA400B43080F8B8E0C0F828482FE0FD1E00007C
:108AB400291F0000092000002D200000E51F0000F0
:108AC400A91F0000132A00005D1F00008924000074
:108AD400B524000039290000B9240000E92400006D
:108AE400192500004925000089250000BF25000044
:108AF40045260000C12500005D290000652900000D
:108B04008D290000BF290000F5250000C0F82C388D
:108B1400C0F83438C0F82843C0F82C33C0F83433D4
:108B2400C0F8A433C0F8AC33C0F80433C0F80C3335
:108B340080F810B3C0F85433C0F85C3380F8601385
:108B4400C0F840C4C0F84894C0F8E89480F8F074C1
:108B5400DFF80C94F34FC0F8A898C0F80078C0F878
:108B64000898C0F84899C0F8E899EF4FDFF8F4A3E3
:108B7400DFF8F49380F85054C0F8A06880F8B05837
:108B8400C0F850784FF00707C0F858A841F2442ABB
:108B940080F85059C0F84434C0F84C34C0F8E0842C
:108BA400C0F8E434C0F8EC34C0F8A438C0F8AC38E9
:108BB400C0F80438C0F80C3880F810B8C0F854383D
:108BC400C0F85C3880F86018C0F840C9C0F844396F
:108BD400C0F84C39C0F8E089C0F8E439C0F8EC3981
:108BE400C0F81095DFF8849380F8F079C0F8909776
:108BF40041F23C29CD4F80F8185580F89857C0F8B9
:108C04000845C0F80C35C0F81435C0F88847C0F8DA
:108C14008C37C0F8943740F8097000F59259C14F69
:108C2400C9F80030DFF8489340F80A9041F2482A26
:108C340040F80A3041F24C2A00F80A1041F28C2A1A
:108C440040F80A6041F2902A40F80A3041F2942A2E
:108C540040F80A9041F2982A40F80A3041F29C2ADE
:108C640000F80A2041F2EC1A40F80A7041F2F01AB6
:108C7400AF4F40F80A3041F2F41A40F80A9041F23A
:108C8400F81A40F80A3041F2FC1A00F80AE041F2FE
:108C94009C1A40F80A7000F58D5AA64FCAF80030A5
:108CA40041F2A41A40F80A9041F2A81A40F80A3096
:108CB40041F2AC1A00F80A5041F2DC2A40F80A707A
:108CC40000F5975A9C4FCAF8003041F2E42A40F864
:108CD4000A9041F2E82A40F80A3041F2EC2A00F8FE
:108CE4000AB041F22C3A40F80AC041F2303A40F856
:108CF4000A3041F2343A40F80A9041F2383A40F8E6
:108D04000A3041F23C3A00F80A2041F2CC3A40F8E9
:108D14000A8041F2D03A40F80A3041F2D43A40F89D
:108D24000A9041F2D83A40F80A3041F2DC3A00F8AD
:108D34000A2041F27C3A40F80A7000F59C5A794FB7
:108D4400CAF8003041F2843A40F80A9041F2883976
:108D5400DFF820A240F8093041F28C3900F80920EC
:108D6400DFF81492C0F86844C0F8709441F268398E
:108D7400C0F86C34C0F8743480F8781440F80940B2
:108D840041F26C3940F8093041F2703940F809A0D9
:108D940041F2743940F8093041F2783900F8091089
:108DA400DFF8D891C0F86849C0F87099C0F86C39F8
:108DB400C0F8743980F87819C0F86C7A5C4F80F880
:108DC4002C5AC0F81C7A80F86C5B5A4F5A4DDFF865
:108DD400B091C0F85C7BC0F8FC5B524F574DC0F8B3
:108DE4000C6B80F81C2B80F8BC2BC0F8103BC0F82F
:108DF400149BC0F8183BC0F8703AC0F8749AC0F8D5
:108E0400783A80F87CEAC0F8203AC0F8249AC0F88E
:108E1400283AC0F8603BC0F8649BC0F8683BC0F8CF
:108E2400ACCBC0F8B03BC0F8B49BC0F8B83BC0F8BA
:108E34004C8CC0F8503CC0F8549CC0F8583C80F8A6
:108E44005CBCC0F8003CC0F8049CC0F8206BC0F8BF
:108E5400285B80F8302BC0F8807AC0F8885AC0F8B4
:108E6400C85B80F8D02B364DC0F8F86A80F8082B20
:108E740080F8A82B334F2B4E334AC0F8083C80F8B7
:108E84000CBCC0F8243BC0F82C3BC0F8843AC0F8B2
:108E94008C3A80F890EAC0F8C07BC0F8C43BC0F8B4
:108EA400CC3BC0F8FC3AC0F8005BC0F8043BC0F807
:108EB400586AC0F85C3AC0F8605AC0F8643A80F85E
:108EC40068EAC0F898CBC0F89C3BC0F8A05BC0F837
:108ED400A43BC0F8504DC0F8582D1C4AC0F8543D6E
:108EE400C0F8302D1A4AC0F85C3DC0F8982E194AD3
:108EF40080F8601DC0F8D82A174AC0F8284DC0F879
:108F0400182C164AC0F82C3DC0F8343D80F8381DA2
:108F1400C0F8904EC0F8943EC0F89C3E80F8A01E65
:108F240030E000BF291F0000132A0000FD1E0000CE
:108F3400092000002D200000E51F0000E1270000AB
:108F4400ED270000A91F0000F927000023280000D6
:108F54004D28000077280000A1280000A728000061
:108F64008D260000DD260000D1290000F52900002F
:108F740021270000BF270000B5270000C9270000F3
:108F8400D5270000C0F8D04AC0F8D43AC0F8DC3A7B
:108F940080F8E01AC0F8104CC0F8143CC0F81C3C2F
:108FA40080F8201CC0F8E84BC0F8EC3BC0F8F02B6C
:108FB400C0F8F43B80F8F81BBDE8F08F00230C499F
:108FC4004FF6FD7203708370437010B58C5C4FF6DE
:108FD400FC728A5C02EB04228280FD22C2708279D8
:108FE40042F02002827141F20842835410BD00BF56
:108FF4006786002038B5837904465A0720D423F0C5
:109004001003C51C818883712846090AFEF790FE67
:1090140021792846FEF78CFEA1792846FEF788FEC2
:10902400A379084A012043F00403A3714FF6FF73A8
:10903400D15C4FF6FE73D35C03EB0123A38038BDF0
:10904400002038BD6786002084B070B5064605A8A8
:1090540080E80E0006A80B4631C810F0010F4FEA55
:10906400600018BF3258304418BF5358984715F061
:10907400010F01464FEA65000CBF234633583044C4
:1090840018BF1B59BDE8704004B018472DE9F04FD4
:1090940000F5A05889B006460F4691464FF0000AE5
:1090A4004FF0000B08F10808002F2CDD98F8003071
:1090B4004BBBB38803AD5A1CB280154A12F803E0C7
:1090C400142303FB0EFE06EB0E04B64408340FCC47
:1090D4000FC523689EF818402B6008AB8DF81C4020
:1090E40013E9030003AB8DE8030030460ECBFFF712
:1090F400ABFF1AEB040A4BF1000BB9F1010F18BFD7
:1091040001243F1BD0E75046594609B0BDE8F08F13
:1091140067860020034B1A780AB1002200E001227E
:109124001A707047A13A002010B504460BF0D6FC23
:10913400204610BD084B1B78DBB207B500228DF822
:109144000730064B1A60064B1B7813B9054800F02C
:1091540093FE03B05DF804FBA13A0020BC79002023
:10916400668600205E860020034B01461B7813B9F7
:10917400024800F0ABBE7047668600205E86002081
:1091840008B50021034800F087FBBDE80840FDF75F
:10919400A7BF00BF5E86002038B5FDF7DBFE08B32D
:1091A400FDF79EFCFDF78EFD0446FDF7E3FE054644
:1091B400812C15D100200024FDF7D2FE0F4B1C702A
:1091C400FEF70EF800F040F9284600F0BBF92146FE
:1091D4000B4800F059FE0B4A0B490C480BF022FCDB
:1091E400142006E0FDF77CFC00F00CF900F042FAD4
:1091F4000A20BDE838400AF04BBA00BF668600205A
:109204005E860020FF520700B53C0000FC390020B8
:1092140008B50A2108480BF0F1F908480BF09CFC4A
:109224000748084A4FF480710DF05AF80648BDE823
:109234000840FCF743BA00BFC53500207039002050
:109244005E860020210000004886002008B5082121
:10925400064800F01BFB064A064907480CF0CBF809
:109264000AF0E8F9054B186008BD00BF5E860020CF
:1092740014390020C93C0000FC390020C0790020CA
:1092840070B5D1F1FF040A4D4FF00C0608BF7F24DE
:1092940011F0800106FB005017BF6B6B4160C3EBFC
:1092A400034303FA02F21CBF92FBF4F3436070BD64
:1092B400847900204FF0020C043091FBFCF32DE97B
:1092C400F04F89B002934B4B1A681E6906925A6894
:1092D400DD690092DA689C6A05929A69069904929B
:1092E4005A6A0392DA6A93F830300793009B03EBCF
:1092F400010C059B002106EB0309049B8A4605EB40
:109304000308039B04EB030E0B46029FBA4554DA91
:10931400744506DD9310012183EAE2139BB243EA0C
:1093240002424FEA2E730AF1010AA6440430C3F143
:10933400170BC3F1120742FA0BFB42FA07F78BEA49
:10934400070B01279F4002FA03F3013F0BEA0707CB
:109354003B43294FC3F3072B0193C3F3074317F888
:109364000BB0264FFF5C9DF804304BEA070B244FEB
:10937400FB5C4FEA9C074BEA030B4FEA990307F0A7
:109384000057B14403F000531F444FEA9803A84424
:1093940003F000533B44BDF81C7003EB8B531B15C7
:1093A400A3F5006313FB07F31BB220F8083C20F875
:1093B400063C009B9C440123A7E70298039F20EAF4
:1093C400E07004FB0074049F05FB0075059F06FB19
:1093D4000076009FBE46069F0EFB007023B1054B2E
:1093E4001860DE609D615C6209B1024BDA6209B00B
:1093F400BDE8F08F84790020EF830020EF84002003
:10940400EF82002008B5FDF797F9034B1860FDF7CC
:1094140073FB024B186008BD686500206C65002072
:10942400A1F1C0031F2B044B96BF01F01F0101F0F3
:109434007F017F3119607047D07900200022014BF1
:109444001A607047D079002038B53248FFF7B6FD6E
:109454003148FCF783FA2F493048FCF751F92F487B
:10946400FCF758F900232E491846585401332C4A66
:10947400B3F5803FF9D100232A4C03F50041185D70
:1094840001335054B3F5805FF7D10023264C03F524
:109494004041185D01335054B3F5005FF7D1002308
:1094A400224C03F56041185D01335054B3F5005F5D
:1094B400F7D11F4B42F674521E4D5A631E4A1F4C7D
:1094C400DA6200231E485A1102F00401DA1002F095
:1094D40002020A43C3F380010A435A555A1002F0A8
:1094E400100103F008020A4359001A559A0021F0AA
:1094F4007F0102F0400211435A0102F020020A43A4
:109504001A540133B3F5807FDDD1BDE83840FFF74D
:109514007FBE00BF70650020F4790020DC79002054
:1095240067860020801F0060802F0060DA1300200F
:1095340084790020EF820020F8FF7F00EF83002071
:10954400EF8400202DE9F34104464548FDF7C8F8AF
:109554002046FDF795FD434980462046FDF70EFD64
:10956400074620460CF0FBF80023411E98420ADD12
:10957400E25C2E2A03F1010203D18B4201D0144490
:1095840001E01346F2E72378374C03F0DF02502A58
:1095940011D13A46022101A8FDF73CFD9DF80430A3
:1095A4009DF805503A46A8F1020143EA0525AB1E91
:1095B40043449EB21CE0362B10D007D8322B0AD07D
:1095C400342B0CBF4FF4804500250CE0412B08D010
:1095D400612B06D007E04FF4005504E04FF4C0457A
:1095E40001E04FF4204505EB08033A4641469EB29C
:1095F4006019FDF70FFD3846FDF726FDFF21EBB29C
:10960400C5F30725F2B2194884F82B3084F82D30BD
:10961400330A84F82F2084F8303084F8323084F808
:10962400343084F8AF3084F8312084F8332084F85F
:10963400371084F8381084F8AE2084F82C5084F85D
:109644002E50FFF7BBFC012244F620610748FFF7C8
:109654001DFD0748FDF744F802B0BDE8F08100BFE6
:10966400D0350020DD35002067860020706500209D
:10967400E135002038B5012254481146FFF706FDB4
:1096840001215348FCF786FA5248FCF73FF9514848
:10969400FCF73CF94E48FCF77AFA0028EBD04C482A
:1096A400FCF775FA10B14A48FCF76EFAFFF742FD71
:1096B400494B1C6814B9494B1C685CB1484B45487C
:1096C40053F8244014F4803118BF0121FCF71CF82E
:1096D400A1B204E021463F48FCF716F821463D4874
:1096E400FCF710F83F4B404D1C6814F0600F46D156
:1096F400296804F0100211F0100102D132B10122E4
:1097040001E01AB911463348FCF700F82B6804F05D
:10971400040213F0040F03D13AB10122114601E00F
:109724001AB901212B48FBF7F1FF2B6804F008025A
:1097340013F0080F02D132B1012200E01AB902215C
:109744002448FBF7E3FF2B6804F0010213F0010F38
:1097540002D132B1012200E01AB903211D48FBF7FE
:10976400D5FF2B6804F0020213F0020F02D132B1CC
:10977400012200E01AB904211648FBF7C7FF0022B2
:1097840049F20A032C60194C1046E15CFFF778FD9E
:10979400012249F20B031046E15CFFF771FD02223E
:1097A40049F20C031046E15CFFF76AFD49F20D0330
:1097B40000220320E15CFFF763FD49F20E030C4A2B
:1097C400E35C03F00F0382F8303038BD706500208D
:1097D400F4790020DC790020D07900206C65002029
:1097E40080020020686500207C79002067860020C4
:1097F4008479002038B50C4C0C48FEF73DFB0C4D29
:109804002046FCF795F820460A4C2A460A490BF0F4
:10981400F2FD2046FBF75EFF2A4620460749BDE8D5
:1098240038400BF0E8BD00BFF479002070650020DB
:1098340014390020DC790020F104000095020000B6
:1098440010B504460BF066F8204610BD00F07F000A
:109854000D4B40F41220C3F8A000C3F8B010C3F8B5
:10986400C020D3F8A02022F48052C3F8A020D3F85B
:10987400A010054A0029FADAD2F8A03023F4803384
:10988400C2F8A030704700BF00800D40014B197032
:10989400704700BF8A3A00202DE9F0410023544D5F
:1098A4000F4642F2107242F2486114202B60A8461F
:1098B400FFF7CCFF4F4E504D072F00F2BF80DFE87B
:1098C40007F0041585A75B6F2C4116224B4B1A60D9
:1098D4004FF4A0724A4B1A60F0224A4B1A604FF4BC
:1098E400B073494A33601360012210E01622434BDF
:1098F4001A604FF4A072424B1A604FF4F072414B5D
:109904001A604FF4B073404A3360136000223F4B37
:1099140014241A6082232B6090E02C22374B1A60A7
:109924004FF42072364B1A60F022364B1A604FF413
:109934003073354A336013600123344A13600422C0
:109944002A6015E02C222D4B1A604FF420722C4B08
:109954001A604FF4F0722B4B1A604FF430732A4A9A
:10996400336013600022294B1A6004232B60012307
:10997400C8F800300A2461E02122204B1A604FF419
:1099840000721F4B1A60F0221E4B1A604FF40C73C6
:109994001D4A3360136001221C4B1A60002312E03D
:1099A4002122164B1A604FF40072154B1A604FF4C3
:1099B400F072144B1A604FF40C73134A3360136043
:1099C4000023124A13602B600F2437E019220B4B3B
:1099D4001A604FF4B0720A4B1A60F022094B1A60F5
:1099E4004FF4C273084A33601360012221E000BFC0
:1099F4004465002004650020287A0020EC640020DF
:109A0400107A0020147A0020187A0020F0640020D4
:109A14001922A74B1A604FF4B072A64B1A604FF488
:109A2400F072A54B1A604FF4C273A44A33601360FA
:109A34000022A34B13241A6082232B601427A14B0A
:109A440042F24862A0491F60A04BA1481A6042F24A
:109A54001072A04B1A602A689F4B1A60FCF750FBE7
:109A64009E499B48FCF756FB9D499948FCF748FBE7
:109A7400022197489FED8C0B0BF0D6F894480BF01D
:109A84006BF8984B0121187809F04AFE01210F2048
:109A940009F046FE0121022009F042FE01210320C3
:109AA40009F03EFE0121042009F03AFE01212120A3
:109AB40009F036FE01210A2009F032FE01210C20B2
:109AC40009F02EFE01210B2009F02AFE01210D20B0
:109AD40009F026FE844BFF228448996A0A60996B38
:109AE4000A60996C0A60D3F818120A60D3F8A810B7
:109AF4000A60D3F8C8100A60D3F8B8100A60D3F823
:109B0400D8100A607A4AD16F21F00C01D167116B29
:109B140021F4FF4141F480711163516F21F003017D
:109B24005167116A21F4C01141F480111162916AE4
:109B340021F00E219162596A0F60596B0F60596CC4
:109B44000F60D3F814120F60D3F8A4100F60D3F889
:109B5400C4100F60D3F8B410D3F8D4300F600521CB
:109B64001F60D36F43F00C03D367536F43F00303B9
:109B7400536702F534225F4B996091605E49C2F8E5
:109B84000001C2F8801001F58061C3F80001C3F838
:109B94008010D8F8001061B1584FC2F80401C2F81F
:109BA40084700822C3F80401C3F884704FF0A063E2
:109BB40002E04FF080730422520243F4400364082D
:109BC4004F4FA2F580724F48013C43F00103C7F8A0
:109BD400800014434C4A3B60C7F80041C2F880003F
:109BE4001360C2F8004102F57052424B106B31B160
:109BF40040F0020010631A6B42F0020205E040F0EC
:109C0400010010631A6B42F00102404C4FF0000E49
:109C14001A633F4823793F4A83769B00177903F1FF
:109C24008043DFF8F8C087764FF0004003F56C23DB
:109C3400394FC3F800E01860013013799B0003F139
:109C4400804303F56C23C3F800E018600420002966
:109C540066D01368082532689D6056429880A3F840
:109C640014E0DE60C3F818E092FBF5F292B2DA83F6
:109C7400DA82C3F810C040F2032C998BA3F806C013
:109C840089B2294399832368DA83DA821F619A8B24
:109C94009D6092B29880DE60A3F814E02A43C3F872
:109CA40018E0A3F806C07BE05A367910340024404B
:109CB400EC640020107A0020147A0020187A002026
:109CC400F064002038650020ED350020F8640020A1
:109CD400703900203C6500202C65002070D70300FB
:109CE400F73500208A3A00203C09002000010400D6
:109CF40000C00F4000C01A40020083000200800030
:109D040000041B400022000100C41A40707A0020A5
:109D140000800E40787A002080C61A4000021B4062
:109D2400D2F800E03268CEF808005642AEF80400DB
:109D3400AEF81410CEF80C60CEF8181092FBF0F2C6
:109D440092B2AEF81E20AEF81620CEF810C040F243
:109D5400022CBEF81C30AEF806C09BB243F00803D8
:109D6400AEF81C302B6813F0800F236898600AD07B
:109D7400DA830120DA8202229880DE601F619982F0
:109D84009961DA8008E0DA839880DA82DE601F6104
:109D940099829961A3F806C09A8B92B242F00802A4
:109DA4009A832B4AD2F8803043F04043C2F8803083
:109DB4002022284BA3F86C200322A3F86E20002253
:109DC400A3F86A20A3F8662041F24462A3F8602055
:109DD400A3F870204FF44272A3F86220A3F8722013
:109DE4008522A3F8742043F22402A3F86C200122F4
:109DF40003F5A033C3F80821174A184BC3F85C22B3
:109E0400174B8022174C1A60236843B9164B186805
:109E1400164B1B68584304300BF038FB2060246851
:109E24008CB1114B002120461A68104B1B685A4311
:109E3400043209F0DDFB0E4B18680E4B2044186009
:109E44000020BDE8F0814FF0FF30BDE8F08100BF95
:109E540000C00F4000401E4085000000003C002070
:109E640010E100E020420020187A0020147A00203B
:109E7400EC640020E8640020024A1368002BFCD044
:109E8400704700BFC47900200C4B0020F0B51E6859
:109E94000B4B1F680B4B1D680B4B1B685A42B0429F
:109EA4000BDA1C4604EB020E774502DD04F8011BB5
:109EB400F8E701302B44521BF1E7F0BD147A00207F
:109EC400107A0020187A0020E8640020034B1868F8
:109ED400034B1B6800FB0130704700BF187A002059
:109EE400E86400200E48006800FB02120D4909686E
:109EF4000A44F0B55142BDF914609DF8187000246D
:109F0400B4420BDA154605EB010E734502DD05F884
:109F1400017BF8E701340244091AF1E7F0BD00BF00
:109F2400187A0020E86400202DE9F74F9DF8385096
:109F34009DF830000195584D9DF83440D5F800E067
:109F4400564DD5F800C013F8015B002D00F0A08039
:109F5400534E174606EBC50505F108060096019E0B
:109F6400002E46D02E7807FB0C18013716F0010F8F
:109F74000EEB080A0CBFA346834616F0020F0AF143
:109F840001090EF808B00AF102080CBFA346834683
:109F940016F0040F0AF1030A0AF802BC0CBFA34628
:109FA400834616F0080F89F801B009F103090CBFC4
:109FB400A346834616F0100F88F801B008F1030891
:109FC4000CBFA346834616F0200F8AF801B00CBFDD
:109FD400A246824616F0400F89F801A00CBFA146A4
:109FE4008146F60988F801900CBF2646064688F893
:109FF400026015F8016B0CFB0718013716F0010F0E
:10A004000EEB080A0CBFA346834616F0020F0AF1B2
:10A0140001090EF808B00AF102080CBFA3468346F2
:10A0240016F0040F0AF1030A0AF802BC0CBFA34697
:10A03400834616F0080F89F801B009F103090CBF33
:10A04400A346834616F0100F88F801B008F1030800
:10A054000CBFA346834616F0200F8AF801B00CBF4C
:10A06400A246824616F0400F89F801A00CBFA14613
:10A074008146F60988F801900CBF2646064688F802
:10A084000260009EB5427FF46AAF083109B25AE714
:10A0940003B0BDE8F08F00BFE8640020187A002008
:10A0A400804F006070B50C4C00210C4E20460C4DC6
:10A0B4000AF0E2FB20460B4C324629460BF09BF992
:10A0C400204600210AF0D8FB324629462046BDE846
:10A0D40070400BF090B900BF707A00201439002052
:10A0E400E1430000787A00207047002070470000A8
:10A0F4000023064A436013680BB9106070475A681E
:10A104000AB11346FBE75860704700BF6C7A002021
:10A114000020704700207047704730B5039C01252C
:10A124001B024560002C9DF8105043F0800318BFBB
:10A134004FF0004443EA0242002D44EA020414BFF3
:10A144004FF4004500252C438460C16021F47F61F5
:10A1540021F00F0101F58053036101F500534361C0
:10A1640001F5405301F580418361C16130BD0000B8
:10A17400436A026A0BB11A6201E004490A600AB137
:10A1840053627047024A1360704700BF5C65002049
:10A1940058650020436A026A0BB11A6201E004495F
:10A1A4000A600AB153627047024A1360704700BFE5
:10A1B4006465002060650020F8B54FF480314D4B94
:10A1C40040244FF480554FF400564FF4404743F277
:10A1D400420E1A6A900704D59F625962C3F828E0B8
:10A1E400F7E7900401D45E62F3E7D00401D45D6222
:10A1F400EFE7002AEDDA12F4803001D09962E8E743
:10A20400520601D45C62E4E73B4A3C4CD2F880300D
:10A2140043F00303C2F880304FF04042384B9A6356
:10A224004FF440425A630522186003F58F130A2045
:10A23400C3F8B4200822C3F8A422324B5A6842F06F
:10A2440080625A604FF08062C3F8842009F020FADB
:10A25400D4F8403143F00203C4F84031D4F840311B
:10A2640013F00205FAD102F0A7FC2B46264A01217D
:10A2740042F823100133202BFAD14FF480720021CD
:10A28400224809F0B5F90023214A13700122C4F8C9
:10A2940090200322C4F8A8211B4AC4F84831C4F80A
:10A2A4005421C4F84C31C4F858311A4B1A4AC4F832
:10A2B4004031D4F8843143F48053C4F88431D4F861
:10A2C4005831D4F85431154BC3F80022144B4FF4D1
:10A2D40080321A60134BC4F84831D4F8483143F043
:10A2E4001203C4F84831D4F8483143F44023C4F885
:10A2F4004831F8BD00800D4000C00F4000022E40E0
:10A3040000A00D4000800042004000209D7B002002
:10A31400477B0020158B01007D520000003C00208B
:10A324000CE100E004000003C36870B504460D4668
:10A33400002B4AD0632948D909F07CF9234BA0604B
:10A344001A68234E5AB96561013D1C604FF04043C1
:10A35400A261E261C6F88850C6F88C3070BDD6F8A8
:10A364008C1021F07F418D4218D272B600204FF03C
:10A374000072491BC6F88C00C6F844211A6865614E
:10A38400013D1C604FF04043A261E0615161D46122
:10A39400C6F88850C6F88C3062B670BD6D1A9369E1
:10A3A4007BB15A69954209D2521B5A61DA69A36199
:10A3B400E2616561DC61E3699C6170BDAD1A1A46B6
:10A3C400EDE76561A361E261946170BDFC64002006
:10A3D40000022E4070B50A4606460369996849068C
:10A3E40001D41B68FAE74021956803F134049160B5
:10A3F4001168196051685960D168D960116919618F
:10A404005169596191699961D1699E62D961D16A31
:10A41400D962116B196302F1340103C984E80300A2
:10A42400D16BD96319460868012801D00968FAE795
:10A434000A601946106000200C68A24205D00C681E
:10A44400486208460C622146F6E7002248620A6226
:10A4540096F8342012F0FD0F05D1094A10685862AD
:10A4640040B9084804E0084A1068586210B907481F
:10A47400036000E00362116001209D6070BD00BFB5
:10A48400586500205C65002060650020646500203C
:10A494002DE9F04F85B082460D4693460393CB8851
:10A4A400B3F5804F57D802F03BFB0646002852D044
:10A4B40002F036FB044608B9304608E0EB88CBB11D
:10A4C40002F02EFB30B9304602F032FB204602F097
:10A4D4002FFB40E095F9007001210023EA888DE804
:10A4E4000A00FB0FFF435946FFF717FE3060FF0FCA
:10A4F400046001E0012730604FF000094FF00108CB
:10A5040029463046CDF804900223CDF80090082265
:10A51400FFF703FE3B4649462046CDF804804A46F1
:10A52400CDF80080FFF7F9FDDAF80030C4F82CB05C
:10A534003146A362EB8823632B6863636B68C4F8BA
:10A544000080A363039BDAF80000E36305B0BDE871
:10A55400F04FFFF73FBF002005B0BDE8F08F2DE9B5
:10A56400F74F8146884617469A4602F0D9FA0646BE
:10A57400002840D07D1E0446AD0B75B102F0D0FA20
:10A5840038B93046356802F0D3FAA64233D02E46A5
:10A59400F7E72060013D0446EFE70123C4F8289063
:10A5A400C4F82C80236027636563A563C4F83CA0CA
:10A5B4003446B7F5804F99F835304146204693BF6D
:10A5C400BA464FF4804A4FF0000B4FF0010B52464D
:10A5D4008DE82008FFF7A1FDBBF1000F04D1D044A2
:10A5E400CAEB07072468E4E73146484603B0BDE8F0
:10A5F400F04FFFF7EFBE002003B0BDE8F08F826894
:10A60400110608B507D48268120406D5836ADB6B89
:10A614001BB1984701E0002008BD012008BD0000DF
:10A624002DE9F8432C4B4FF000081C68002C50D047
:10A634002046FFF7E4FF256A002844D020462E4632
:10A64400FFF796FDA36858063AD5A76A20462C461C
:10A65400002502F06DFA9EB1B36AD6F820909F42AD
:10A6640001D04E46F7E73046FFF782FD0DB12E626A
:10A6740000E03546C6F82080A64208BF4C46F0E705
:10A684003B6923F01F033BB19A6851061DD53B611A
:10A69400C7F80C80C7F81880002DC7D0AB681A041F
:10A6A40008D5FA6B32B143F040032846AB60AB6A7D
:10A6B400DB6B98472E6A284602F03AFA3546EBE7F8
:10A6C400204602F035FA2C46B0E79A681A681B68EF
:10A6D400D7E7BDE8F88300BF5C6500202DE9F041B1
:10A6E400524CD4F844516E03C4F844510FD5504B26
:10A6F4001E6866B13046FFF782FF376A28B13046DC
:10A70400FFF736FD304602F013FA3E46F1E7280320
:10A714000FD5484B1E6866B13046FFF770FF376AA5
:10A7240028B13046FFF736FD304602F001FA3E46C6
:10A73400F1E7A90701D5FFF773FF6A073ED5D4F8FF
:10A7440084613A4A46F02A03C4F88431B3071DD51C
:10A7540016F00108384B0ED01978012916D80121BA
:10A7640025F080751970354BC2F880304FF04043A6
:10A77400C2F884300AE083F800800222304B314F63
:10A784009A63386800F070FDC7F80080370715D465
:10A79400294A1378022B11D170070FD503211170A8
:10A7A40042F21072C4F880204FF04042C4F8842072
:10A7B400D4F88421910501D5214A5363EA011AD5BD
:10A7C4001D4B1A78012A08D102221A70D4F8843158
:10A7D40043F48073C4F884310DE0032A0BD10422BE
:10A7E4001A700022D4F884011146C0F3816000F08D
:10A7F400FFFA144B1860AB0115D5134A116891B1D7
:10A804008B6913604BB10022DA615B69013BC4F8C8
:10A8140088304FF04043C4F88C30C8680368BDE802
:10A82400F0419B681847BDE8F08100BF00022E404C
:10A834005C65002064650020477B0020A086010041
:10A8440000A00D40087A0020FC640020844B002AFC
:10A8540008BF01225943036B2DE9F04F1B7D85B0DE
:10A86400090C022B4FF0010360D10F2A01F15701AB
:10A874004FF0FF35DFF8ECC128BF0F224909013A38
:10A8840003FA02F2B2F5807FA8BF4FF48072D408B5
:10A8940018BFA3B20024A0F840302B462746002658
:10A8A40017F80CE017448E44764538BF7646FF2FE0
:10A8B400DFF8B0E1F4D9B54288BF234604F10104BE
:10A8C40088BF3546A242E9D1BB2D01D90020C4E09E
:10A8D400C9B21C46A0F84420A0F8463080F84A10BB
:10A8E400FF2C06D81EF804500D440EF804501444EE
:10A8F400F6E7012A01D1FF220EE0022A03D103F078
:10A904000101552207E0042A99BF03F00301112233
:10A9140003F0070101228A40DB0880F83620A0F802
:10A924004230002380F83730012096E0052443EAC2
:10A934005305AA4204D9013C4FEA4303F7D120232B
:10A944009AB20392BDF80C20A0F8402090F835206C
:10A9540022B984314A090221029203E066310222BB
:10A96400490902924FF0FF324FF0000C1546E646BB
:10A974000192E0463B4A4FF0000B02EBC806144636
:10A98400029A96F800A096F802909244F7788944C7
:10A9940032790F44CA450A4405D9BA4509D9524502
:10A9A40038BF524608E0B94503D94A4538BF4A463C
:10A9B40002E0BA4238BF3A46019F0136BA4238BF74
:10A9C400DE460BF1010B3CBF01924546BBF1040F7F
:10A9D400D6D19844B8F11F0FCCD90CF1010C9C4589
:10A9E400C7D1019ABB2A3FF671AFBDF80C20AEB2B5
:10A9F4009DF808C0C9B2A0F84420A0F84660A0F8A9
:10AA040048E080F84AC080F84B101F2D18D80EEB90
:10AA1400C5021D44A75C02F102086744A75414F858
:10AA240008700F4404F8087002F10308043214F8A3
:10AA340008700F4404F80870A75C0F44A754E4E7B7
:10AA44000123A0F8426003FA0EF280F836201C229B
:10AA540002FA0EFE80F837E0184605B0BDE8F08F24
:10AA6400AB2A01009D7B0020F0B51C4D40F002068E
:10AA7400B0F84040B0F842102F461F292CD855F8A2
:10AA840021204FEA810ED3070AD402F0060C22F0EB
:10AA94001F03BCF1020F0FD1B3F840C064450BD9BA
:10AAA400026047F80E6015E0834213D01A68D2079B
:10AAB40006D41B6823F01F03B3F840209442F3D953
:10AAC4001A46824206D0126832F01F02F9D11A687F
:10AAD40002601E602144D0E7F0BD00BF00400020AA
:10AAE4002DE9F84F0A9F05460E4690469A4602F015
:10AAF40007F80446002800F08A8002F011F8814625
:10AB040028B9204602F004F84846BDE8F88F4FF013
:10AB1400400B60220021204608F06AFD5A460021BD
:10AB2400484608F065FD0123032EC9F80030C9F832
:10AB340008B0C4F810902563636184F835A084F8E4
:10AB4400346010D10B9A39462046FFF77FFE8246C7
:10AB5400002861D1484601F0EBFF204601F0D8FF00
:10AB64005046BDE8F88FB8F1000F08D06B680BB9F8
:10AB74006C6004E09A6B0AB11346FBE79C6316B160
:10AB840000210B4605E02B7D0121012B8CBF002306
:10AB940001236A7D287D42F0704242EA003242EA93
:10ABA400082242EA074242EAC36343EA813194F845
:10ABB4003630616043F08043EA7D43EAC253AA7DA4
:10ABC40043EA024394F8372043EA0223A36036F0B1
:10ABD400020317D1124B44F00201D3F858216AB989
:10ABE400626842F4004262602160C3F85841D3F8BD
:10ABF400402142F02002C3F8402108E0136823609A
:10AC0400116004E0032E204604D1FFF72DFF2046F7
:10AC1400BDE8F88FBDE8F88FB8F1000FB0D0A5E714
:10AC240000022E40F8B590F83430044613F0FD0FBE
:10AC340068D00022614850F822309100DE0711D418
:10AC440023F01F039C4207D123680B500AE021F034
:10AC54001F018C4204D00B461968CD0702D4F6E7D5
:10AC6400216819600132202AE5D1236BB4F84460CD
:10AC74001B7D94F84A70022BB4F8463007D1504932
:10AC8400FF2B25D85A5CD21B5A543344F8E71A4692
:10AC9400B4F848E094F84B5049491F2A18D80EEBF1
:10ACA400C2033244C85C03F1020CC01BC85411F83F
:10ACB4000C00401B01F80C0003F1030C043311F8E1
:10ACC4000C00401B01F80C00C85C401BC854E4E7AE
:10ACD4003C4B1D686DB3AB6A2E6A9C4201D035466D
:10ACE400F8E72846FFF756FA236933F01F0203D02A
:10ACF4009D42F4D01B68F8E79D42F0D0284601F04D
:10AD040017FFECE7036823F01F0398421FD12E4B73
:10AD1400D3F8402122F02002C3F84021D3F8442183
:10AD240012F40042FAD1284BC3F85821274B1D686E
:10AD34006DBB206930F01F0304D0056801F0F8FEF4
:10AD44002846F7E72046BDE8F84001F0E1BE1A685E
:10AD540022F01F02944201D01346F8E762681204FD
:10AD640003D55A6842F400425A6022681A60164BAE
:10AD7400D3F8402142F04002C3F84021D3F84421E3
:10AD84009706FBD52022104BC3F84421CEE7AB6ACB
:10AD94002E6A9C4201D03546CAE72846FFF7E8F9F7
:10ADA400236933F01F0203D09D42F4D01B68F8E7F7
:10ADB4009D42F0D0284601F0BBFEECE700400020A5
:10ADC4009D7B00206465002000022E405C6500200D
:10ADD4000023064A8360436013680BB91060704710
:10ADE4005A680AB11346FBE7586070475065002063
:10ADF400F7B505460F46164601F072FE04460028D4
:10AE040039D02422002108F0F3FB257508230025FE
:10AE1400E675204665752A46A775294600932B4694
:10AE24000195FFF75DFE0646206020B9204601F03B
:10AE34005FFE304620E001F083FE22680F4B206164
:10AE44002046D36301230E4982F835300D4A13702E
:10AE54004FF400230C4A81E80C002B460B4AFFF701
:10AE640017FB0B4A13680BB9146004E09A680AB123
:10AE74001346FBE79C60204603B0F0BD915B0000E5
:10AE8400E05F00203A86002080060001E0570020A1
:10AE9400D8790020F0B50E695EB3D76A18B1335C77
:10AEA4000133DBB200E003461FB37A78032A20D1D2
:10AEB400335400253A7803EB52013129C2BFC3F160
:10AEC40032025200D2B2A91CCCB2A24206EB030455
:10AED40007D9302B0D4604D80133795CDBB2E1701D
:10AEE400F1E70022E2700130C0B2022801D83354E5
:10AEF400F9E7F0BD2DE9F04F2E4F85B00646002549
:10AF04003C68DFF8B8800397DCB1A268BAB9B8F836
:10AF1400003020462168093B0093274BD1F800906C
:10AF24003146C84750B163680DB16B6001E0039AC4
:10AF340013600023A6606360F46038E0254664680B
:10AF4400E2E71E4B1E4DB3F80080A8440935454581
:10AF54002DD26B7895F800A0042B26D1BAF1090FF5
:10AF640023D1039B4FF00009C5EB080B1C68E4B127
:10AF7400A368C3B923680122CDF800B031461B6829
:10AF840020461F462B46B84760B16368B9F1000FED
:10AF940002D0C9F8043001E0039A1360F3686360D7
:10AFA400F460A660A1466468E1E75544CFE705B0C4
:10AFB400BDE8F08F50650020E95700201A7B00207F
:10AFC400E0570020084B094A10B511681878013081
:10AFD4000A46802828BF012022B1547DA042F6D021
:10AFE4009268F9E7187010BD3D860020D8790020DA
:10AFF4002DE9F0410746C06B28B1036839465B6808
:10B00400BDE8F0411847BB6A0B268E4D1C6B237EAE
:10B014000E2B00F21581DFE813F00F0029003E002B
:10B024005900650074008A009300A900B300C900A8
:10B03400D000DD00F6000B012168824B4A68D87904
:10B0440022F0FF6323F4E02343EA00434B60FFF75D
:10B05400B9FF002300047C491A4640F4A0604B6009
:10B0640008602046FFF714FA0123DEE076494FF426
:10B07400901520684B886375426822F07F02134361
:10B08400704A43602046714B81E828000023FFF793
:10B09400FFF90223C9E02B7963766B79A376AB7948
:10B0A400E3766A7A2B7A43EA0223E383EA7AAB7A79
:10B0B40043EA02232384A97BEB7B2A7C6B700B433A
:10B0C40029701343AA7076D0032357E05E49604881
:10B0D400604B614A81E8090000232046FFF7D8F954
:10B0E4000423A2E02B79032B65D96B79032B62D15E
:10B0F400EA79AB7943EA022363842B78E3B105232D
:10B104003CE0504A608C12F8043B4F491B0443F066
:10B11400407343F4D0630B6040F0FF63204643F474
:10B1240080234B600023FFF7B3F906237DE03A4602
:10B1340021460020FFF7AEFE6B78E3B107231DE044
:10B14400404A608C537804323F491B0443F04073F7
:10B1540043F4D0630B6040F0FF63204643F4802344
:10B164004B600023FFF794F908235EE03A4621463A
:10B174000120FFF78FFEAB78EBB10923237646E776
:10B18400304A608C937804322F491B0443F0407397
:10B1940043F4D0630B6040F0FF63204643F4802304
:10B1A4004B600023FFF774F90A233EE03A46214638
:10B1B4000220FFF76FFE267629E723494FF4102378
:10B1C400264A204681E80C0000231E4AFFF760F956
:10B1D4000C232AE01B4A2046D1789378204A43EA7C
:10B1E40001231949B3F5006F88BF4FF4006313803E
:10B1F40013881A4A1B040A604B600023114AFFF7A4
:10B2040047F90D2311E00F4B20460F49DA792277D5
:10B214001A7A62775B791B0443F410630B60002392
:10B224001A464B60FFF734F90E232376BDE8F0810C
:10B234002046FFF75FFE0F2300222376094B1A7086
:10B24400BDE8F081E0570020E05F002080060001A7
:10B25400800600030000FC07E4570020800600027B
:10B264001A7B00203A860020F8B5054600282FD026
:10B27400C4680027174E54B1236820461B699847B9
:10B2840063683268A760626034601C46F3E76C68E8
:10B294002CB1A66B2046FFF7C5FC3446F8E72868B6
:10B2A400FFF7C0FC0C4A136893B1AB420DD1AB68F5
:10B2B4000CB9136000E0A360286908B101F04EFCEA
:10B2C4002846BDE8F84001F013BC1C469B68EBE738
:10B2D400F8BD00BF50650020D8790020F8B50546B8
:10B2E40000F1100400F12006002754F8040F20B1E7
:10B2F4000368A968DB6998472760B442F5D1F8BDB3
:10B30400406910B103681B6A1847704710B5CC0830
:10B3140011F0070100EB040317BF005D0846084164
:10B32400013318BFC1F10801914205D213F8014B52
:10B334008C4008312043F7E707D91F2A9FBF012318
:10B3440003FA02F202F1FF32104010BD2DE9F04F72
:10B35400012A87B004460F461D46DDF840E001D0BF
:10B364000020FAE0BEF1180FFAD91B795A1E012AFF
:10B37400F6D86A79032AF3D1AA79012A02D1EA79A3
:10B38400012AEDD06A7A082AEAD9A97A2129E7D1D3
:10B3940095F80EC0BCF1000FE2D00620032111FB8A
:10B3A4000C018A42DCD102F10906B645D8D300214A
:10B3B40001EB4100284490F80F80B8F1220F0AD124
:10B3C40090F811C0017C41EA0C21B1F5487FA4F842
:10B3D400D01304D9C4E701316145E9D3C0E707219B
:10B3E40011FB03618E45BBD3012B22D1A95D072933
:10B3F400B6D12A44917A0529B2D1117B0329AFD160
:10B4040092F80EE0567BD07A46EA0E2692F80FE0C8
:10B4140010F00F02A4D000F0F0008028A0D138462C
:10B424008DE84040FFF75CFB0023E0602361A684C5
:10B4340077E0AB5D072B93D1AB189A7A052A8FD1AD
:10B444001A7B032A8CD1997B5A7B93F80BA042EA8E
:10B45400012BDA7B1AF00F01049281D01A7C072A9F
:10B464007FF47EAF5A7C052A7FF47AAF93F8139069
:10B47400B9F1030F7FF474AF1A7D9E7C93F81580A5
:10B484009B7D42EA082816F00F0205933FF468AF4B
:10B494000AF0F003802B03931ED116F0F00A7FF418
:10B4A4005FAF049B0A46CDF800B049460193384685
:10B4B4000123FFF715FB059BE060324601934946E3
:10B4C400CDF8008053463846FFF70AFBA4F824B0B1
:10B4D4002061A4F8268021E0039B002B7FF440AF79
:10B4E40006F0F006802E7FF43BAF059B4946CDF86D
:10B4F4000080384601930123FFF7F2FA049BE060D1
:10B50400524601934946CDF800B03846039BFFF7F5
:10B51400E7FAA4F824802061A4F826B02369104A2D
:10B52400DA63E36838460F4A0F49DA630023B4F854
:10B53400D0236361A361E3612362AB7884F8A4360A
:10B54400AB78A16204F1280143EA024304F130021A
:10B55400E3622346FEF79CFF012007B0BDE8F08FAD
:10B564008D610000C76600008106002210B5044604
:10B57400032100F5787001F006FB04F5A0600521B5
:10B5840001F00EFB04F5C860012101F02BFB2046FD
:10B59400BDE81040FFF71CBC70B504460D461148C9
:10B5A400114909F0F0FAD4F87836EA6A60699A42E7
:10B5B40002BF94F8753623F0010384F87536D4F885
:10B5C4007C36EA6A9A4202BF94F8753623F0020385
:10B5D40084F8753628B1036829469B68BDE8704035
:10B5E400184770BD70390020443600200146C06BF6
:10B5F40008B1FFF7D1BF70470023064A43601368C0
:10B604000BB9106070475A680AB11346FBE75860DB
:10B61400704700BF387A0020F8B50B4B05460E463C
:10B624001C687CB123682946AA6820461F683346F3
:10B63400B84728B1022805D1012385F8803601E0F6
:10B644006468EEE72046F8BD387A00202DE9F0471B
:10B65400002400F13005B0F8D08307462646214681
:10B66400A844A1464FF0010A80F8D243454501D3CE
:10B6740000224FE02B78FE2B02D105F20115F5E7ED
:10B6840003F00302022A08D0032A0AD0012A0DBFBC
:10B694006A7801350022023506E0B5F80120033549
:10B6A40002E0D5F8012005354545E1D803F0FC0357
:10B6B400842B14D008D8082B14D0802B28D0042B2A
:10B6C400D4D11FFA82F9D1E7A02B0DD002D8902B48
:10B6D4001ED0CBE7B02B1BD0C02B14D0C6E787F805
:10B6E400D2A3C3E791B2C1E75EB9032C09D841EAFA
:10B6F40009413846FFF790FF07EB84030134E4B2B5
:10B704005861013603E00EB93146AFE7013EF6B2A7
:10B714000021ABE7032C06D8231D013407EB830378
:10B72400E4B25A60F6E7BDE8F087000070B504465D
:10B7340040690D4620B96A6B1D4B9A4237D105E02A
:10B744000368DB6898470028F5D070BDB4F8D0339F
:10B754002A6B9A422BD12046FFF778FF2346A28C0E
:10B7640004F55471E068FEF7FAFE2346A28C04F552
:10B774006471E068FEF7F3FEA06840F24C53C28B9C
:10B784009A4214D1038CB3F51A7F03D040F22F42AE
:10B7940093420CD1074B04F12801074AA3624FF4EA
:10B7A4008023E3622346BDE87040FEF771BE70BD9E
:10B7B400810600222109F4038B3A00202DE9F04F81
:10B7C400B0F8D033002400F13009A3B0A046A3465A
:10B7D4004B442746A2460990159116A811920021C0
:10B7E40030220F9307F004FF059404940E940894F8
:10B7F4000D94039407940C940F9B994580F06681F3
:10B8040099F80030FE2B04D199F8013003339944A0
:10B81400F2E703F00302022A0BD0032A0ED0012A16
:10B824000DBF99F8015009F10109002509F1020938
:10B8340008E0B9F8015009F1030903E0D9F801500F
:10B8440009F105090F99894500F2408103F0FC03D1
:10B85400742B3DD010D8142B24D004D8042B1ED024
:10B86400082B3ED0C8E7242B27D0282B45D0182BF3
:10B87400C2D1ADF8585042E0942B2CD007D8842B79
:10B884002CD0902B00F01A81802BB5D16BE0B02B1B
:10B8940000F01481C02B50D0A02BADD131E0ABB25D
:10B8A4000893A9E7012A01D16BB202E0022A02D16E
:10B8B4002BB20493A0E704959EE7012A01D16BB251
:10B8C40002E0022A02D12BB2059395E7059593E78E
:10B8D4001FFA85FB90E71FFA85F88DE7EBB20D930D
:10B8E4008AE7172F88D81F2D86D922AA7B1C02EB42
:10B8F4004706DFB226F8305C7EE7ADF85A50FF27E2
:10B904007AE7039BA3B9089ABDF8583043EA024387
:10B914000C93079B032B9DBF099A013307994FF0A2
:10B92400000A9FBFDBB202EB81020793D2F814A096
:10B93400039B0133DBB20393C0E0039B002B00F0B5
:10B94400BD80013B13F0FF03039340F0B780BAF1CD
:10B95400000F00F0B380DAF8003050464FF0000AD0
:10B964009B699847AAE0099B93F8D2332BB19DF8C1
:10B9740054300D9A9A4240F0A18015F001030693C9
:10B9840040F08D80BAF1000F00F08980DAF80030C1
:10B994005046059A0C9900922A461B691E46049B40
:10B9A400B04715F0020503D1089B26461F0474E036
:10B9B400182F06D9BDF85A300126BDF85850069301
:10B9C40019E0B8F1010F11D9012F0FD818BF0E9B40
:10B9D4004FF001060CBFBDF8585003F47F454FF6F5
:10B9E400FF7318BF05F58075069304E0069E4FF6B5
:10B9F400FF7335460693089B01220A941B04129395
:10BA04000BF1FF33109302FA03F3139302FA0BF3CF
:10BA14005B42149300230B930B9B43453FD226B107
:10BA2400069B9D420BD26F1C0AE06F1C22AB172FA2
:10BA340003EB450528BF172735F8305C00E02F4697
:10BA4400129B5A460A992B4311980E93FFF75EFCFA
:10BA5400049B0246002BDAF8003007DA10991E29FD
:10BA640004D8139908421CBF14990A435B695046D1
:10BA74000E9998470A9B0E953D465B440A930B9B8F
:10BA840001330B93C8E75A4631461198FFF73EFC41
:10BA9400049B834206DD5E4401354545F3D308FB30
:10BAA4000B440BE0059B8342F5DBDAF8003040EAF7
:10BAB4000701012250465B699847ECE74FF0000309
:10BAC4000027ADF85830ADF85A3095E623B0BDE8FC
:10BAD400F08F70B504464069CD6A0E6B18B10368E7
:10BAE4005B68984748B994F8D233A3B933462A46D9
:10BAF4004FF480712046FFF761FE04F56473A28C55
:10BB0400E0689D4223460CBF294604F55471BDE804
:10BB14007040FEF724BD012EEFD92978731E6A1CEC
:10BB240041F48071E6E70146C06B08B1FFF7D1BF6D
:10BB3400704770B5044600F55876002594F89E3396
:10BB44009D4206D256F8040F08B1FFF78DFB01356C
:10BB5400F4E700251C2204F55970C4F8A4532946BF
:10BB640084F89E53C4F86053C4F8805384F8A153F6
:10BB740084F8A253C4F8A75307F03AFD84F8AB53F2
:10BB840084F8AC5384F8AD5384F8AE5384F8AF53BF
:10BB940084F8B05384F8B15384F8B25384F8B3539F
:10BBA40070BD0000F8B504460D460AB10020F8BD8A
:10BBB4004D49C0F838134D49C0F81813A96921F04C
:10BBC4007F4121F0FF01B1F5106FEFD1E97E022929
:10BBD400ECD880F8982303F1100206981030811AEB
:10BBE40019440F2957D912F8101C092951D112F8F8
:10BBF4000F1C04294DD112F80C1C012949D112F84B
:10BC04000B1C092945D112F8096C022E41D812F8EF
:10BC1400071C07293DD112F8061C052939D112F851
:10BC2400051C01F0F001802933D112F8041C03290A
:10BC34002FD112F8031C01292BD112F8021C41BB8D
:10BC440094F8981312F80DEC12F80E7C31B984F8BC
:10BC5400997312F80D6C84F89A6309E094F899C307
:10BC6400674518D194F89B73B7420FD284F89AE3CE
:10BC740012F8096C84F89B6312F8056C06F00F0641
:10BC840084F89C6312F8016C84F89D63013184F894
:10BC940098131032A3E794F89833002B86D0002130
:10BCA4001C2204F55970C4F8A41384F89E13C4F834
:10BCB4006013C4F8801384F8A11384F8A213C4F8A1
:10BCC400A71307F095FC0A4B04F5627204F556714C
:10BCD400C4F858334FF480132846C4F85C33234621
:10BCE400FEF7D6FB0120F8BD92360020A8360020CE
:10BCF400A006002910B5044607210C3000F036FFD9
:10BD040004F59070022100F03EFF04F5F070042168
:10BD140000F046FF04F53870012100F063FF20466F
:10BD2400BDE81040FFF754B870B504460E4601B3A1
:10BD340090F89E3399421CD890F8A123012592B91A
:10BD44000C4B80F8A153B540C0F858330346C4F8EF
:10BD54005C1300F556718068FEF79AFB94F8AB33D8
:10BD640023EA050503E08D4090F8AB331D4384F8C6
:10BD7400AB5370BD2303080070B590F89E3304469E
:10BD84000E468B4224D390F8A1330125D3B9002960
:10BD940080F8A15300F5617205FA06F514BFA323D8
:10BDA400A023C0F8583341F4802300F55671C0F83D
:10BDB4005C3303468068FEF76BFB94F8AC3323EAEC
:10BDC400050503E08D4090F8AC331D4384F8AC5373
:10BDD40070BD00002DE9F04104460E4607F02AFC30
:10BDE40004F546739E4219D194F8B373B7B3012591
:10BDF400A84694F89E339D4209D808FA05F33B42BD
:10BE040003D029462046FFF7B7FF0135F1E7304656
:10BE140044F62061BDE8F041FEF786BA04F54E739E
:10BE24009E421BD194F8A263C6B1751E254495F8B1
:10BE3400A433082B12D1A368002794F8A303324635
:10BE440084F8A27304EB8604597DFEF7D1FF044BFA
:10BE5400C4F860031F70092385F8A433BDE8F0819A
:10BE64003986002070B504460E4601B390F89E331F
:10BE740099421CD890F8A123012592B90C4B80F863
:10BE8400A153B540C0F858330346C4F85C1300F519
:10BE940056718068FEF7FCFA94F8AD3323EA050581
:10BEA40003E08D4090F8AD331D4384F8AD5370BD6D
:10BEB4002301100070B504460E4601B390F89E337A
:10BEC40099421CD890F8A123012592B90C4B80F813
:10BED400A153B540C0F858330346C4F85C1300F5C9
:10BEE40056718068FEF7D4FA94F8AE3323EA050558
:10BEF40003E08D4090F8AE331D4384F8AE5370BD1B
:10BF04002301110070B504460E4601B390F89E3328
:10BF140099421CD890F8A123012592B90C4B80F8C2
:10BF2400A153B540C0F858330346C4F85C1300F578
:10BF340056718068FEF7ACFA94F8AF3323EA05052E
:10BF440003E08D4090F8AF331D4384F8AF5370BDC8
:10BF54002301120070B504460E4601B390F89E33D7
:10BF640099421CD890F8A123012592B90C4B80F872
:10BF7400A153B540C0F858330346C4F85C1300F528
:10BF840056718068FEF784FA94F8B03323EA050505
:10BF940003E08D4090F8B0331D4384F8B05370BD76
:10BFA4002301130070B504460E4601B390F89E3386
:10BFB40099421CD890F8A123012592B90C4B80F822
:10BFC400A153B540C0F858330346C4F85C1300F5D8
:10BFD40056718068FEF75CFA94F8B13323EA0505DC
:10BFE40003E08D4090F8B1331D4384F8B15370BD24
:10BFF4002301140070B504460E4601B390F89E3335
:10C0040099421CD890F8A123012592B90C4B80F8D1
:10C01400A153B540C0F858330346C4F85C1300F587
:10C0240056718068FEF734FA94F8B23323EA0505B2
:10C0340003E08D4090F8B2331D4384F8B25370BDD1
:10C044002303040010B540F6013390F89A1390F8D6
:10C054009923044643EA014300F55671C0F85C2372
:10C064000022C0F8583303468068FEF711FA012312
:10C0740084F8A13310BD70B505460024012695F857
:10C084009E339C420BD806FA04F3D5F8802313425E
:10C0940003D021462846FFF76FFE0134EFE72B4615
:10C0A40005F56071D5F860030122BDE87040FEF724
:10C0B40056BA0146C06B08B1FFF7DDBF704738B50B
:10C0C40090F8B33304460D462BB944F6206100F5CD
:10C0D4004670FEF729F9012194F8B333A9401943B6
:10C0E40084F8B31338BD012303FA01F190F8B33394
:10C0F40023EA010180F8B313704700002DE9F041F1
:10C10400054614460E4600297AD090F89E3399428B
:10C1140076D84F1E074497F8A423092A70D8DFE87D
:10C1240002F00505121212121236515BE40767D5AC
:10C13400022387F8A433FFF7C2FF31462846BDE83F
:10C14400F041FFF78FBEE0071DD50132D2B2072AB6
:10C1540087F8A42354D12B4B197800294DD12A49AF
:10C164000978002949D10121284619703146FFF781
:10C17400BAFF314687F8A4232846FFF73BFF85F82A
:10C18400A263BDE8F0812846FFF7ADFF33E0A107C5
:10C1940018D53146FFF706FF0823A20587F8A43314
:10C1A40005D414F4806F0CBF0023022300E00123A4
:10C1B40085F8A33305F54E7046F2A811BDE8F041A9
:10C1C400FEF7B2B814F001041AD131462846FFF73D
:10C1D40049FE0C4B1C700EE014F0010410D100EB6E
:10C1E4008108D8F86003FFF73FF8C8F86043314688
:10C1F4002846FFF737FE012300E0062387F8A4331F
:10C20400BDE8F081398600203A86002037B50B4618
:10C2140000225F4D044680F8A1235A6B098FAA427D
:10C2240022D05C4DAA4202D0A32A43D13BE090F82D
:10C234008A3380F89E3390F88B3380F89F3390F8DC
:10C244008D3380F8A03390F89833012B01D9FFF790
:10C25400F9FE012594F89E339D422BD829462046A9
:10C26400FFF762FD0135F5E790F89E33994225D139
:10C27400D0F8603313BB90F89D33012590F89C23CC
:10C28400032101932B4600958068FEF729FC426840
:10C29400414A2346C4F8600304F56071C2632A4628
:10C2A400FEF75DF906E01A6B042A07D1DB6A1A6807
:10C2B400FFF724FF94F8A133002B67D194F8AB1354
:10C2C40049B191FAA1F12046B1FA81F103B0BDE878
:10C2D4003040FFF729BD94F8AD1349B191FAA1F1AB
:10C2E4002046B1FA81F103B0BDE83040FFF7BABD92
:10C2F40094F8AE1349B191FAA1F12046B1FA81F153
:10C3040003B0BDE83040FFF7D5BD94F8AF1349B191
:10C3140091FAA1F12046B1FA81F103B0BDE83040B1
:10C32400FFF7F0BD94F8B01349B191FAA1F120469A
:10C33400B1FA81F103B0BDE83040FFF70BBE94F8C9
:10C34400B11349B191FAA1F12046B1FA81F103B0D8
:10C35400BDE83040FFF726BE94F8AC1349B191FA1A
:10C36400A1F12046B1FA81F103B0BDE83040FFF7F6
:10C3740003BD94F8B21349B191FAA1F12046B1FA80
:10C3840081F103B0BDE83040FFF734BE03B030BDE7
:10C3940023030800A0060029536C0000704790F89E
:10C3A4008432013BDBB280F8843203B943617047C5
:10C3B400A0F10C00FFF7F3BF0123C0F8801280F84E
:10C3C4008532002380F886327047A0F10C00FFF715
:10C3D400F3BFF8B50B0C04460E461B04B3F17F4FB4
:10C3E4003BD089B2002938D0012390F887E200F2CB
:10C3F400862003700023DDB275451CD230F8027F1D
:10C404000133B942F7D142BBD4F87C3213B1D4F82A
:10C414008002984794F88732013BDBB284F8873274
:10C424009D421AD204EB45020135B2F88A12EDB2EC
:10C43400A2F88812F4E782B1D4F8783213B1D4F8B0
:10C444008002984794F88732032B9FBF5A1C03F548
:10C45400A27384F8872224F81360F8BDA0F10C00BD
:10C46400FFF7B7BF002343627047A0F11800FFF73E
:10C47400F9BF8B78834210D0CB7883420DD00B79EF
:10C4840083420AD04B79834207D08B79834204D00C
:10C49400CB791B1A5842584170470120704700005D
:10C4A40038B50D460F220749284609F060F90446BD
:10C4B40030B92A460449054808F065FB204638BDD2
:10C4C400012038BDB7360020C7360020703900205F
:10C4D400A0F11800FFF7E4BF012A73B504460D4626
:10C4E40046D1069A182A43D91879002850D05A7987
:10C4F400032A3DD19A79012A3AD1DA79012A37D12E
:10C504005A7A092A34D19A7A212A31D19A7C072A73
:10C514002ED1DA7C052A2BD11A7D02F0F001802974
:10C5240026D112F00F0221D0597D032920D1D88AB7
:10C53400083838281CD81B7E082628460193012376
:10C544000096FEF7CDFA134AA0652346C26304F1B0
:10C5540064013246FEF703F840F2D943EA8B9A426B
:10C564004FF0000306D140F6213205E010460FE0FB
:10C5740000200DE040F62122E26504F15C0123660F
:10C58400002223462846FDF783FF012084F8910208
:10C5940002B070BDDD750000F8B505460E461848BA
:10C5A4001F461849144608F0EEFA6B6A0BB1B34201
:10C5B40021D16869F8B9AA6802BB04F45F43B3F5F2
:10C5C400A06F1AD114F0400018D06FB10F220E4999
:10C5D400384609F0CCF8044630B90C49084808F04C
:10C5E400D2FA6C622046F8BD0949054808F0CBFA36
:10C5F4006E620120F8BD0020F8BD1046F8BD00BFF2
:10C604007039002007370020B73600203837002063
:10C614006D370020A0F11800FFF7BEBF90F88532F7
:10C6240010B50446E3B190F88632B3B9D0F87C3241
:10C6340083B194F887326BB1013BD4F87C22D4F8EF
:10C644008002DBB284F8873203F5A27334F8131046
:10C654009047EEE7002384F88732002384F885327C
:10C6640010BDA0F10C00FFF7D9BF00000B498B42AD
:10C6740002D00B498B420ED1836893420BD141699E
:10C6840009B18A4207D1436190F88432013380F8BA
:10C694008432012070470020704700BF80000100F1
:10C6A40001000C00A0F10C00FFF7E0BF10B5044638
:10C6B4000221803000F067FA042104F5A07000F034
:10C6C4006FFA012104F5107000F08CFA2046FEF791
:10C6D4007FFB04F10C00FEF78FFF04F11800FDF757
:10C6E40007FD002384F8903210BD0346806868B1CA
:10C6F40093F8912252B940F621311A66D965012185
:10C7040083F8911203F15C01FDF7C2BE012283F8A4
:10C7140090227047002310B580F8913240F62133FF
:10C724004A6B04469A4210D10A6B72B940F621232F
:10C73400026600F15C01C3650123BDE8104080F886
:10C74400913203468068FDF7A3BE94F890322BB172
:10C754002046FFF7CAFF002384F8903210BD7047CB
:10C76400F0B5560619D500242B4D062606FB04F316
:10C774005F5BBA420ED190F8782012F0010F264A7E
:10C78400134401D01A7944E05A88150641D502F0C1
:10C794007F0202E00134102CE8D100231F4D35F84C
:10C7A40023609C00B24203D11C4B23449A7830E0AE
:10C7B4000133192BF3D154062AD490F8783011F0B0
:10C7C400220F4FF0000018BF42F040029B07144BA9
:10C7D40048BF82F0400233F81040A24208D111F061
:10C7E400110F02D000F01F0213E000F120020AE052
:10C7F40001306028EFD100230A4931F81300824246
:10C8040003D103F1A00292B203E00133602BF4D10F
:10C8140000221046F0BD00BFB80E0020540E0020C8
:10C82400581200201813002010B5044680F86E102A
:10C8340080F86F20FFF794FFA36CA4F86C0013B189
:10C84400BDE810401847FFF78AFF10BD0346806813
:10C8540050B1064A03F15C01DA654FF480321A667E
:10C8640003F17802FDF714BE704700BF21090002EE
:10C8740090F8783010B403F001048C4207D061F3CF
:10C8840000035DF8044B80F87830FFF7DFBF5DF8F4
:10C89400044B704790F8783010B4C3F340048C42D2
:10C8A40007D061F341035DF8044B80F87830FFF75B
:10C8B400CDBF5DF8044B704790F8783010B4C3F3E3
:10C8C40080048C4207D061F382035DF8044B80F846
:10C8D4007830FFF7BBBF5DF8044B704710B5532A9F
:10C8E400044680F86E1084F86F2009D190F878100F
:10C8F40001F00101BDE8104081F00101FFF7B8BF6C
:10C90400392A09D190F8781081F00201BDE810406D
:10C91400C1F34001FFF7BEBF472A09D190F8781050
:10C9240081F00401BDE81040C1F38001FFF7C4BFEA
:10C93400FFF716FFE36CA4F86C0013B1BDE81040D8
:10C944001847FFF70CFF10BD2DE9F041044600F134
:10C95400710600F1770700F1640816F8015F032DF2
:10C964000ED941462846FFF784FD48B92A4694F873
:10C9740070102046FFF7B2FF636D0BB1284698474D
:10C98400B742EAD1636D33B904F1650604F16B076C
:10C9940004F170081CE00025012606FA05F394F85A
:10C9A4007020DBB2134208D094F86420134204D1FF
:10C9B40005F16700636DC0B298470135082DECD1CD
:10C9C400E2E741462846FFF754FD58B3B74204D086
:10C9D40016F8015F032DF9D9F3E7236D63B92146F6
:10C9E400A06D082251F8643F23674B6863672346B0
:10C9F400BDE8F041FDF7B3BD0025012606FA05F3B5
:10CA040094F87020DBB2134208D194F864201342E6
:10CA140004D005F16700236DC0B298470135082D95
:10CA2400ECD1DCE72A4694F864102046FFF7FCFEBC
:10CA3400236D002BCAD028469847C7E70146C06B30
:10CA440008B1FFF781BF70472DE9F8430D4604464E
:10CA54001F4990461F4808F096F82B78012B29D1DE
:10CA640004F17107022604F16409B0450ADD17F8E0
:10CA7400012F032A04D949461046FFF7FAFCE0B116
:10CA84000136F2E76E1C05F1070804F17009374618
:10CA940017F8012F032A04D949461046FFF7E9FC89
:10CAA40088B1B845F4D1336801202367736863679C
:10CAB400BDE8F8830020BDE8F88394F870102046A0
:10CAC400FFF70CFFDCE769782046FFF7ADFEE8E7E7
:10CAD4009737002070390020A0F11800FFF7B4BF89
:10CAE400024B186808B102681A6070474865002054
:10CAF400024B1A6818600260704700BF4865002046
:10CB0400024B186808B102681A607047306500204B
:10CB1400024B1A6818600260704700BF306500203D
:10CB2400024B186808B102681A6070475465002007
:10CB3400024B1A6818600260704700BF54650020F9
:10CB4400054B186830B102681A6000230370437003
:10CB54008370C370704700BF4C650020024B1A6895
:10CB640018600260704700BF4C650020242310B594
:10CB740003FB010104468C4204D220462434FFF70F
:10CB8400B7FFF8E710BD602310B503FB01010446AD
:10CB94008C4204D220466034FFF7BAFFF8E710BD98
:10CBA40010B500EB811104468C4204D22046403477
:10CBB400FFF7BEFFF8E710BD08B501210648FFF7EF
:10CBC400D5FF01210548FFF7DEFF04210448BDE835
:10CBD4000840FFF7E5BF00BF08650020A040002023
:10CBE40020410020352310B503FB010104468C428B
:10CBF40004D220463534FFF7B1FFF8E710BD002317
:10CC0400C3600361704770B5B0F84250044690F8B1
:10CC14005230AD0803F0FF0243B1EBB2816B9200D6
:10CC240080F8523003460069FDF799FC94F85330BC
:10CC340003F0FF0253B1EDB22346E16B920084F896
:10CC440053502069BDE87040FDF789BC70BD0000F9
:10CC5400012AF7B504460D4640F0C6801A78092A21
:10CC640040F0C2805A78042A40F0BE8059790129E4
:10CC740002D19A79032A04D00239102940F2B480EF
:10CC84000021089800221844093384F8542084F8B9
:10CC94005520984251D91F78032F40F2A580DE1900
:10CCA400B042C0F0A1805A78042A46D00B2A44D05E
:10CCB400242A0DD19A78511E032902D80121334622
:10CCC400E7E7F12A40F09080DB78022BF6D08BE086
:10CCD400052A2FD1062F40F28780DA78023A012AFA
:10CCE40000F282809A7812F0F00713D0802F7BD163
:10CCF40094F85470002FE2D102F00F0284F854200B
:10CD0400DA7884F856205A791B7943EA0223A4F886
:10CD14004030D4E794F85570002FD0D184F85520D2
:10CD2400DA7884F857205A791B7943EA0223A4F865
:10CD34004230C4E7252AC2D056E0002954D094F8E2
:10CD44005420E2B1B4F84030B4F84A10994216D3F2
:10CD54000020009394F85610012301902846FDF713
:10CD6400BFFEE06068B1234A2346616BC263B4F836
:10CD74004020FDF7F4FB012384F8483001E0002350
:10CD8400E36094F85520BAB1B4F84230B4F84A10CC
:10CD9400994211D3002694F8571028468DE848008C
:10CDA4003346FDF79DFE206140B1134BC36384F805
:10CDB400526084F8536001E0002323610023A4F847
:10CDC4004E30A4F8503084F8593084F85A3084F83E
:10CDD4005B3084F85C30A4F88031E36833B92069AF
:10CDE400003018BF012002E0002000E0012003B061
:10CDF400F0BD00BF997A0000C37A000010B5044664
:10CE0400032100F5F070FFF7BEFE04F54070072122
:10CE1400FFF7C6FE04F598600121FFF7E3FE002347
:10CE24002046C4F88431C4F88831C4F88C31C4F87D
:10CE34009031C4F89431C4F89831C4F89C31C4F8E2
:10CE4400A031C4F8A431C4F8A831C4F8AC31C4F892
:10CE5400B031C4F8B431C4F8B831C4F8BC31C4F842
:10CE6400C031C4F8C431C4F8C831C4F8CC31C4F8F2
:10CE7400D031A4F84E30A4F85030E3602361BDE80B
:10CE84001040FDF7A5BF8A680B6BC2F30E42991AD6
:10CE9400B0F84E30B0F85020890870B50446002030
:10CEA40088420ED0656B55F8205045B1B4F84C60FB
:10CEB4000133B34228BF0023666C46F82350013087
:10CEC400EEE79342A4F85020A4F84E3024BFB4F8FF
:10CED4004C105218013AD31AB4F84020B3EB920F15
:10CEE40006D32346616BE068FDF739FB012300E0BC
:10CEF400002384F8483070BD0146C06B08B1FFF7C9
:10CF0400C2BF7047CB6A826B934203D1002380F87F
:10CF140052307047C26B934202D1002380F85330E1
:10CF240070470146C06B08B1FFF7ECBF704790F83B
:10CF34004030013BDBB280F8403003B98360704776
:10CF4400012380F8423070470B0C89B2092B10B5CD
:10CF54000FD10139072924D8012390F8434003FA5B
:10CF640001F112B924EA010100E0214380F84310E1
:10CF740010BD012B0FD13039082912D8DFE801F098
:10CF840005071011111111110900426410BD8264CA
:10CF940010BDC26410BD0C2B03D1B1F50E7F00D1BE
:10CFA400026510BD90F842302BB1012380F8413066
:10CFB400002380F842307047002383617047A0F15A
:10CFC4000C00FFF7F9BF000070B504460E460E488A
:10CFD40015460E4907F0D7FDA3690BB1B34210D132
:10CFE400A06870B905F45F43B3F5A06F0AD115F0DA
:10CFF400800007D00649044807F0C5FDA66101205A
:10D0040070BD002070BD00BF70390020C7370020FC
:10D01400FF370020A0F10C00FFF7D6BFC2B10B7898
:10D02400022B17D14B78042A80F8433091F902304F
:10D03400436491F90330836407D991F90430052AD4
:10D04400C3641CBF91F905300365012280F84120B7
:10D054001046704700207047A0F10C00FFF7DEBFB8
:10D06400A3F10113012B0BD883680BB19A4207D1AA
:10D0740090F840308260013380F8403001207047DE
:10D084000020704710B50446FEF7B6FA04F10C0010
:10D09400BDE81040FDF72CB82DE9F843089D07467C
:10D0A400164603EB01090C464C450ED03B6832464C
:10D0B40021463846DB6804F10108984730B1204620
:10D0C400099A31464446A847EEE70120BDE8F883B3
:10D0D4002DE9F04105461F4602EB01080C46444584
:10D0E4000DD02B68204606991E6AB8472146024691
:10D0F40028460134B0470028F1D1BDE8F081012071
:10D10400BDE8F0814FF0FF307047704737B50546F2
:10D114000C4606F039FB1C4B984202D800232B80A6
:10D124002EE0694607F016FE9DF806309DF80510BE
:10D13400503B9DF804209BB27F2B0BD80131C9B220
:10D144000C2907D81F2A05D842EA411242EA432390
:10D154009BB200E000239DF802102B8017299DF854
:10D1640001209DF800300AD83B2A08D83B2B06D86A
:10D17400520142EAC12242EA53039BB200E0002377
:10D18400238003B030BD00BFFFA5CE120A46D0F8FD
:10D19400841400B58FB051B1002368468DF8003077
:10D1A4008DF801308DF8023002F0BAFB0DE0D0F8B2
:10D1B400880450B18DF831100B468DF832108DF87B
:10D1C40033100146684600F013FE0FB05DF804FB0F
:10D1D4000A46D0F8841400B58FB071B100236846B4
:10D1E4008DF800308DF801308DF8023002F098FB94
:10D1F400A8B1684602F0D1FA11E0D0F8880470B101
:10D204008DF831100B468DF832108DF8331001462D
:10D21400684600F0EDFD10B1684600F0BDFE0FB0A9
:10D224005DF804FB0A46D0F8841400B58FB079B1D8
:10D23400002368468DF800308DF801308DF80230F7
:10D24400012302F06DFBA8B1684603F0DFF911E099
:10D25400D0F8880470B18DF8311001238DF83210A4
:10D264008DF833100146684600F0C2FD10B16846DF
:10D2740000F04FFE0FB05DF804FB10B5D0F8844405
:10D284008EB00A466CB1002304F5896168468DF8B6
:10D2940000308DF801308DF80230012302F002FCD9
:10D2A40010E0D0F8881461B1012301F58961684662
:10D2B4008DF831408DF832408DF8334000F0B8FFDE
:10D2C40000E008460EB010BDD0F8843430B51546E1
:10D2D4008FB0ABB1002203F5896468468DF8002055
:10D2E40013468DF801208DF802200A46214602F0EB
:10D2F400C3FAD8B12A462146684602F028FC15E054
:10D30400D0F8880490B100F589640A4668468DF81F
:10D31400313021468DF832308DF8333000F00AFD7B
:10D3240020B12A462146684600F0E2FF0FB030BD26
:10D33400D0F8803433B198794FF4007303FA00F0D5
:10D3440080B27047D0F8840408B1D0F83C04704728
:10D3540003460430D3F8842410B512B1D469013CD7
:10D3640004E0D3F888440CB1D4F83044FFF7E0FF6C
:10D37400A4FB000110BD38B50346051DD0F8840494
:10D3840020B1C469013C03F0D9FD08E0D3F8880456
:10D3940020B1D0F8304401F0BAFE00E00446241A6B
:10D3A4002846FFF7C5FFA4FB000138BD38B500F5DA
:10D3B4009265FF23044680F8C41480F8B8342846E4
:10D3C40005F0B8F8C4F88C54284604F08FFC30B942
:10D3D400D4F88C142046BDE8384003F019BF00206F
:10D3E40038BD70B588B0064601A805AD06F29C4468
:10D3F40080E80E0007C885E80B00204695E80E007B
:10D4040004F01EF9C6F88C442CB196F8B304B0FAB3
:10D4140080F0400900E0204608B070BD7FB50C469E
:10D4240005461E4805F08AFCFE2C85F8CD440ED135
:10D434004FF00001281DFFF7B9FF044685F8CC041E
:10D4440040BB2E20032106F06BF9204623E0362C46
:10D454004FF000001FD8124B2E1D8DF805000293CB
:10D46400C5F8C03404AB03908DF8044085F8BD04BE
:10D47400C5F8C404304685F8BC4413E90E00FFF730
:10D48400B0FF20B1D5F89014304603F0C1FE85F802
:10D49400CC0400E0012004B070BD00BFAD7C0000EE
:10D4A40040787D0130B590F8B83485B00446FF2B40
:10D4B40004D190F8C414FFF779FF19E0D0F8BC1434
:10D4C400D0F8C0248DF8043004AB90F8B95402911C
:10D4D4008DF80550039213E90E00FFF782FF38B16F
:10D4E400D4F88C14204605B0BDE8304003F090BE5B
:10D4F40005B030BD2DE9F041D0F890448CB006461B
:10D504001F460CB9002024E0236820469B699847F5
:10D51400B0F5405F8046F5D94FF4007007F0B6FFD0
:10D5240005460028EED0B8F1806F02463B462146FE
:10D5340001A802D901F0AEF901E003F0DBFA0446D8
:10D54400284607F0ABFF002CDCD0301DFFF7AAFF04
:10D5540001200CB0BDE8F0817FB5D0F89064054699
:10D564000EB9002027E090F8CC2490F8CD34BAB15D
:10D57400FE2B05D03368694630469B6B98471AE00A
:10D58400336830465B6C9847421CF3D090B995F8E9
:10D59400CD34FE2BE5D103212E2006F0C1F8E0E7BF
:10D5A400FE2B03D1064B9B689B03DAD5281DFFF79E
:10D5B40079FF00E0012085F8CC0404B070BD00BF01
:10D5C400008000421548164A164BC0F89424164AA7
:10D5D40003600023C0F8A024144AC0F88434C0F8BF
:10D5E400A8240722C0F88834C0F8AC24012280F8AB
:10D5F4009C3480F8B524292280F89D3480F8BA340C
:10D6040080F8C83480F8CC34FF2380F8B724084964
:10D61400084A80F8CD3407F0EEBE00BF0C6000204D
:10D6240010080020E00700207008002000093D00D9
:10D63400AB7C000014390020F0B500F1240385B060
:10D6440005460F4601AC164693E8070084E8070038
:10D654007A012146286A01F0ECFC012805D1324602
:10D664002146286A01F096FC00E0002005B0F0BDD8
:10D6740010B5044600F02AFD002384F8313084F804
:10D68400333010BD38B50D46144600F12401002294
:10D69400006A01F07FFC20B143892B8003890120BB
:10D6A400238038BD38B50D46144600F1240100220C
:10D6B400006A01F06FFC20B1C3892B8083890120AB
:10D6C400238038BD38B50D4690F83110044651B961
:10D6D400382205F08DFF40230120256284F8313083
:10D6E40084F8330038BD002038BD0000F0B40C7855
:10D6F4004D1C202C01D12946F9E71A4F1160916085
:10D704000D460E4615F8014BDCB12F2C13D01F2CFF
:10D7140024D9A4F12201C9B21D2903D827FA01F1A1
:10D72400C9071BD404F0BF013C2917D05C2C0DD1D0
:10D7340014E02F2C05D10E4611F8014B202CF8D102
:10D74400F9E71E601146F0BC01F04EBB2E2C01D14E
:10D754002946D5E7202CFBD09560F9E70020F0BCE2
:10D76400704700BF010100312DE9F84F90F83330C4
:10D7740004460E461546DF0777D5580603D494F8B9
:10D78400313019070CD5D4E90001D4E9042310EB96
:10D79400050841F100094B4508BF424500D2151A5E
:10D7A400A94604F1180AB9F1000F43D0206AD4E95C
:10D7B4000023D0F8381401EA0208C8F3080BB8F1C2
:10D7C400000F1ED1134307D194F831305A064CBFD1
:10D7D400D0F83434E36905E094F833305B0603D5BC
:10D7E400A3690133A3610CE05246A16901F0EDFB8A
:10D7F40000283ADB05D194F8313013F0500F19D1D9
:10D8040033E0276A4FEA5822A16997F845E40239C0
:10D81400D7F82C0401FA0EF1014401EB0208BBF124
:10D82400000F4FD1B9F5007F4CD3D7F81C128845AF
:10D8340004D147E0C9EB0500BDE8F88FB9F5806F66
:10D844002AD301234FEA592B03FA0EF39A1A93456C
:10D8540028BF9346884512D80BEB080399420ED291
:10D8640007F5047005F015FA48B994F832304FF012
:10D87400FF3043F0020384F83230BDE8F88FD7F864
:10D8840014023246414603681F695B46B8470028C4
:10D89400EBD04FEA4B270AE0D7F814023246414650
:10D8A4000368DB6898470028DFD04FF400773E44D4
:10D8B400C7EB0909D4E90023D21943F10003C4E9F1
:10D8C400002370E70022414607F5047005F007FACB
:10D8D4000028CAD0CBF5007700EB0B0130464F454A
:10D8E40028BF4F463A4605F0E9FDE0E7F7B50122C7
:10D8F4000DF1070104468569D0E90067FFF734FF9D
:10D904000128A5610CBF9DF807004FF0FF30C4E962
:10D91400006703B0F0BD2DE9F74F1F4690F831B012
:10D924008369044616460193BBF1000F52D0D0E937
:10D934000089B94508BF904550D056EA070302D183
:10D944000023836143E01BF0080F05D0D0E90401F4
:10D95400B94208BF90423DD3236A16F1FF3093F8D1
:10D9640045A447F1FF3100930AF1090A5FFA8AFAE4
:10D97400524607F045FD94F833200546530603D577
:10D98400E3691D44A56122E018F1FF30524649F1D4
:10D99400FF3107F035FD854202D358EA09030AD165
:10D9A4001BF0400F16BF009BE369D3F83434A36126
:10D9B40004F1180809E02D1AFAE74246A169206A21
:10D9C400013D01F002FB002804DD002DF5D1C4E97E
:10D9D400006703E0019B0020A36100E0012003B085
:10D9E400BDE8F08F2DE9F04F9A4690F831308DB0B4
:10D9F40004460E46154673BB91F8313013F0500FB0
:10DA040029D00AF00303012B00F08281022B40F09D
:10DA14007A8103230AF0080949EA03090DB32B6943
:10DA24004FF00F08002230460E33B3FBF8F808F12C
:10DA3400020800235FFA88F8FFF76DFF4FF0000B30
:10DA44005F46202204A93046FFF78EFE002800F02E
:10DA5400BC80202808D0002084F8310084F83300EA
:10DA640062E14FF00308E9E79DF81020110611D494
:10DA740027B93368203B0193B369009347453CBF02
:10DA84000137FFB212B14FF0000BDAE7002D40F07E
:10DA94009C80E0E7BBF1000F27D1474538BF002742
:10DAA400852ACED13822594620464FF0010B05F085
:10DAB4009FFD9DF811309DF8142084F8303002F059
:10DAC4003703D20658BF43F0080384F83130336A71
:10DAD4002362B36963623368203BA36296F83330F0
:10DAE400C3F3801384F82C30ABE7C02A2BD19DF804
:10DAF400113084F83390980744BF49F0400384F808
:10DB04003330DDE90623C4E90423099BE361DDE93D
:10DB14000A23C4E902231DB91AF4006F9BD126E03D
:10DB24002B682A696B604FF00003AB819DF81330BA
:10DB34009A42A8D1BDF81420AB8AD11AD1F1000BB6
:10DB44004BEB010B7DE7C12A9DD12A4604A920464F
:10DB540001F0CCF808B9834673E7AA89002A7FF458
:10DB640070AF6968AA6891427FF46BAFD4E71AF486
:10DB7400884F03D194F833309A0705D594F831309F
:10DB840013F0110F7FF467AF1AF4806F10D094F87C
:10DB940033309B077FF55FAF002200232046FFF759
:10DBA400BAFE00283FF457AF204600F07FFC08E09F
:10DBB4001AF4804F00F0AE802046D4E90423FFF726
:10DBC400AAFE00283FF447AFA4E01AF4007F3FF414
:10DBD40042AF19F0020F3FF43EAF002D3FF43BAFCC
:10DBE40047451CD2202204A93046FFF7BDFD50B999
:10DBF4003046D6F818A000F088FA00283FF42BAF7E
:10DC0400C6F818A0ECE720287FF425AF27B93368BD
:10DC1400203B0193B36900930137FFB2E0E7382258
:10DC24000021204696F8337005F0E2FC336AC7F30E
:10DC3400801708F1FF3A2362082384F82C705FFAF6
:10DC44008AFA84F831300027009B6362019BA36247
:10DC54002B68AF816B605FFA87FBC3454FD201220B
:10DC640059462046FFF7E8FC064600283FF4F3AE89
:10DC740090F90020002AFFF6EEAE2022002105F0E4
:10DC8400B7FCBBF1000F1ED185233370284B84F8F9
:10DC940030A086F801A01B687BB10DF10B020DF1D9
:10DCA4000E0103A89847BDF80C307381BDF80E30FF
:10DCB40033819DF80B3033751FE045F221437381A6
:10DCC400F381738219E0BBF1010F0CD169F07F037A
:10DCD400C02286F801B0327084F833302B69F370B7
:10DCE400AB8AB38009E0C12306F11E0B3370AA8905
:10DCF40092B96968AA6891420ED10137ABE7204610
:10DD040000F0E4F910E0002B7FF4A5AE012381E6D6
:10DD140002237FE6012007E0284605F0F1F826F803
:10DD2400020F5E45E3D1E8E70DB0BDE8F08F00BF18
:10DD34002C7A0020F0B51F4697B0002305460C4608
:10DD440001928DF851308DF852308DF85330ADF882
:10DD5400143090F831300BB1002047E091F83130A5
:10DD640013F0500FF8D013782F2B12D1019B1A788F
:10DD74002F2A02D101330193F8E7216A1AB9284600
:10DD8400FFF7A0FC32E008A8FFF79CFC0028E3D0D2
:10DD940008AC01AB02AA01992846FFF7A7FC0028AA
:10DDA400DAD0019B1B78DBB1002302AA2146284666
:10DDB400FFF718FE0028CFD008AA2B4605F1300E35
:10DDC40014461868083353F8041C1646734503C6F2
:10DDD4003246F6D1186830602846FFF749FCD8E788
:10DDE4003B4602AA21462846FFF7FCFD17B0F0BDCA
:10DDF40019B101F58961FFF79DBF0846704730B43A
:10DE0400134690F8312072B991F8315015F0500F43
:10DE140009D0D1E90045002504F01F042C4302D1A8
:10DE240030BCFFF7DFBD002030BC704710B50023C5
:10DE34000478CA03012B42EA5101C25C12FA81F14F
:10DE440089B204D1852C14BF0122032200E00122EF
:10DE540013441F2BEDD9084610BD10B5044604F039
:10DE640018FF58B104F5047004F013FF30B1D4F86E
:10DE740040040368BDE81040DB691847002010BD6A
:10DE8400F8B50446006AA16901B10131012200F02C
:10DE9400DCFF0128054601D8002638E001230146AD
:10DEA400206A1A4601F024F806460028F4D0A26934
:10DEB40094F8333022B943F0400384F8333025E03A
:10DEC400590613D50132954220D023F04003E1696D
:10DED40084F83330A369994208D24F1C206A3A4629
:10DEE40001F0C9F80028D7D03946F3E74FF0FF32E4
:10DEF4002946206A01F0BFF80028CDD0A16929B1D4
:10DF04002A46206A01F0B7F80028C5D0A56130463A
:10DF1400F8BD70B590F8333004469A0701D4002058
:10DF240070BDC5690DB9002528E05B0614D5066AE5
:10DF3400D0E9020196F8452410F1FF3002F10902FC
:10DF440041F1FF31D2B207F05BFA0023421C2946AB
:10DF5400304600F0CDFF03E02946006A01F0A8F83E
:10DF64000028E0D1DBE701222046FFF765FB0135FD
:10DF74000028D4D0037803F07F030370E9B294F847
:10DF840030308B42EFD20023206A84F8313084F899
:10DF94003330FFF762FF70BD10B590F8313088B0B0
:10DFA4000446D90601D400201DE000220023FFF717
:10DFB400B2FC202269462046FFF7D6FB38B1202860
:10DFC400F1D19DF800301A06EDD4002BF1D10823CD
:10DFD400204684F8313094F8333043F0020384F857
:10DFE4003330FFF796FF08B010BD00002DE9F34170
:10DFF40000260546DFF8D0803746F1B295F8303078
:10E004008B424AD300222846FFF716FB0446002819
:10E014004FD00378C02B1DD0C12B37D0852B48D1CE
:10E0240095F8313003F037038380D8F8003033B3E8
:10E034000DF103020DF1060101A898479DF8033084
:10E04400BDF806206375BDF80430A281E381228205
:10E05400638214E095F8333013F0400F437814BF13
:10E0640043F0020323F002034370D5E90423C0E91B
:10E074000223EB694361D5E90223C0E906232A6A36
:10E0840092F8103243F0010382F8103239462046E8
:10E09400FFF7CCFE01360746AFE7012205F1240164
:10E0A400286A00F077FF20B14780286AFFF7D5FE81
:10E0B40030B995F83230002043F0010385F832304E
:10E0C40002B0BDE8F08100BF2C7A002010B590F8B2
:10E0D400313004460BB9012010BD90F833301A06D4
:10E0E40007D503F07F0380F83330BDE81040FFF715
:10E0F4007DBF006AFFF7B1FE0028ECD194F83230FE
:10E1040043F0010384F8323010BD2DE9F04190F85A
:10E1140031300446580603D5206A01F091F800E036
:10E12400A068236AD3F83C341844B0F1806F58D205
:10E134002046FFF7A5FE002853D0256A95F8103233
:10E14400D90705D505F5047004F0A3FD002848D0CF
:10E154004FF0FF33002605F508754FF4007245F8BB
:10E16400043C314605F8106C284605F041FA226A51
:10E17400A3694FF0010892F84514023BD2F82C74BD
:10E184008B401F44236A93F8452408FA02F2B242F2
:10E1940009D9D3F840042A46B91903681B6A984779
:10E1A400F8B10136EEE794F83120520614D494F80D
:10E1B400332062F07F02D4E9020184F83320D3F8DB
:10E1C4003C24002380185941C4E90201D4E9040124
:10E1D40012184B41C4E904232046BDE8F041FFF77F
:10E1E40075BF0020BDE8F08110B591F831300446C8
:10E1F40013F0500F1AD040F60223FFF7F3FBA8B137
:10E204001023204684F83130FFF77FFF70B1A369F3
:10E2140020460022E3610023FFF77DFBC123204653
:10E2240084F83330BDE81040FFF750BF002010BD24
:10E23400F0B51F4697B0002305460C460192ADF891
:10E2440014308DF851308DF852308DF8533090F8E9
:10E254003130002B49D191F8313013F0500F44D0B4
:10E2640013782F2B0DD1019B1A782F2A02D1013359
:10E274000193F8E7216A08A8FFF724FA002834D0AC
:10E2840008AC01AB02AA01992846FFF72FFA60B344
:10E29400019B1B781BB3002302AA21462846FFF7E3
:10E2A400A1FB98B108AA2B4605F1300E1446186854
:10E2B400083353F8041C1646734503C63246F6D198
:10E2C400186830602846FFF7D3F9DAE76FB102AA7D
:10E2D40021462846FFF788FF0028E3D105E002AA7B
:10E2E40021462846FFF780FF00E0002017B0F0BD6C
:10E2F400F0B500239DB004468DF831308DF83230EE
:10E304008DF833308DF869308DF86A308DF86B30C4
:10E3140090F8313013F0180F01D100203AE0006A70
:10E324000B6A9842F9D140F601236846FFF702FDD3
:10E334000028F2D00EAA234604F1300716461868C6
:10E34400083353F8041C1546BB4203C52A46F6D1CC
:10E35400186809AA04F12403286007CA83E807009F
:10E364009DF83030204684F8303094F8333063F030
:10E374007F0384F83330FFF7A9FE0028CDD00023B3
:10E384003046159302238DF86B3008238DF86930DD
:10E39400FFF7BFFD1DB0F0BD2DE9F84F1C4690F806
:10E3A4003130064688461B079DF828B09DF82CA0FE
:10E3B4009DF830509DF8349039D5A2F2BC7297B2D2
:10E3C4007F2F34D8631E0B2B31D80BF1FF331E2B58
:10E3D4002DD8BAF1170F2AD83B2D28D8B9F13B0F05
:10E3E40025D8FFF773FE10B34FEA690319F0010F44
:10E3F4004BEA441443EA451508BF4FF0000944EAC8
:10E4040047244FF0000745EACA2518BF4FF06409B6
:10E41400A4B2BB46ADB208F0010AF9B296F83030A6
:10E424008B4234D300223046FFF706F910B900209E
:10E43400BDE8F88F0378852B04D0F8D3C03B012BBB
:10E444001FD9F4E796F83130326A03F0370383803A
:10E4540092F8103243F0010382F81032BAF1000F3F
:10E4640001D00582448218F0020F1EBF80F8149078
:10E474000581448118F0040F1EBF80F81590858132
:10E48400C48159460137FFF7D1FC8346C5E7012211
:10E4940006F12401306A00F07DFD0028C7D0A0F801
:10E4A40002B0306AFFF7D9FCBDE8F88F73B590F875
:10E4B400333004469A0701D4002054E0C569002D86
:10E4C40040D003F04003866903F0FF01F3B1236AEF
:10E4D400D0E9020193F8452410F1FF3002F109025A
:10E4E40041F1FF31D2B206F08BFF421C2EB1013D47
:10E4F400731CAD1B01932A4401E00195E6611AB334
:10E5040000230199206A00F0F3FC19E08EB102AAFD
:10E51400006A42F8041D314600F057FD0028CBDBA9
:10E5240009D04FF0FF32A169206A00F0A4FD10B9B0
:10E53400C2E70195C661019931B1206A00F0B8FDC6
:10E5440010B9B9E701200EE0D4E900232046C4E95C
:10E554000223C4E9042394F8333063F07F0384F87E
:10E564003330FFF7B3FD02B070BD00002DE9F74F63
:10E5740090F83330894604469246990740F1BB80AF
:10E584001A0706D404F11803D0464FF0010B009388
:10E5940062E0D0E90423FFF7BEF90028F2D1AAE033
:10E5A400206A2668D0F838341E40C6F30805002EC9
:10E5B40056D0D4F820E0760AA1699EF845240239A1
:10E5C400DEF82C34914019443144002D7CD1B8F547
:10E5D400007F80F09A80D4E90423D4E900679F4245
:10E5E40008BF964234BF012205220EF5047004F0E0
:10E5F40076FB00287FD0C5F5007628444946464579
:10E6040028BF46463544324604F058FFB5F5007F2E
:10E6140006D1206A00F5047004F03BFB00286AD0A0
:10E62400B144C6EB0808D4E90001821941F10003A2
:10E6340010461946C4E90023D4E904238B4208BFD9
:10E64400824209D294F83330024663F07F0384F89F
:10E6540033300B46C4E90423B8F1000FA0D135E0F0
:10E66400A76937B394F833305B061AD590F845247C
:10E67400E36909320193D2B2D4E9020110F1FF3007
:10E6840041F1FF3106F0BCFE019B1844874205D3DB
:10E694002046FFF7F5FB00288BD12CE00137A7615A
:10E6A40087E7009A394600F090FC002823DB80D1EC
:10E6B400EEE7E36933B92046FFF7E2FBD8B1A3697B
:10E6C400E36176E7A36174E701228EE7D4E90001F0
:10E6D400D4E902238B4208BF824202D2C4E9020178
:10E6E40002E0254B1B6873B194F8333063F07F0369
:10E6F40084F8333007E094F83230002043F001030B
:10E7040084F8323035E0504633E0B8F5806FDEF8F7
:10E714001C72DEF8140214D30BFA02F34FEA582CDD
:10E724009E1B6346B44528BF3346B9424FEA43268D
:10E7340002D8CA18974215D30268556A4A46A847B0
:10E744006CE7B9424A4602BF4FF0FF338EF81052CD
:10E75400CEF81C3203681B6A98470028CBD04FF4CC
:10E7640000765DE74FF0FF328EF81052CEF81C228F
:10E77400E2E703B0BDE8F08F2C7A002083680146FD
:10E78400C3F3080363B100200A69D0540133B3F51D
:10E79400007FF9D1C8680A69036809681B6A1847C9
:10E7A40001207047826803460069C2F3080210B46E
:10E7B4008154586801EB700159609968013199607E
:10E7C40040F2FF118A420AD1D86819680268146AB3
:10E7D4004A1C1A601A6923465DF8044B1847012045
:10E7E4005DF8044B704738B50C46C9B20546FFF7CF
:10E7F400D9FF28B1210A2846BDE83840FFF7D2BF27
:10E8040038BDF8B500240746846080E81200A0B241
:10E8140004F06EFCA04206460AD001463846FFF7D3
:10E82400E2FFA0B3651CB5F5803F0BD22C46EEE7A2
:10E83400651CB5F5803F0AD2A8B204F059FC8542A4
:10E8440005D122E03846BDE8F840FFF797BF2C1BFE
:10E85400B4F5007F0CD34FF6FF713846FFF7C3FFC2
:10E86400A8B1A1B23846FFF7BEFF0028DBD10EE005
:10E874003446A54201D82546D5E7A1B23846FFF76C
:10E88400B2FF01340028F4D101E00135D1E70020C2
:10E89400F8BD00002DE9F04F1F46034687B00D4632
:10E8A400D96014461A610B68019008469B69984721
:10E8B400B0F5801F814607D2002F00F013819249E2
:10E8C4003846F7F70FFC09E10026012301365B0007
:10E8D400F6B2202E05D09945F8D81C2E01D808236D
:10E8E40003E0A6F10B08C8F347031A2E0293029A19
:10E8F4004FF0000186BF013601234FF40053204638
:10E9040088BF76104FF0010B4FF0000888BFB3406A
:10E914000093009B5E009B00C3EB090A0493029BD7
:10E924002AFA03F303FA02FA4FF40072039304F091
:10E934005FFE072384F8BFB184F8C0B1B24484F801
:10E94400C231FE2384F8C181224684F8C331FF23F7
:10E95400C4F8C661414684F8C431284684F8C531F8
:10E964004AF65523C4F8CAA1A4F8FE312B681B6AE1
:10E974009847002800F0B1804FF4007241462046C9
:10E9840004F036FEEB2304F2FD12F4212370762307
:10E99400266463709023C4F84480A3704523C4F8AC
:10E9A40048A0E3705823C4F84C8023714623A6651D
:10E9B40063714123C4F86490A3715423A4F86A805A
:10E9C400E371202384F86EB023726372A372009BF8
:10E9D40084F8708023656365039BE36504232366E1
:10E9E4004FF48073A4F86830092384F86C309DF8E0
:10E9F400083084F86D30802384F86F3004F1770395
:10EA040003F8011F9342FBD14FF000094AF6552346
:10EA1400C846A4F8FE31A9F16A03012B06D9B9F15D
:10EA2400700F1CBF14F8093003EB780809F10109D1
:10EA3400B9F5007FEFD12B682246314628461B6A80
:10EA44009847002849D02B68224606F10C01284635
:10EA54001B6A9847002840D04A460021204606F108
:10EA6400010A04F0C5FD4AF6552306F1090904F22A
:10EA7400FF1BA4F8FE31631E0593059B13F8012FB9
:10EA84009B4502EB7808F9D12B682246514628466B
:10EA94001B6A984708B32B6822460AF10C012846E2
:10EAA4001B6A9847C8B10AF1010ACA45E5D106F1C3
:10EAB4000B0A4FF400720021204604F099FD059BD7
:10EAC40013F8012F9B4502EB7808F9D12B682246F5
:10EAD400494628461B6A984738B91FB10B4938463E
:10EAE400F7F700FB4FF0000AF0E02B68224609F12B
:10EAF4000C0128461B6A98470028EED009F101034F
:10EB0400534505D09946DAE7263800207D380020A1
:10EB1400231F04F5FE7243F8048F9A42FBD12B683D
:10EB24002246514628461B6A98470028D5D02B68B0
:10EB3400224609F10D0128461B6A98470028CCD0CB
:10EB44001FB164493846F7F7CDFA009B4FF40072C1
:10EB5400002120461E44039B4FEA830904F048FD2C
:10EB6400F82309F2072904F113022370FF214FEA65
:10EB7400592A234603F8011F9A42FBD14FEA9939D7
:10EB84004FF00008B8FBF9F309FB138323B91FB155
:10EB940051493846F7F7A6FA2B68224606EB0801D6
:10EBA40028461B6A9847002897D0B8F1000F05D172
:10EBB4004FF400724146204604F01AFD08F10108A2
:10EBC400C245DFD11FB145493846F7F78BFA029B9E
:10EBD4004FF0010808FA03F8039B03F1070A4FEA10
:10EBE400DA0A0AF2FF1B4FEA5B2BD845FFF475AF34
:10EBF4004FF40072002120464FF0000904F0F8FCA5
:10EC0400072323702B682246049928461B6A49442B
:10EC1400984700283FF461AFB9F1000F01D184F89F
:10EC2400009009F10109CB45ECD11FB12C493846BC
:10EC3400F7F758FA009B0198334403EB0809494657
:10EC4400FFF7DFFD00283FF448AF019B9B68B3EB5F
:10EC5400482F3FF642AF1FB122493846F7F742FA30
:10EC64004FF4007200212046002604F0C1FC8122EA
:10EC74000323C14484F82020022223706263822289
:10EC8400C4F838A084F84020019A52686365019B57
:10EC940062649B68E665A3652B68224606EB09015E
:10ECA40028461B6A9847824600283FF416AF2EB9BF
:10ECB4004FF400723146204604F09AFC0136B04508
:10ECC400EAD11FB108493846F7F70CFA504607B0A5
:10ECD400BDE8F08F3C38002063350020B9380020AF
:10ECE40049380020603800206F3800202DE9F041B9
:10ECF40015460E4601F11E08AB8936F8024F43B99A
:10ED04006A68AB689A4204D1B4FA84F04009BDE859
:10ED1400F081284604F0F4F804F0EAF907462046A6
:10ED240004F0E6F9874204D14645E5D10120BDE867
:10ED3400F0810020BDE8F0812DE9F84F90F83130E2
:10ED440082468946002B47D002F1FF380D46022740
:10ED5400002488449AF83030BB4237D30022394625
:10ED64005046FEF769FCB8B30378C12B34D106468C
:10ED740000F11E0B234636F8024F73B104F510520E
:10ED840092B2B2F5806F27D29B021648C4F30904ED
:10ED94001840044304F580300CE004F520539BB282
:10EDA400B3F5006F02D38CB1204603E0B3F5806F56
:10EDB40007D311E04246294604F00DF930B1054667
:10EDC4000024B345D6D10137FFB2C3E70023C9EB12
:10EDD40005002B70BDE8F88F002089F80000BDE81D
:10EDE400F88F00BF00FC0F0070B50B6800240D46BF
:10EDF4004FF6FF764B608C810C61AB891BB96A6856
:10EE0400AB689A4219D0284604F07AF8B04212D07E
:10EE140004F06EF9E30343EA540454FA80F4C4F3AF
:10EE24004E0343EAC433041214FA83F42B69013306
:10EE3400A4B22B61E1E7002070BD2869AC820138DF
:10EE4400FE288CBF0020012070BD2DE9F84F8046BC
:10EE54009246894609B18C1E01E0D0F82044D8F8C6
:10EE640030349C4228BF0024012304F00707C4F374
:10EE7400C80B2646254603FA07F7FFB2D8F82C1428
:10EE84000022404601EB153103F029FF70B33B46E5
:10EE94005946475C1F4205F101050DD1AA1B524595
:10EEA4000BD1B9F1000F04D1BAF1010F08BFC8F8B2
:10EEB4002064B01CBDE8F88F2E46AC4215D0D8F8BB
:10EEC4003024954204D25B0013F0FF03E2D103E047
:10EED40000264FF400713546013101234FF0000B39
:10EEE400B1F5007F1F46D4D3C8E70120BDE8F88FF1
:10EEF4002DE9F84317468A1E0646D0F83004D11986
:10EF04009846814240D8D6F82034B8F1000F09D091
:10EF14009A420BD8994209D9814228BF0021C6F8E8
:10EF2400201403E09A4238BFC6F8202402F00705F3
:10EF34000123D6F82C14C2F3C80403FA05F501EB37
:10EF44001231EDB20122304601F1010903F0C7FE8E
:10EF5400D0B103192A4600F500701978114214BF84
:10EF64000124002444450FD05140013F19700ED0B4
:10EF7400520012F0FF02F0D1013314460122494637
:10EF840098421546E9D1DDE70020BDE8F883012069
:10EF9400BDE8F88338B50D46D0F8381400F5047090
:10EFA4006B6819402B689C1E90F8353204FA03F301
:10EFB40003EB5123D0F81C12194403F090FE18B14E
:10EFC4006B68C3F30803184438BD38B5D0F830343F
:10EFD4000C46154601338B4202D24FF0FF3038BD48
:10EFE400D0F82414002200F5047001EBD41103F0CE
:10EFF40076FE0028F1D0A400C4F308040059286068
:10F00400013018BF012038BD73B5064602AD002497
:10F0140045F8041D2A4601993046FFF7D6FF00281B
:10F0240004DB04F10104F5D1204600E0002002B025
:10F0340070BD70B50D46D0F83844496806460C409A
:10F04400A3180A446A6090F845440934E4B223FAE8
:10F0540004F474B12B7A23B12B6801332B60013C87
:10F06400F7E72A4629683046FFF7AFFF0128F6D0B4
:10F0740070BD012070BD012938B50C46154601D874
:10F08400002038BDD0F8303401339942F8D8D0F894
:10F094002414012200F5047001EBD41103F01FFEC7
:10F0A4000028EDD0A400C4F308040551012038BDA4
:10F0B4002DE9F34107460C460E4601AA214638467F
:10F0C400FFF783FFB0F1000801DA00251BE00022FE
:10F0D40021463846FFF7CFFF05460028F5D0621CCD
:10F0E400B8F1000F02D0019B9A4208D00023921B72
:10F0F40031463846FFF7FCFE0028E6D0019E019C0D
:10F10400B8F1000FD9D1284602B0BDE8F0812DE94D
:10F11400F04100240646D0F82C1400F50477254667
:10F124000022384601F1010803F0D9FD00B300F1D3
:10F13400FF3E05F5805C1EF8011FFF2901D108344C
:10F144000AE049B10822012319424FEA430318BFD8
:10F154000134013ADBB2F7D10835D6F830048542E0
:10F1640002D3001BBDE8F08165454146E3D1D7E7F2
:10F17400BDE8F081F0B54FF0FF330446002587B0B9
:10F184000846E3601146C4F81C3284F8445405ABC5
:10F19400C4F8400404F50872606004F5047725702F
:10F1A400C4F8140284F8105202950195009503F0F6
:10F1B400D1FD10F0FB0F01D100203CE0059E2A4652
:10F1C4003846314603F08BFD05460028F4D01B4930
:10F1D4000522033006F0CBFA01460028ECD195F85D
:10F1E4006C30092BE8D12B6D3344C4F824346B6D97
:10F1F400C4F82834AB6D1E44C4F82C64EB6DC4F819
:10F2040030342B6EC4F8343495F86D300125C4F8CD
:10F214002004204684F8453409332A4605FA03F3CA
:10F22400C4F83C34013BC4F83834FFF70EFE4023E5
:10F23400284684F8443407B0F0BD00BF8D38002060
:10F2440010B50446D0F83414FFF7DEFE94F84534C4
:10F254000933DBB2984010BD10B50446283003F0E2
:10F2640018FD50B104F50E7003F013FD28B12068A9
:10F274000368BDE81040DB691847002010BD024652
:10F2840038B552F8105F04468068294601F0F3FD52
:10F2940078B1A37815B943F0400305E0013522693C
:10F2A400AA4202D023F04003A370A37863F07F0343
:10F2B400A37038BD2DE9F0410378044603F0200320
:10F2C40003F0FF050BB1002635E042691B4B9A425F
:10F2D400F9D8FFF7D4FF06460028F4D0A068052229
:10F2E400216983792830023950F8147C99400F44FD
:10F2F400394603F0F4FC80460028E4D02946012571
:10F304004FF4007204F074F9A3681A79AA420AD976
:10F3140018684246E91903681B6A98470028D2D046
:10F324000135EDB2F0E79A794FF4007393406269C6
:10F3340012FA83F363613046BDE8F081FFFD1F00DC
:10F3440010B5044680680A462830A16903F0C7FC5A
:10F3540020B1A38803F00F0300EB431010BD70B578
:10F36400047805460E4684B92422214604F040F967
:10F37400AE60F379102B03D0202B06D1402300E09C
:10F38400202301202B70A87070BD002070BD38B5FB
:10F39400CB6804460D4623B98968BDE83840FFF7B9
:10F3A400DEBF2422002104F023F91023012023705E
:10F3B400A070AB68A360EB68236238BD2DE9F74FFA
:10F3C4008378044689461646DD0776D50378180700
:10F3D40003D5E36962699B1A07E0990608D5A36817
:10F3E4001A896369C3EB42139BB29E4228BF1E462F
:10F3F40037464FF0000804F1100A002F41D023785B
:10F40400626913F0200FA068C2F308054FEA522185
:10F4140002D0036A194424E090F8058001EA080840
:10F42400BDB9B8F1000F14D122B95A064CBF036A12
:10F43400236A49E01B0705D5A378590602D5236939
:10F44400013341E05246216901F0B2FC002834DB6B
:10F4540013D0A36821699A7902395B6991401944F0
:10F464004144D4F808B0002D4ED1B7F5007F4BD3FA
:10F47400DBF83430994206D146E0237813F0700F5C
:10F484001BD0F01B52E0B7F5806F2CD322787D0A95
:10F49400920606D49BF80420C8EB0202954228BFCA
:10F4A4001546994212D84A1993420FD20BF12800FB
:10F4B400019103F0EEFB019940B963784FF0FF30FE
:10F4C40043F00203637031E02361C2E7DBF82C00F0
:10F4D4004A460368D3F810B02B46D8470028ECD02E
:10F4E4004FEA452B09E0DBF82C004A460368DB6849
:10F4F40098470028E1D04FF4007B6369D944CBEBF3
:10F5040007075B44636178E700220BF1280003F0EE
:10F51400E6FB0028D1D0C5F5007B41194846BB4520
:10F5240028BFBB465A4603F0C9FFE6E703B0BDE86F
:10F53400F08F73B501220DF1070104464669056990
:10F54400FFF73CFF0128666125610CBF9DF80700A9
:10F554004FF0FF3002B070BD436937B5C3F34315B4
:10F56400044605B169B901220DF107012046FFF7F0
:10F5740025FF40B2012801D0002008E063691F3351
:10F5840000E02033A0686361383000EB451003B01D
:10F5940030BD2DE9F0410446076900780E46002885
:10F5A40046D065698D4247D009B921613AE0020726
:10F5B40003D5E36999423BD807E0830605D5A368E0
:10F5C4001B89B1EB431F33D82CE0D4F808E0731E39
:10F5D400A1789EF80620490602F10902D2B223FA64
:10F5E40002F303D5226A134423611BE0691E21FA46
:10F5F40002F2934200D34DB942064CBFDEF82020FC
:10F60400226A22611D4604F1100809E09B1AF9E7F9
:10F6140042462169A068013D01F0CAFB002807DDCC
:10F62400002DF5D1A378666123F02003A37003E0D5
:10F6340027610020BDE8F0810120BDE8F081F8B524
:10F644000F4616460021242204461D4603F0D0FF2F
:10F65400B868A68006F00F0600F138023B6AA06085
:10F6640002EB4612E360D17A0E073FD401F0170192
:10F674002170D37A13F0180F9DF8183008BF41F0A9
:10F684000801E37005F0030308BF2170012B08D0C3
:10F69400022B04D053BB6B0528D4012302E00323BF
:10F6A40000E00223A370A3789F0703D5217811F00B
:10F6B400110F1BD105F008016E0543EA0103A37085
:10F6C400436B918AA361538B43EA014104D589B109
:10F6D40001F011FC70B909E02162D369E3616B04A4
:10F6E4000DD5E1692046FFF754FF40B90020207092
:10F6F400A070F8BDA37863F07F03A370EFE7012047
:10F70400F8BD2DE9F743037806460D469146BBBB89
:10F714000B7813F0700F33D04C6914F01F042FD101
:10F72400274600212846D5F81480FFF715FF38B383
:10F7340003782BB32E2B01D10024F2E7E52BFBD069
:10F74400C27A02F0080E0EF0FF01BEF1000F0FD1D5
:10F75400C4B1421E0A30CB0143EA510112F8013F01
:10F7640053FA81F19042C9B2F5D18F4208D109E030
:10F774000F2AE1D15A06D4D503F01F04477BD0E702
:10F78400002007E000944B46C8F34F122946304648
:10F79400FFF755FF03B0BDE8F08310B503780446C6
:10F7A400DA061FD50021FFF7F4FE01212046FFF7FA
:10F7B400D3FE10B9637853B114E003783BB1E52B61
:10F7C400F3D02E2BF1D0C37A1B07EED40AE0082322
:10F7D40020462370A37843F00203A370BDE81040D1
:10F7E40000F014BF002010BD37B503780446002B89
:10F7F40034D090F90230002B2ADA0121FFF7A0FD62
:10F80400054628B96378002043F00103637026E0BD
:10F814000378E52BF6D023781B0744BFE369C36163
:10F82400236A43831B0C83820E4B1B6863B10DF167
:10F8340003020DF1060101A89847BDF804302B839B
:10F844006B82BDF80630EB82A37803F07F03A370CC
:10F85400A068FFF701FD0028D4D000E0012003B028
:10F8640030BD00BF2C7A002010B50446FFF7BCFF62
:10F8740000232370A37010BDF0B51F4695B000237C
:10F8840006460C4601928DF808308DF809308DF843
:10F894000A30ADF8383003780BB100203EE00B7825
:10F8A40013F0700FF9D013782F2B12D1019B1A7813
:10F8B4002F2A02D101330193F8E7A1681AB930461F
:10F8C400FFF74DFD2AE002A8FFF749FD0028E4D028
:10F8D40002AC01AB0BAA0199304600F04BFE0028A4
:10F8E400DBD0019B1B789BB100230BAA2146304639
:10F8F40000F018FD0028D0D0354602AC0FCD0FC45F
:10F904000FCD0FC42B6830462360FFF7ADFFDFE750
:10F914003B460BAA2146304600F004FD15B0F0BD6D
:10F9240019B101F58961FFF7A7BF0846704770B5A3
:10F9340006460C46FFF758FF054608B900250EE0B9
:10F9440000213046FFF7FCFC0028F7D0214600F1E7
:10F95400200350F8042B984241F8042BF9D128468F
:10F9640070BD30B589B00D4614466946FFF7DFFF18
:10F9740028B1BDF810302B80BDF80E30238009B0BB
:10F9840030BD30B589B00D4614466946FFF7CFFF48
:10F9940028B1BDF818302B80BDF81630238009B08B
:10F9A40030BD2DE9F0410B7888B004460E4613F0C3
:10F9B400700F1CD040F6022300F0B4FCB8B101274C
:10F9C40010252046A7702570FFF774FC78B12369D1
:10F9D400002120462362FFF7DCFD2046FFF704FFE9
:10F9E40028B139462046FFF7ABFC034608B900208E
:10F9F40055E0C57202466F4600F1200C6D46106852
:10FA0400083252F8041CBE466245AEE8030077464D
:10FA1400F5D19F8A2021B3F81A802E238DF8003067
:10FA24000023EA1801330A2B5170FAD1A06801228D
:10FA3400216A837928300239994050F8143C1944DA
:10FA440003F04DF903460028D1D0ADF81470AE464A
:10FA540007460DF1200CADF81A807246083703CA28
:10FA6400624547F8080C47F8041C9646F5D12E2247
:10FA740020338DF80120326A08AE110CADF81A203B
:10FA8400ADF814102A46083303CAB24243F8080CEE
:10FA940043F8041C1546F5D1A068FFF7DDFB08B058
:10FAA400BDE8F081F0B51F4695B0002306460C462C
:10FAB4000192ADF814308DF82C308DF82D308DF87E
:10FAC4002E300378002B3FD10B7813F0700F3BD00E
:10FAD40013782F2B0CD1019B1A782F2A02D10133D2
:10FAE4000193F8E7A1680BA8FFF739FC60B30BACEE
:10FAF40001AB02AA0199304600F03CFD20B3019B02
:10FB04001B78DBB1002302AA2146304600F00AFC30
:10FB140058B135460BAC0FCD0FC40FCD0FC42B68B5
:10FB240030462360FFF7A0FEE1E76FB102AA214649
:10FB34003046FFF736FF0028EBD105E002AA214644
:10FB44003046FFF72EFF00E0002015B0F0BD2DE990
:10FB5400F04303789BB00027044613F0180F88463F
:10FB640091468DF820708DF821708DF822708DF8F3
:10FB740044708DF845708DF8467001D10020B3E0D3
:10FB840082688B689A42F9D12646FFF72DFE11ADA3
:10FB94000FCE0FC50FCE0FC53368394620462B60F4
:10FBA400FFF7CEFB0028E9D003466A4600F12007A0
:10FBB4006D461868083353F8041C1646BB4203C646
:10FBC4003246F6D1227808AE02F0080202F0FF03B2
:10FBD40052B140F601234A4641463046FFF74CFEF7
:10FBE4000028CBD0002707E04A4641463046FFF7BD
:10FBF40059FF0028C2D0109F0E9B01212046A3610B
:10FC0400BDF82430A3809DF82330E3700B9BE360A0
:10FC140000238DF820308DF82230FFF791FB002867
:10FC2400ACD00DF10D0300F10D020DF11D0153F8DF
:10FC340004EB8B4242F804EBF9D1198811809B78CC
:10FC440093709DF80B30C372002F3CD0A068BB1E8C
:10FC54000022817928308B4050F8141C194403F099
:10FC64003EF800288AD000F12003AE4600F1400C93
:10FC74001868083353F8041C7246634503C2964659
:10FC8400F6D13946A06801F036F900283FF476AF82
:10FC9400A0680122216A837928300239994050F8FA
:10FCA400143C194403F01BF800283FF467AF00F13B
:10FCB40020032A46083303CAB24243F8080C43F827
:10FCC400041C1546F5D1002311A8199302238DF8BD
:10FCD400463008238DF8443000F098FC00283FF4A7
:10FCE4004DAFA068FFF7B8FA1BB0BDE8F0832DE96B
:10FCF400F84F1C46037806460F461B079DF828B0AC
:10FD04009DF82C909DF830A09DF8345002D400202A
:10FD1400BDE8F88FA2F2BC721FFA82F8B8F17F0F27
:10FD2400F5D8631E0B2BF2D80BF1FF331E2BEED844
:10FD3400B9F1170FEBD8BAF13B0FE8D83B2DE6D851
:10FD4400FFF752FD0028E2D001213046FFF7F8FA10
:10FD54000028DCD04BEA44146B1044EA4828FC0722
:10FD640043EA4A131FFA88F843EAC92348BFA0F8B4
:10FD74001280B9079BB207D515F00105A0F81080D1
:10FD8400C38118BF642545737A0744BFA0F818805F
:10FD9400C382B068FFF760FABDE8F88F13B58378C3
:10FDA40004469B0701D400202AE0036A3BB301699F
:10FDB40089B102AA0023806842F8043D00F0F8FFEC
:10FDC4000028F0DB09D06FF070422169A06801F0CF
:10FDD40024F810B9E7E701930162019949B963690D
:10FDE4002046E361A37863F07F03A370FFF7FCFC74
:10FDF40006E0A06801F07FF80028F0D1D3E70120E5
:10FE040002B010BD2DE9F84F8378894604461546A3
:10FE1400990740F18E801A070AD46369DB439D4237
:10FE240000F287802F464FF0000A4FF0FF3B46E078
:10FE3400C169FFF7AEFB0028EFD17AE0A068C2F3F6
:10FE44000808467916EA52263DD0D4F808E021691C
:10FE54009EF8063002399940DEF8143019443144D2
:10FE6400B8F1000F48D1B7F5007F6CD26269E3693D
:10FE74009A4243D2A37813F0200F0CBF012205222B
:10FE84000EF1280002F02BFF002852D0C8F50076AE
:10FE940040444946BE4228BF3E46B044324603F081
:10FEA4000DFBB8F5007F05D1A068283002F0F1FE03
:10FEB40000283ED06369B144BF1B33446361626967
:10FEC400002FBBD11CE0B8F1000FBED1216941B1B4
:10FED400A3785B0621D5E3699A421ED201312161E0
:10FEE400B3E7236A33B92046FFF7C9F908B3236996
:10FEF4002362AAE72361A8E70122C1E70522BFE73D
:10FF0400E3699A4201D9E26102E02D4B1B68BBB15F
:10FF1400A37863F07F03A37012E004F1100200F0F1
:10FF240047FF002805DB3FD12046FFF7A8F900284A
:10FF34003AD16378002043F001036370BDE8F88F81
:10FF44002846BDE8F88FB7F5806FDEF83420DEF878
:10FF54002C0014D39EF804309E1B7B0AB34228BFA6
:10FF640033468A424FEA432603D303EB010C62452E
:10FF740015D30268D2F824804A46C04798E78A42DB
:10FF84004A4608BF8EF828A0036808BFCEF834B0EC
:10FF94001B6A98470028CCD04FF400768AE78EF885
:10FFA40028A0CEF834B0E4E7D4F808E021699EF83C
:10FFB400063002399940DEF81430194453E700BF83
:10FFC4002C7A0020411E00F10A020020C30143EAFA
:10FFD400500011F8013F53FA80F09142C0B2F5D1BC
:10FFE400704710B549010446FFF7D3FA28B12046FB
:0CFFF4000021BDE81040FFF7AFBA10BDBF
:02000004600199
:100000002DE9F04F05468DB01646074688469946BD
:1000100003AC0FCD0FC40FCD0FC42B680125236097
:10002000336873600023B3814D451CD8C5EB0801CC
:1000300003A889B2FFF7D7FF834608B900202AE05A
:100040004FF0000A5FFA8AF25946384600F0A4FDE4
:10005000B38904464BB97268B3689A4205D1B0FAC5
:1000600080F0400917E0012015E0304602F04AFF19
:100070000190204603F03EF8019B0446184603F029
:1000800039F88442DAD10AF1010ABAF10D0FD9D157
:100090000135EDB2C8E70DB0BDE8F08F2DE9F04FA6
:1000A00005468DB016468A461F4603AC4FF0010B3D
:1000B0000FCD0FC40FCD0FC42B68002506F116001D
:1000C0002360A846FFF780FF33688146B5817360DF
:1000D000BB4528D8CBEB0A0103A889B2FFF783FF01
:1000E000002843D0059ABB4500F104044FF00001FD
:1000F00092F8283043F0010382F828300CBF4BF00F
:1001000040035B4680F80C8080F80D9003704FF040
:100110000F03A0F81A80C372B38933B97268B36849
:100120009A4202D119E0012020E03046019102F00C
:10013000E9FE0199042902D824F8030C03E00A29F6
:1001400094BF2080608001310234C9B20D29E3D10F
:100150000BF1010B5FFA8BFBBAE725B101354FF6C6
:10016000FF70EDB2E6E728460125E3E70DB0BDE8F4
:10017000F08F024600F120012DE9F04352F8153BC3
:100180002024876802F8014F9142FBD11E782E3E51
:1001900018BF01261D4601332A782E2AFAD07B1E6D
:1001A000AB429E4607D800224FF0070C4FF00809DB
:1001B0001146904610E09EF80020013B2E2AEFD118
:1001C000F1E72B782E2B0AD1AE450CD14FF00A0C5B
:1001D00008214FF010090135BD42F2D344E0222B33
:1001E00013D07C2B11D0A3F12A04052C01D82D2B80
:1001F0000BD1A3F13A04052C07D9A3F15B04022C1F
:1002000003D9A3F121045D2C04D903F0C003802B92
:1002100013D124E0614507D9BCF10A0F23D0AE45C4
:1002200021D30EF1FF351AE0A3F16104192C08D88F
:10023000203B49EA0202DBB209E06145ECD85F23CA
:100240000026A3F14104192C98BF49EA08084C1C68
:100250000144E4B28B75062C03D8047501E0002636
:10026000B9E72146B7E70026837D202B11D03EB1A8
:1002700018EA020F18BF022242750120BDE8F08380
:10028000027D0123437510447E2282753122C2759E
:10029000F3E70020BDE8F0832DE9F84307460E465A
:1002A0000D7D62244FF07E0801F1160903F0C4F9B8
:1002B000032D80B228BF03252B1DDBB200F00F02F7
:1002C000F118013B0009092ADBB294BF3032373202
:1002D0009D428A75F2D373190021384683F816803F
:1002E000FFF759F901213846FFF738F9014628B9D7
:1002F0007878B0FA80F04009BDE8F88303784BB114
:10030000C37A1B07EED40B22484605F023F90028D8
:10031000E8D102E00120BDE8F883601E10F0FF0480
:10032000C4D12046BDE8F8832DE9F04F8BB00E46CE
:10033000924603930B78069013F0700F01D10020C2
:1003400014E1069B1B78002BF9D113690D220C33A5
:10035000B3FBF2F3DBB202939AF815309B0700F07F
:100360000281029B03F1010B5FFA8BFB4FF0000946
:1003700000213046FFF70FF9C8460AF116034C4634
:100380004D46CDF81090CDF8149007937769002171
:100390003046C7F34F17FFF7E1F818B97378002B11
:1003A00060D0CCE70378E52B00D043B9002C08BF20
:1003B000B9465C453CBF0134E4B223B952E05C4528
:1003C00038BF002403E0E52B01D10025DEE72E2B0A
:1003D000FBD0C27A0F2A27D175B903F01F08029A01
:1003E0004245D3D1590602D4DDF80880CEE7437BDD
:1003F00090461546049309E008F1FF385FFA88F843
:100400004345E2D1437B049A9A42DED1B8F1010F11
:10041000BCD1791C2B465246304689B2FFF7F0FD1D
:10042000002808BF0025B1E71307CED44DB1B8F1BD
:10043000010F84D1FFF7C8FD049B83427FF47FAF97
:100440000CE00B22079905F085F800289ED19AF858
:100450001530D80702D50123059397E7039B1905AB
:1004600079D56CE7039B9A057FF569AF03F0030329
:10047000013B012B3FF663AF002C08BFB9465C453A
:1004800002D3059BBBB91DE000213046FFF766F89B
:1004900010B973784BB152E70134E4B2EFE7B368B7
:1004A0001B791C44E4B2A345EBD93046FEF704FFA8
:1004B0000028F4D143E751463046FFF7EDFE00280F
:1004C0003FF43DAF0BF1FF3552463046EDB209EB3C
:1004D00005072B46BFB23946FFF7E0FD00283FF481
:1004E0002EAF39463046FFF77EFD044600283FF424
:1004F00026AF2022002103F07DF8534653F8162F33
:1005000022605A6862601A8922819B7AA3729AF8E3
:10051000153003F018032373164B1B687BB10DF1E4
:1005200023020DF1260109A89847BDF82430238243
:10053000BDF82630E3819DF82330637304E045F273
:100540002143238223836382B26892F8283043F0E8
:10055000010382F8283000953A46039B31460698FD
:10056000FFF76FF802E04FF0010BFFE60BB0BDE8BC
:10057000F08F00BF2C7A0020F7B514461E460846BF
:1005800001310378202BFAD00025204F206003781A
:1005900043B32F2B26D001AA011D02F069FD88B3B9
:1005A000019AB2F5803F2CBF022301237F2A1D440C
:1005B00013D81F2A26D9D3B2A3F12201C9B21D290B
:1005C00003D827FA01F1C9071CD403F0BF033C2B61
:1005D00018D05C2A16D02E2AD9D0202AD7D025614F
:1005E000A060D4E72369013BFE2B0BD8024610F82C
:1005F000013B202BFAD02F2BF8D032602046FFF79A
:10060000B8FD00E0002003B0F0BD00BF01210031C3
:10061000F0B500238BB004468DF804308DF805301A
:100620008DF8063083789A0717D5016A19B180686A
:1006300000F063FC88B101212046FEF783FE0546E9
:1006400058B1FFF7C1FCE526002307462E70237042
:10065000A370A068FEF702FE08B900202FE0E3783F
:100660006BB3214601A8FEF794FE0028F5D00125C2
:10067000E378AB42F1D3A18801A8491B89B2FFF707
:10068000B2FC0028E9D0C37A0F2BE6D1027802F041
:100690001F039D42E1D1437BBB42DED10670A168BE
:1006A00091F8283043F0010381F82830530603D530
:1006B000A068FEF7D3FD02E00135EDB2D8E70BB03C
:1006C000F0BD0000486810B50C4658B10B894A8946
:1006D00001339BB29A420B8104D80349F5F704FD1C
:1006E00000232381206810BD63350020F0B5044647
:1006F00087B00E46154600214FF40072406A02F0A2
:1007000079FF206A10B12049F5F7EEFC636A03AA6D
:10071000E0690393236AE168049300230131ADF893
:1007200014306B09ADF81630036800926A1E9F6A98
:10073000164BB84708B9002024E0206A10B11449CC
:10074000F5F7D2FCF822636A102E4FF0FF001A7002
:100750004FF001030CBF04220C22616AC85401331C
:100760009A42FAD1E069626A0368E1681B6A9847B5
:100770000028E0D0E069E568A1680368626A29445E
:100780001B6A984707B0F0BD3C38002061B20000FA
:10079000B938002038B5446A4FF40072002105468C
:1007A000204602F027FFEB2390222021237076239E
:1007B0006370234603F8022F04F10A0203F8011FB5
:1007C0009342FBD14FF40073A4F80B3095F82B3013
:1007D00063732B8DE38102232374F82363752B69E4
:1007E000E361AB6923624AF65523A4F8FE3138BDB4
:1007F00070B504464FF400720021406A02F0FAFE20
:10080000656A2269216805F2BF1002F09FFBA369A7
:10081000226905F2C31021681A44013A02F096FBDE
:1008200094F82A30002185F8C2312369E069C5F8BF
:10083000C631A369626AC5F8CA314AF65523A5F8DC
:10084000FE310368BDE870401B6A1847F8B54FF4E5
:1008500080730446456AD0F814E090F82B2043607A
:100860006368C3EB0E01B1FBF2F101F20116360A27
:10087000700000F1A107BB420AD3DB1BA66003F1A5
:1008800080062661A1F6F576B6F5704F03D209E031
:1008900080336360E4E7206A002852D02A49F5F7E4
:1008A00023FC4EE081330126E36000F1210326851D
:1008B000204601FB0233B3F5803FA36134BF04231C
:1008C000062384F82A30FFF793FF002839D020460A
:1008D000FFF760FF4FF4007305F135022021A5F802
:1008E0001130A368EB82802385F82430292385F812
:1008F0002630164BC5F8273005F12A0303F8011FEF
:100900009342FBD1462385F83630412385F83730B2
:10091000542385F83830312385F83930362385F86B
:100920003A30E069626A036821691B6A984740B1FE
:1009300062682046E3681021D21ABDE8F840FFF74C
:10094000D5BE0020F8BD00BF9338002087D6120026
:10095000F8B54FF400530446456A03614FF48043F1
:1009600090F82B10436043696268981AB0FBF1F06D
:1009700000F18106F6094FEA460E0EF500570937D9
:10098000BA4203D202F500526260EDE74FF6F4730B
:10099000A660984207D8206A002800F0A08051493C
:1009A000F5F7A2FB9BE0A2F5005300FB01222046D5
:1009B000CEEB03039BB2238503F50053E360A2F55E
:1009C0000053A361484B9A4294BF0B230C2384F835
:1009D0002A30FFF70DFF002800F081802046FFF746
:1009E000D9FEA36805F1510220216B620223EB625C
:1009F00001232B8606236B86802385F8403029232C
:100A000085F84230394BC5F8433005F1460303F809
:100A1000011F9342FBD1462385F85230412385F8CC
:100A20005330542385F85430332385F8553032231E
:100A300085F85630E069626A036821691B6A984745
:100A400000284CD0E06921690368626A06311B6A9C
:100A50009847002843D04FF400720021606A02F0EA
:100A6000C9FD234BE069C5F8FC31036821691B6AA5
:100A7000626A02319847002831D0E0692169036831
:100A8000626A08311B6A984748B31A4BE0692B60C9
:100A900003F1FF53626A03F500532033C5F8E431D4
:100AA0004FF0FF33C5F8E831C5F8EC310368216930
:100AB0001B6A0131984790B1E06921690368626A55
:100AC00007311B6A984750B1A268204694F82B3032
:100AD000202103EB4202BDE8F840FFF707BE0020EB
:100AE000F8BD00BF933800200004FB0087D6120039
:100AF000000055AA5252614138B5036204460B68A2
:100B0000C161426208469B69984700F2FF736061C9
:100B1000DB0A062B236006D8206A10B11B49F5F7C3
:100B2000E3FA002038BD102B01D8022315E0202B5A
:100B300001D8042311E0402B01D808230DE0802BBD
:100B400001D8102309E0B3F5806F01D8202304E019
:100B5000B3F5004F94BF40238023B0F5800F84F895
:100B60002B30204602D2FFF771FE01E0FFF7F0FEC6
:100B70000546206A25B138B10549F5F7B5FA03E015
:100B80000028CED00349CAE7012038BDA73800208D
:100B9000BC380020CA380020042A04D801EB4201E6
:100BA000B1F8010070470A2A03D801EB4201888896
:100BB00070470C2A9ABF01EB4201C8880020704799
:100BC000F8B50E4601781746D1B311F0600407D08E
:100BD000012A35D92F230120337000237370F8BD0B
:100BE0002146FEF7AFFB58B30546214608222346AF
:100BF00008292C7804D1202C1ED010222E240FE09E
:100C0000A4F1410E0135BEF1190F07D890F80CE0A0
:100C100012EA0E0F04D02034E4B201E0202C08D0F8
:100C200003F1010E9C46774506D05FFA8EF306F875
:100C30000C4001310C29DBD100221846F254F8BDDA
:100C400000203070F8BD00002DE9F04F00248BB07B
:100C500003780746894690468DF804408DF8054094
:100C60008DF80640002B5FD0C37813B9FFF7A8FFBB
:100C70005DE0014601A8FEF78CFB002854D008F186
:100C8000FF384D460126C844FB78B34247D3B988A4
:100C900001A8891B89B2FFF7A6F98346002843D033
:100CA000C37A0F2B40D1037803F01F039E423BD140
:100CB00023464FF0000A5FFA8AF259463846FFF79A
:100CC0006BFF044673B100F5105292B2B2F5806F1B
:100CD0002AD29B021748C4F309041840044304F5C0
:100CE00080300BE000F520539BB2B3F5006F01D3C9
:100CF00020B914E0B3F5806F07D315E042462946CA
:100D000002F06BF958B1054600240AF1010ABAF164
:100D10000D0F01D02346CEE70136F6B2B4E700232B
:100D2000C9EB05002B7002E0002089F800000BB031
:100D3000BDE8F08F00FC0F00FFF786BF1368B3F526
:100D4000807F30B51C4628BF4FF4807401EB44050A
:100D5000A94207D231F8020B0028F9D150680130BE
:100D60005060F5E71B1B136030BD1368802B30B556
:100D70001C4628BF802401EB8405A94207D251F804
:100D8000040B0028F9D1506801305060F5E71B1BB7
:100D9000136030BD10B503780446DB0702D501F0BF
:100DA0007AFF30B1002304F1100023704FF0FF33BD
:100DB000E36010BD012970B505460C46164602D801
:100DC0004FF0FF3070BDC3699942F9D8C379202B29
:100DD0000ED18169022200F50E7001EBD41101F0F1
:100DE00080FF0028ECD004F07F0450F824300FE09E
:100DF000102BE5D18369C1F30721022200F50E70A3
:100E0000194401F06EFF0028DAD0E4B230F8143053
:100E1000EA6993429ABF01203360002070BD012926
:100E200038B50C46154601D8002038BDC369994233
:100E3000FAD8C379202B0ED18169032200F50E70F8
:100E400001EBD41101F04DFF0028EDD004F07F0438
:100E500040F824500FE0102BE6D18369C1F307213D
:100E6000032200F50E70194401F03BFF0028DBD08F
:100E7000E4B220F81450012038BD2DE9F341C468D4
:100E800005460E4690468C4207D20C460027013498
:100E9000EB699C4203D9CFB9EC680127F7E7A6427A
:100EA00014D001AA21462846FFF784FF00280DDB55
:100EB000EDD0019B002BEAD107B1EC606FF07042DE
:100EC00021462846FFF7ABFF074608B9002710E088
:100ED0002EB96B6A002B0ADB013B6B6207E02246EE
:100EE00031462846FFF79BFF0028F2D1EEE7C8F80D
:100EF0000040384602B0BDE8F08173B505460C46A7
:100F000001AA21462846FFF755FF061E01DA0020F8
:100F100014E0002221462846FFF781FF0028F6D082
:100F20006B6A002BA4BF01336B62EB689C423CBF31
:100F300004F1FF34EC60019C002EE1D102B070BDE1
:100F40007FB50446406A002821DA002304F50E70BC
:100F500025690393E36901330293FFF71BFF024600
:100F600010B94FF0FF3012E0E3792068202B02AB7C
:100F70000168019301D1074B00E0074B00932B461A
:100F80004E69A169B0470028EBD00398606204B0B5
:100F900070BD00BF07B90000D9B800002DE9F043CB
:100FA0004FF0FF3300270446012600F1280887B0E0
:100FB0000D4691462160C771C660E162436380F8C7
:100FC0002870C4F83C12C0F8443280F838724046A9
:100FD000FFF7E0FE029702460197009705AB4946EE
:100FE000284601F0B9FE10F0FB0F41D0059D3A46AE
:100FF0004046294601F075FE002839D0037C022BBB
:1010000036D1B0F80B30B3F5007F31D132E0013A80
:101010002ED0A6795B000136DBB2A6718B42F6D1E9
:10102000C38A23610BB9436A2361C189B0F81120D7
:1010300029442669228101EB4603A1615101236203
:1010400001F2FF1103EB6121B0F81330616103B9C4
:10105000036A691A1944A379D9404B1CE3614FF024
:10106000FF33636240F6F47399420BD80C23E371AB
:10107000002016E0417B0922A7714B1E217163718C
:101080003346CBE74FF6F47399428CBFC36A102303
:101090004FF00100266384BF23622023C4F840621E
:1010A000E37107B0BDE8F083F8B5002406460D46AD
:1010B00084638F6BC46387B10146242000F0A7F8D6
:1010C0000470447084700446B063AD6B0FCD0FC4E0
:1010D0000FCD0FC42B68236015E0CB6B9BB101468D
:1010E000382000F094F880F8317080F8327080F881
:1010F0003370F063EB6B03F1340253F8041B93423B
:1011000040F8041BF9D13046F8BD10B50446806B99
:1011100010B1FEF7ABFB38B9E06B40B1FCF7AAFAAF
:1011200028B10023E36310BD0023A36310BD00209A
:1011300010BD2DE9F0410446174698460D4611B9F9
:101140000020BDE8F081FFF7E0FFD5F8806496B19C
:101150002146242000F05BF80022434602704270D2
:1011600082703A46A063D5F88014FEF7DBFBE0B14D
:101170000120BDE8F081D5F88434002BE0D0214671
:10118000382000F044F8434680F831603A4680F851
:10119000326080F83360E063D5F88414FCF72AFEEF
:1011A0000028E5D1E063BDE8F081A063BDE8F081EF
:1011B000F8B50D4604461746FFF7A7FFAE6B8EB194
:1011C0002146242000F023F8002202704270827031
:1011D0003A46A063A96BFEF796FA08B10120F8BD64
:1011E000A063F8BDE86B88B12146382000F00FF805
:1011F0003A4680F8316080F8326080F83360E0630E
:10120000E96BFCF7FEFD0028E8D1E063F8BD084675
:1012100070470000F8B500260446C0F8881401465F
:10122000C0F880644FF49060FFF7F1FF012280F86E
:101230004464054680F8796480F87A6480F87B64B9
:10124000C4F88404D4F88814FDF796FF1D4F58B1F4
:1012500005F589663046FCF70DFA29463046FCF75D
:1012600033FA08B1184B22E00026214640F26C40C8
:10127000C4F88464FFF7CBFF0122C671054680F8ED
:10128000486480F8496480F84A64C4F88004D4F85B
:101290008814FFF783FE80B105F589663046FEF7B6
:1012A000E5FA29463046FEF75CF830B1074B1A687C
:1012B00002B91D603C600120F8BD00203860C4F810
:1012C0008004F8BD807A0020347A0020847A0020DF
:1012D00038B504464FF47A750020A560207120735C
:1012E000A064E0642046034D40F8105BFFF721FF47
:1012F000204638BD20070020C07D7047407E7047E3
:10130000036810B41C690123A4465DF8044B6047D0
:10131000807E7047704710B504461C2103F0BAFD6B
:10132000204610BD1FB503686946DB6B9847B0B314
:101330009DF8003013F0C0031FD19DF806009DF802
:10134000073000F003009DF80A209B0043EA802349
:101350009DF8080043EA9010431C9DF8090000F036
:101360000300400040EAD2109DF8052002F00F0271
:101370001044073803FA00F011E0402B0ED19DF81D
:101380000900431C9DF8070000F03F0003EB0040FC
:101390009DF8083000EB0320800200E0002005B03B
:1013A0005DF804FB70B5067E04466EB9051D28463F
:1013B00001F0EFFB3146A07D01F05FFBFF212846E5
:1013C00001F044FC0123237670BD38B5037E04464A
:1013D0006BB1251D0121807D01F04FFBFF212846C7
:1013E00001F034FC284601F0EFFB0023237638BDE2
:1013F00070B5037D0546012B0FD0067E0EB9FFF7B1
:10140000D1FF281D01F00CFCB0F1FF0418BF01242E
:101410002EB92846FFF7D9FF01E0002070BD204615
:1014200070BD00002DE9F843184B044688469146EC
:101430001F681E46051DBFB2284601F0F1FBFF28BC
:10144000607607D133689BB2DB1BB3F5967FF3DD83
:101450001D230BE0FE2801D0182307E04A46414631
:10146000284601F0E3FB607638B125232046E3757A
:10147000FFF7ABFF0020BDE8F883284601F0D0FB62
:10148000284601F0CDFB0120BDE8F883087B002051
:101490002DE9F0411F46037D04460D46022B1646FA
:1014A00002D103698B4208D02368294620461B6D70
:1014B0009847C8B10223256123750025BD4206EB7C
:1014C000452106D023682046DB6C984760B1013582
:1014D000F4E723691D44637D25615BB123682046E1
:1014E000DB69BDE8F04118472046FFF76EFF00209A
:1014F000BDE8F0810120BDE8F0812DE9F0471F46ED
:10150000037D04460D46022B1646DDF8208002D1ED
:1015100003698B4208D02368294620461B6D9847F3
:10152000E8B102232561237505EB06094D450BD073
:1015300041462846B847236801462046DB6C013502
:1015400098470028F2D10AE023691E44637D266192
:101550005BB123682046DB69BDE8F04718472046A9
:10156000FFF733FF0020BDE8F0870120BDE8F087DA
:10157000F8B50A4B0E46071D1D681C46ADB238462D
:1015800001F04EFBFF2806D023689BB25B1BB342E1
:10159000F5DD0020F8BD0120F8BD00BF087B00206C
:1015A0002DE9F341037D04460D4601922BB10368FA
:1015B000DB69984708B9FF2031E0237E13B9204644
:1015C000FFF7F0FE25B14FF496712046FFF7D0FFEC
:1015D000261D0DF107070DF1030845F040013046C7
:1015E00001F034FB17F80119304601F02FFBB84524
:1015F000F8D1002D30464FF00B050CBF9521872107
:1016000001F024FB304601F00BFB304601F008FBF3
:101610000306607603D5013D15F0FF05F5D102B054
:10162000BDE8F08170B504460D461646372100220C
:10163000FFF7B6FF324629462046BDE87040FFF767
:10164000AFBF00002DE9F04788B004464FF0000A14
:10165000DFF8889101AD84F818A084F817A084F809
:101660001AA0D9F8007085E80E009DF804009DF8D6
:101670000560A075DDF8088001F0FCF90121A07D6E
:1016800001F0FBF9544B06F00106A360072386F036
:101690000106E36005AB95E80700251D83E8070018
:1016A00028460ECB01F07EFA6675204684F814A019
:1016B0000A26FFF777FE0121A07D01F0DEF9013E49
:1016C000FF21284601F0C2FA16F0FF06F7D1314695
:1016D0000A26A07D01F0D1F9002220461146FFF72D
:1016E0005FFF0128824612D0013E16F0FF0601D1AD
:1016F000012355E04FF4027AFD21284601F0A6FAB5
:10170000284601F08DFABAF1010AF9D1E4E74FF465
:10171000D57208212046FFF743FF43070ED402236A
:101720000426A376013E284601F07AFA607616F088
:10173000FF06F7D1AA2803D0062331E084F81AA0C7
:1017400023682046BFB29B6C984702280CBF4FF01D
:1017500080460026324629212046FFF763FF824655
:1017600040B1D9F800309BB2DB1BB3F5FA6FF1DD65
:10177000172315E0236820469B6C9847022808D061
:101780002046FFF722FE0723C4F808800120E3600B
:101790001FE052463A212046FFF702FF30B11223E4
:1017A0002046E375FFF711FE002012E0284601F005
:1017B00037FA00F0C000C028284604BF0323A376F0
:1017C00001F02EFA284601F02BFA284601F028FAFB
:1017D000D6E708B0BDE8F087801A0600087B002035
:1017E000F8B500220E463A210446FFF7D9FE30B183
:1017F00012232046E375FFF7E8FD0020F8BD351DF4
:10180000271D384601F00CFA05F8010DB542F8D154
:101810002046FFF7DAFD0120F8BD38B51546002255
:101820000446FFF7BDFE10B11B23E3750AE029460D
:1018300010222046FFF7F6FD054618B12046FFF7B7
:10184000C4FD03E000252046FFF7BFFD284638BD54
:101850000A460921FFF7E1BF0A460A21FFF7DDBF6B
:1018600038B503680D4604469B6C984703284FF033
:101870001201204618BF6D022A46FFF791FE30B1D3
:101880000C232046E375FFF7A0FD002038BD0120A2
:1018900038BD2DE9F0411F46037D04460D46012B5E
:1018A000164602D103698B420AD029462046FFF72B
:1018B000D7FF10B90020BDE8F08101232561237511
:1018C0000025BD4206EB452108D04FF400722046AA
:1018D000FFF7A8FD0028EDD00135F2E723691D448C
:1018E000637D25612BB123682046DB69BDE8F041AB
:1018F00018470120BDE8F0812DE9F0471E46037D21
:1019000004460D46012B1746DDF82080DDF82490B3
:1019100002D103698B420AD029462046FFF7A0FF77
:1019200010B90020BDE8F08701232561237505EB80
:10193000060A55450DD04FF4007239462046FFF790
:1019400071FD0028EDD028464A4639460135C0478A
:10195000EFE723691E44637D26612BB1236820468F
:10196000DB69BDE8F04718470120BDE8F08710B5F6
:1019700000220C210446FFF713FE30B10923204654
:10198000E375FFF722FD002010BD2046FFF71DFD87
:10199000012010BD027D0021022A017502D10368D9
:1019A0005B6D1847012A01D1FFF7E1BF01207047A5
:1019B00038B503680D4604469B6C984703284FF0E2
:1019C0001901204618BF6D022A46FFF7E9FD30B124
:1019D0000E232046E375FFF7F8FC002038BD0120F8
:1019E00038BD7FB503680E4669460446DB6B154675
:1019F000984780B39DF80A305A060CD403F03F0391
:101A00009DF80B205B0043EAD2136A1C3243134259
:101A100001D027231EE0A37E20212046032B1CBFDC
:101A200076026D023246FFF7BBFDC8B92A46212176
:101A30002046FFF7B5FD024690B926212046FFF764
:101A4000AFFD68B942F210712046FFF791FD0546DF
:101A500040B92823E37520460025FFF7B6FC04E0D3
:101A60002623F7E72046FFF7B0FC284604B070BDF8
:101A700038B54FF416710446FFF77AFD054620B1DC
:101A8000FD21201D01F0E2F801E01E23E375204650
:101A9000FFF79BFC284638BD70B5041D1646054669
:101AA000204601F0D3F84FF400723146204601F091
:101AB000D2F8FF21204601F0C9F8FF21204601F0AD
:101AC000C5F8204601F0ACF8687600F01F00052844
:101AD00006D020232846EB75FFF777FC002070BD69
:101AE000012070BD38B50D464FF416710446FFF75E
:101AF0003FFD10B92423E37505E02A46FC2120466A
:101B0000FFF7CAFF18B92046FFF75FFC002038BD79
:101B1000036870B59B6C0D4604461646984703282B
:101B20004FF01801204618BF6D022A46FFF738FD16
:101B300010B10D23E3750AE03246FE212046FFF77F
:101B4000ABFF054618B12046FFF73FFC03E0002538
:101B50002046FFF73AFC284670BD10B4447D1CB106
:101B60005DF8044BFFF7D4BF03685C6A0123A44609
:101B70005DF8044B60470000074B0021074A99635A
:101B8000186B106012681A639A6C22F081029A64D2
:101B9000034B1970704700BF00002C40247A0020CE
:101BA000F5850020064BC3F8CC01C3F8D001C3F87B
:101BB000BC01C3F8C001C3F8C401C3F8C801704731
:101BC00000801F40034B04481B6B1840B0FA80F0A4
:101BD0004009704700002C4001000F00024B586A7A
:101BE00000F00100704700BF00002C40034B586A12
:101BF00080F08070C0F30060704700BF00002C4090
:101C0000014B1878704700BFF5850020034B586AD8
:101C100080F40060C0F3C020704700BF00002C407B
:101C2000034B586A80F48060C0F38020704700BF87
:101C300000002C40034B04481B6B1840B0FA80F0A6
:101C40004009704700002C4002007F114FF47A7366
:101C500006225843224B596AA3F51033D3F80031BA
:101C6000C1F3C22103F03F030131B3FBF2F21D4B7C
:101C7000B3FBF2F30122B3FBF1F1092330B51401F8
:101C8000B1FBF4F4A04202D30124134609E0013B66
:101C9000FAD05200F3E7102C03EB020505D0013413
:101CA0002B46B1FBF3F5A842F5D34FF47A70D2017D
:101CB00043430D4802F47F42B1FBF3F10B4B196033
:101CC000C16A21F47F2323F47F6343F460231A4322
:101CD000631E42EA0313C362436A1B07FCD530BD8F
:101CE00000C00F4000EC695E00002C40DC64002066
:101CF000014B1878704700BF833A0020014B1868E9
:101D0000704700BF247A0020054B03F1100253F8FE
:101D1000040B934241F8040BF9D10120704700BF36
:101D2000CD820020054B03F1100253F8040B9342BF
:101D300041F8040BF9D10120704700BFDD8200207B
:101D4000024B01201B680B60704700BFC879002060
:101D500070470000F8B50746064D01F06DFC0646D9
:101D6000B847044620B101F067FC801BA842F7D9B0
:101D70002046F8BD40420F002DE9F0410C4C0646CC
:101D8000DFF83080206001F057FC0746B047054679
:101D900050B101F051FCC01B404502D90023236023
:101DA00003E003F08DF8F1E720602846BDE8F081FC
:101DB000207A002040420F0010B504460C2103F0A9
:101DC00069F8204610BD000008B50020FFF7EAFEC4
:101DD000084B47F2B80241F2B801C3F8BC23C3F87C
:101DE000C023C3F8AC23C3F8B013C3F8B423C3F8BB
:101DF000B82308BD00801F40054B1B7833B1054B4D
:101E00001B78002B14BF032002207047012070476D
:101E1000467B0020597B002038B5044614480D4607
:101E2000FFF798FFF8B9134BA1029D6007D59A6C94
:101E3000E1B222F0FF029A649A6C0A439A6424F099
:101E4000FF040C4D0C48EC60FFF784FF58B92A6B77
:101E50000A4B1A601A682A631A68D20703D51B68EE
:101E600013F4702F01D0002038BD012038BD00BF11
:101E700079C7000000002C4061C70000247A0020D0
:101E800008B5044B04481968FFF7C6FF08B1034BB7
:101E9000186908BDCC79002000001A0D00002C4004
:101EA00008B5FFF7EDFF80F48070C0F3002008BD97
:101EB000FFF7E6BF7FB5134B0D461968FFF7ACFF80
:101EC000E8B1114B05F10F061A6900925A690192A7
:101ED0009A690292DB690393002323F0030404AAA6
:101EE000144403F003020133D10054F8102C0F2BDB
:101EF00022FA01F206F8012DEFD10023EB7304B0B2
:101F000070BD00BFCC79002000002C40054B186844
:101F100010F0020005D01B6803481840B0FA80F0AA
:101F200040097047247A002000007F11F8B51D4653
:101F3000930706460C46174600D12DB925221A4BA9
:101F40001A704FF4FD7208E01848FFF715FF38B11A
:101F50000A22154B1A7040F2FD12154B1A6020E050
:101F60000122144B2D041A70134A144B2A40186096
:101F700042F40072124B1F605A60124A9A63124B6D
:101F80001B780BB9610200E021463046FFF744FFA1
:101F900038B10E48FFF7F0FE18B9BDE8F840FFF77A
:101FA000B5BF0020F8BD00BF833A00203DCA000045
:101FB000F4640020F58500200000FF1F247A002033
:101FC00000002C4002007F11597B00209DC70000BB
:101FD000174A137813F0C00319D19079D37900F020
:101FE0000300917A9B0043EA8023107A43EA901021
:101FF000431C507A527900F0030002F00F024000B7
:1020000040EAD1101044073803FA00F07047402B23
:102010000BD1507A431CD07900F03F0003EB004015
:10202000137A00EB0320800270470020704700BF46
:10203000DD820020037ADB0708D50A4B1B6803B159
:102040001847094B187860B1FFF72ABF074B1B7878
:102050000BB1FFF7EFBD064B586A80F08070C0F3FC
:1020600000607047207A0020457B00205C7B0020C8
:1020700000002C4070B51646427A0D462AB103681E
:10208000DB699847044600284DD028498B7A03F035
:10209000400202F0FF047AB903F03F03CA7A5B0002
:1020A00043EAD213721C2A43134205D02722204B45
:1020B0001A7040F2EB2227E01E4B1B780BB96D0221
:1020C000760229461C48FFF7A7FE044628B90F22CE
:1020D000174B1A7040F2F32216E031461748FFF70B
:1020E0009BFE044628B91022114B1A7040F2F622CA
:1020F0000AE000211248FFF78FFE044638B911228A
:102100000B4B1A7040F2F9220E4B1A600BE00E488E
:10211000FFF720FE38B12822054B00241A704FF437
:102120003F72084B1A60204670BD00BFDD82002060
:10213000833A0020597B002000001A2000001A2159
:1021400000001B26F46400203DCA000010B50F4CAF
:1021500023780BB9012010BD0D48FFF7FBFD0023CC
:102160000C4A2370116B0C4B19601968116320B96C
:102170001A680A4B1340002BECD01F22084B00209A
:102180001A7040F28122074B1A6010BD5C7B002060
:10219000D1C7000000002C40247A002000007F11ED
:1021A000833A0020F464002038B5174C002117480A
:1021B000A36A23F48033A362FFF72EFE054638B9E5
:1021C0000922134B1A7040F24222124B1A6019E096
:1021D0001148FFF7D1FD40B10A220D4B00251A70BE
:1021E00040F246220B4B1A600CE0636A9B0709D54C
:1021F000616BA36AE26A23F4803342F08062E26298
:102200006163A362284638BD00002C400000DB0C4F
:10221000833A0020F464002089C7000038B50C46DA
:10222000FFF794FF0546002830D0194B5A6AD105B4
:1022300007D49A6A22F480329A629A6A42F400328F
:102240009A629A6A134842F480329A62FFF782FDDA
:10225000A0B9231F0E4904F5FE744A6A5205FCD545
:1022600003F1400253F8040F9A420862FAD19442F3
:102270001346F2D10122084B1A7007E02122074BC6
:1022800000251A7040F2F732054B1A60284638BD17
:1022900000002C40BDC700005C7B0020833A00207A
:1022A000F464002010B514480C46FFF765FD40B1FA
:1022B0000A22124B00201A7040F25F42104B1A6043
:1022C00010BD104B9A6A22F480329A624FF4007269
:1022D0005A600D4B1B780BB9610200E021460B4898
:1022E000FFF79AFD30B90E22044B1A7040F26B4290
:1022F000034B1A6010BD00BF3DCA0000833A0020A6
:10230000F464002000002C40597B002020003A1982
:10231000F8B507460C4615463E7AF6071DD59607D2
:102320000FD0CE18B44227D03B682A462146384603
:102330001B6A984708B90020F8BD013405F50075FF
:10234000F0E70E48FFF7F2FDB0B90E220C4B1A7001
:1023500040F251420B4B1A60F8BDCE18B4420BD07C
:102360003B682A46214638461B6A0134984705F5E2
:1023700000750028F2D1DEE70120F8BD27003A19E8
:10238000833A0020F464002070B5037A1546ADF559
:10239000007D0446DA070E4618D5AB0706D029465D
:1023A0006D464FF40072684601F08AF801232A4610
:1023B00031461A48FFF7BAFD00282CD10D22184BE0
:1023C0001A7040F21942174B1A6024E0FFF7BEFE64
:1023D00008B900201FE0637A022B02D163689E4295
:1023E0000FD023682046DB6998470028F1D0236886
:1023F000314620461B6D98470028EAD002236660CC
:102400006372236829462046DB6C98470028E0D099
:102410006368013363600DF5007D70BD01003A18FB
:10242000833A0020F4640020F8B507460C461546B0
:102430003E7AF6071DD596070FD0CE18B44227D0A6
:102440003B682A4621463846DB68984708B9002091
:10245000F8BD013405F50075F0E70E48FFF766FD9D
:10246000B0B90C220C4B1A704FF464720B4B1A600B
:10247000F8BDCE18B4420BD03B682A4621463846F8
:10248000DB680134984705F500750028F2D1DEE7D6
:102490000120F8BD37003A12833A0020F46400208E
:1024A00038B504461A480D46FFF754FC28B10A22F5
:1024B000184B1A7040F29D1220E00122164B214663
:1024C0001A70164B164A1860164B17481D605A6052
:1024D000164A9A63FFF7A0FC38B904220D4B1A7014
:1024E0004FF4D272124B1A6038BD1248FFF744FC09
:1024F00040B12522074B1A7040F2A7120C4B002066
:102500001A6038BDFFF702FD0028F2D038BD00BFC9
:102510003DCA0000833A0020F5850020247A00207F
:102520004000010000002C4011003A0602007F111B
:10253000F46400209DC700002DE9F04300230172E0
:102540009F4F91B09F49A04DA04E437205202B7024
:102550003B700B7033709E4BD3F8002142F0800229
:10256000C3F80021D3F8002122F03F02C3F8002174
:10257000D3F8002142F01802C3F80021D3F800215B
:1025800022F08002C3F8002103F51033D3F8802035
:1025900042F00C02C3F880205A6A22F460525A6258
:1025A000DA6942F48032DA615A6A42F400625A62AD
:1025B000FFF7F8FA874B88469A6C42F000429A641B
:1025C000DA6A42F0807242F40042DA62DA6A814CDE
:1025D000D101FBD44FF4C870FFF738FBFFF7F4FBD1
:1025E0007D4B7E4A63637E4BC3F8F82160227D4BAE
:1025F0001A70A3F262334FF480421A60E36A43F028
:102600000063E362E16A11F00061FBD10846FFF765
:1026100003FC044620B9012340F296222B7048E0C7
:1026200003244FF4D5717048FFF7F6FB60B1694B96
:102630001B69B3F5D57F04D006234FF427722B70A6
:1026400085E00123337001E0013CEAD13378674C27
:10265000002B674E08BF4FF4401400F0EDFF814699
:1026600000216448FFF7D8FB002867D02146624864
:10267000FFF7D2FB002861D000F0DEFFC9EB0000BD
:10268000B0425BD8534B1A69002AE9DA19695B4AF0
:102690005B48116000211B695A0044BF012388F880
:1026A0000030FFF7B9FB044630B902234FF42C7217
:1026B0002B70544B1A607EE000215348FFF7ACFBAF
:1026C000044620B9032340F2B3222B70F1E7414EB8
:1026D000DFF8548133694D491B0C4D481B04C8F881
:1026E0000030FFF7E7FB044620B907234FF42E72B2
:1026F0002B70DEE747494848FFF7DCFB044620B96A
:10270000082340F2BB222B70D3E7D8F800104348CF
:10271000FFF782FB044620B9052340F2BE222B704E
:10272000C7E7D8F800103348FFF776FB58B102210D
:102730003B48FFF771FB044628B10CE0172340F239
:10274000A7222B7003E0142340F2C2222B702D4BE2
:1027500000241A602FE0B36A69466FF07F4023F0CF
:102760000603B362B36A43F00203B3624FF010137F
:102770007364FFF795FE18B19DF80D309B0702D4E6
:1027800046F2A8120DE069462648FFF789FE0028A8
:10279000F6D09DF8103003F00F03012BF0D14CF26E
:1027A00050320520FFF7FEF91046FFF74FFAFFF70A
:1027B0000BFB01233B70204611B0BDE8F08300BF46
:1027C000457B0020597B0020833A0020467B002077
:1027D00000800D4000002C400B007F1115C7000049
:1027E000003C00206EE400E000001A0800003040C9
:1027F00040420F0000001A3700000229C87900206B
:1028000000000902F464002000001A03DD820020A9
:1028100000000909CD8200200000090A00001B0702
:1028200000001A06F1FFFF80CC790020264B5A6A7F
:1028300070B596050C460DD49A6A22F480329A62DD
:1028400072B69A6A42F400329A629A6A42F480320C
:102850009A6262B61D48FFF77DFA58BB1A49231FDA
:1028600004F5FE7408464A6A1505FCD503F14002DA
:10287000066A154D43F8046F9A42F9D19442134603
:10288000F1D11348FFF766FA28B11D22114B1A70D7
:1028900040F24E3213E02A6B0F4B1A601A682A631B
:1028A0001A6892070ED51B680C481840B0FA80F0E1
:1028B000400970BD1A22074B1A7040F24332084B90
:1028C00000201A6070BD00BF00002C40A9C70000A6
:1028D000D1C70000833A0020247A002000007F1135
:1028E000F464002010B514480C46FFF745FA40B1D7
:1028F0000A22124B00201A704FF46872104B1A60B3
:1029000010BD104B9A6A42F480329A624FF4007202
:102910005A600D4B1B780BB9610200E021460B4851
:10292000FFF77AFA30B90C22044B1A704FF46B722D
:10293000034B1A6010BD00BF3DCA0000833A00205F
:10294000F464002000002C40597B002030003A1233
:1029500070B5037A1646ADF5007D0446DA070D46DC
:102960001CD5B30721484FF001030CBF34466C4619
:102970002246FFF7DBFA054638B90B221C4B1A70CA
:1029800040F261321B4B1A602CE0B4422AD04FF463
:1029900000726946304600F093FD23E0FFF7D6FB56
:1029A00008B900251EE0637A012B02D163689D42BD
:1029B0000ED023682046DB6998470028F1D02946CD
:1029C0002046FFF78FFF0028EBD00123656063727C
:1029D00031462046FFF72AFF05460028E1D063680C
:1029E0000133636028460DF5007D70BD11003A117A
:1029F000833A0020F464002070B5124A00250E4688
:102A000045722946936A104823F480339362FFF796
:102A100003FA044638B909220C4B1A7040F2C2324C
:102A20000B4B1A600CE05EB10A48FFF7A5F938B10C
:102A30000A22064B2C461A7040F2C632044B1A602A
:102A4000204670BD00002C400000DB0C833A0020C3
:102A5000F464002089C7000010B50446FFF776FB38
:102A600038B1637A2BB120460121BDE81040FFF751
:102A7000C3BF10BD012100F055BE00F021BE000013
:102A800013B502AB03E90600C37C0099002B2ED0DE
:102A900072B6C37CDA0705D5324A4369146823400D
:102AA00083621360C37C9B0705D52F4A8369146832
:102AB0002340C3621360C37C5C0705D52B4AC369FE
:102AC0001468234003631360C37C1A0705D5284AA2
:102AD000036A1468234043631360C37CDB0605D597
:102AE000244A436A146823408363136062B6836890
:102AF0008B422AD0204B81609A69204BC2F301148B
:102B0000C2F3826253F824300132B3FBF2F211B106
:102B1000B2FBF1F300E013467BB1B2FBF3F291425A
:102B200038BF0133B3F5817F02D2022B04D901E013
:102B300040F20113023B00E000235A0843EA02235B
:102B4000120402F47F021343C360036800221A6177
:102B500003225A62C2681A64019A1A6601221A6133
:102B600002B010BD80E100E084E100E088E100E017
:102B70008CE100E090E100E000C00F40C8080020B8
:102B800003685966DA6D12F4F81FFBD0586FC0B2B3
:102B9000704708B5031D006893E80600FFF770FF53
:102BA00008BD00001FB50DF1100E0EE90E00039BCD
:102BB00003B9044B0360006805B05DF804EB00F056
:102BC000FDBA00BF203900200368DA7CE2B1D107EA
:102BD00002D5996A0D4A1160DA7C920702D5D96A4A
:102BE0000B4A1160DA7C500702D5196B094A116053
:102BF000DA7C110702D5596B074A1160DA7CD206DC
:102C000002D59A6B054B1A60704700BF00E100E0E7
:102C100004E100E008E100E00CE100E010E100E088
:102C200008B5FF210068FFF7ABFF08BD70B50C4683
:102C300016460546FF21204600F0DCFC2868334696
:102C40002246214600F0C6FB002070BD08B5006892
:102C5000FFF796FF08BD531EB3F5007F70B506461B
:102C6000ADF5007D0C46154609D2684600F028FCFB
:102C70002B466A466946306800F0ACFB08E00D441C
:102C8000AC4205D014F8011B3068FFF779FFF7E775
:102C90000DF5007D70BDF8B503780446DA071DD543
:102CA000406804F11006E168036832461B6A9847E1
:102CB000054608B9002512E023789B0704D4237841
:102CC00023F0010323700AE0201D324683C8036805
:102CD00039441B6A98470028F1D1EBE701252846C3
:102CE000F8BD436870B504460E4615460BB9002082
:102CF00070BDC3688B4213D0FFF7CDFF0028F6D01C
:102D00006B0703D50023E660237009E0606804F1D7
:102D1000100231460368DB6898470028F2D1E6E7E5
:102D2000237805F0030520461D4300F8105B70BDB5
:102D300000231370014B1B68184700BF307A002036
:102D4000024B034A1A60034B186070472C7A00202C
:102D5000CDD80000307A00202DE9F74F0CAE0546A3
:102D600014469A46019196E8C00109B90020C2E0D4
